:020000040000FA
:1000000092EF01F01200FFFF10EF04F01200FFFF6B
:1000100000000901C80E926F66806650010B06E071
:100020000901925103E009019207F7D7120000007D
:100030000901C80E926F66846650040B06E0090140
:10004000925103E009019207F7D71200D9CFE6FFDA
:10005000E1CFD9FF3F0E6816676A666AFE0EDB5075
:100060006712FD0EDB506812678AE552E7CFD9FFB1
:100070001200D9CFE6FFE1CFD9FFFE0EDB506A6E4A
:1000800067AE02D0FF0E30D00F0E671408080CE0E8
:100090000F0E67140B0808E06850040B03E168506A
:1000A000010B1FE0000E20D00F0E6714080804E0BB
:1000B0000F0E67140B0818E10901C80E926F685003
:1000C000010B04E0925102E09207F9D76850040B4B
:1000D00001E0010E496E1F0E66144910F7E166AC8F
:1000E00002D0FE0E01D0000EE552E7CFD9FF12007C
:1000F000D9CFE6FFE1CFD9FF0000FE0EDBCFE6FF50
:10010000B8DFE552006E005003E091DF005000D0F0
:10011000E552E7CFD9FF120000007ADF700EE66EDD
:10012000E7DFE552000901E028D0800EE66EE0DF4F
:10013000E552000901E021D0E66ADADFE552000964
:1001400001E01BD0400EE66ED3DFE552000901E06E
:1001500014D0016A1E0E015C0FE20150EA6A000F22
:10016000E96E060EEA22EF50E66EC2DFE5520009A4
:1001700001E003D0012AEED75ADF12000000016A25
:100180001E0E015C09E20150EA6A000FE96E060EDC
:10019000EA22EF68012AF4D712000000016A1E0E5D
:1001A000015C09E20150EA6A000FE96E060EEA22DC
:1001B000EF6A012AF4D712000000EFDFE66A080EAA
:1001C000E66E44DFE552E552090E696E21DF700EDE
:1001D000E66E8EDFE552000901E01CD0800EE66E6F
:1001E00087DFE552000901E015D0C80EE66E80DF1A
:1001F000E552000901E00ED0E66A7ADFE552000917
:1002000001E008D0E00EE66E73DFE552000901E080
:1002100001D00DDF12000000CFDF0601050E026FD6
:100220000601340E036F0601460E146F0601050E1B
:10023000176F0601040E186F0601640E196F060190
:10024000010E1A6F0601670E1B6F0601020E1C6F6E
:100250000601600E1D6F60DF1200000037D836D82F
:100260008D8A8D8C84848C80120009018E6B09012B
:100270008A07000E8B5B09018D5109018C5D04E03A
:1002800084948C908D9A8D9C8E2FFED709018D5170
:1002900009018C5D06E009018CB18C8009018CB3E9
:1002A00084848E2FFED78CC98DF9120000000900BE
:1002B000F5CF89F90900F5CF88F9090188510901BD
:1002C00086270901895109018723120000000901CD
:1002D000886B896B0901540E885D3D0E895905E2D2
:1002E0000901882B000E8923F5D7120000000901AF
:1002F000886B896B0901220E885D060E895905E21B
:100300000901882B000E8923F5D7120000008250C6
:10031000010B03E08250020B02E1010E02D0000E3D
:1003200000D01200C16A0F01DF0E256F0F01F70E1A
:10033000246F0F01E00E236F3A0EC06EEF0E896E30
:100340008A6A8B6A9E0E8C6E900E8D6E8E6A8F6A94
:10035000010E906E916AEF0E926E070E936E930EE1
:10036000946E600E956E030E966E7F0E976E060E5F
:10037000986EFE0E996E9A688A8AC79EC698C78C38
:10038000F00EC616C680C68A240EAC6E190EAF6E6D
:10039000900EAB6EF29EA698636AFE0E626E010E20
:1003A000616E7F9E7F9C7F84550E7E6EAA0E7E6E50
:1003B0007F82F28E01DFB0DE50DF0901916BA6DF94
:1003C000000904E10A0E0901915D09E2640E0901C8
:1003D000915D05E27BDF7ADF0901912BF0D77F94F5
:1003E00009019151630802E216EF02F00901866BE0
:1003F000876BF66A080EF76EF86A58DF000009018D
:100400008851891102E102EF04F050DF800EF618E6
:1004100005E1FD0EF71802E1010EF81801E0F5D72D
:1004200009018651871102E102EF04F001D81200A0
:10043000F2DE09018C6B09018BA703D00901010EC3
:100440008C6F13DF9EAA17D0AECF8FF9490E09012A
:100450008F5D0AE14B0EAD6E49DF580EAD6E46DF83
:10046000330EAD6E43DF02D08FC9ADFF440E0901DC
:100470008F5D01E101D0DDD709018A6B8B6B09012A
:10048000020E8C6F09018AA902D009018C6BEDDE86
:100490002FD8020EF85C05E1420EAD6EF86A0ED858
:1004A000FF000CD8410EAD6EEAD712000000550EC9
:1004B0007E6EAA0E7E6E7F8200001200940E7F6E0A
:1004C000F5DF000EE96E090EEA6E0A000901100E52
:1004D000846F0901080E856FEE50F56E0F00852FB1
:1004E000FBD7840E7F6EE2DF842FF3D77F94120058
:1004F00000000901906B0901846B09018451496E68
:100500004A6AD8904A5004E6840E495C000E4A5864
:1005100014E29EAAFED7AECF8FF909018451EA6A90
:10052000000FE96E090EEA228FC9EFFF09018F5112
:10053000090190270901842BE0D7090190510BE1B3
:10054000030E0901825D07E280C9F6FF81C9F7FF4A
:1005500082C9F8FF03D04E0EAD6ECBD71200FFFF5D
:10056000FFFFFFFFFFFFFFFFFFFFFFFFFFFFFFFF9B
:10057000FFFFFFFFFFFFFFFFFFFFFFFFFFFFFFFF8B
:10058000FFFFFFFFFFFFFFFFFFFFFFFFFFFFFFFF7B
:10059000FFFFFFFFFFFFFFFFFFFFFFFFFFFFFFFF6B
:1008000000001200280EE66E09ECFEF0E552A7EF9C
:10081000FDF01200FFFFFFFFFFFFFFFFFFFFFFFFE5
:1008200009EF24F01200FFFFFFFFFFFFFFFFFFFFB4
:1008300000005FECC3F0B90E496EDF0E4A6E010E88
:1008400039EFCEF05FECC3F0200E496EE00E4A6E39
:10085000010E39EFCEF05FECC3F0050E4B6EE10EEA
:100860004C6E010E4D6EFE0EDBCF4EF032ECC5F03D
:1008700009ECD2F05BEFC3F05FECC3F08E0E496E73
:10088000DE0E4A6E010E39EFCEF05FECC3F0790E4A
:10089000496EDE0E4A6E010E39EFCEF05FECC3F00A
:1008A0001B0E496ED20E4A6E010E39EFCEF035ECBA
:1008B000CEF0050DAAECCEF00A0E49260A0E4A2209
:1008C000FD0EDB504924E96E000E4A20EA6EEF501F
:1008D0005BEFC3F02EC1E6FFBEDFE5521200350E1E
:1008E0000124CFEFCCF05FECC3F0440E496ED30E81
:1008F0004A6E010E39EFCEF0A3EFC8F0FBECCAF060
:1009000079EFD3F0ADECCDF079EFD3F0E80E496E8E
:10091000030E4A6E79EFD3F0010155513C0DF3CF30
:1009200016F2F4CF17F21200ADECCDF037C23DF065
:1009300038C23EF0F7EFD2F0E66ABBEC26F0E552A3
:100940001200010E0DEFC4F0020E0DEFC4F087C2CD
:10095000E6FF60EFD1F0E66A60EFD1F001018AB7FF
:100960003B0C300CADECCAF019E37FECCFF002E6A3
:10097000D4ECCCF013E2ADECCAF010E37FECCFF096
:1009800002E6D4ECCCF00AE2ADECCAF007E37FEC6F
:10099000CFF002E6D4ECCCF001E2010C000C020E28
:1009A0000101805D0BE2805102E0010E01D0000EDA
:1009B000E8B08A88E8B003D08A9801D08A98070EF8
:1009C000936EF18E8051010803E2F19E170E936E33
:1009D00012002150100B08E06E0E02010B5D04E3C3
:1009E000EDECC4F001E021981200B1ECCDF0010172
:1009F000A86BB19F1200020E0101805D03E18150DE
:100A0000100B06E0030E805D04E18150100B01E045
:100A1000000C010CF0DF000901E1000C010156A1FE
:100A2000010CD70E83ECD2F01E0803E2F00E005C3E
:100A300001E3000C010C480EE66EC10EE66E010EDD
:100A40008FECC3F09CECCBF006E18FECC9F003E037
:100A500001011E0EA86F66C100F064ECC8F00A0E1A
:100A6000665D02E2200E1A6F1200410EE66EC10EA4
:100A7000E66E010E8FECC3F09CECCBF006E18FEC40
:100A8000C9F003E001011E0EA86F67C100F000501D
:100A90000FE00101030E016FD7ECD9F001012D0E1B
:100AA000196F0A0E675D04E2200E196F2D0E1A6F82
:100AB00012003A0EE66EC10EE66E010E8FECC3F028
:100AC00068C100F000500AE00101030E016F64EC00
:100AD000C8F00A0E685D02E2200E1A6F12000101D2
:100AE00048511200800E071406E02050010B03E16C
:100AF0000201215101E0000C010C0201010E3A6FCC
:100B00007E0E7CECC4F001011E0EA86F1200EBEF0C
:100B1000CBF035ECCEF004080FE08AECC4F00EE028
:100B2000FE0EDB500A0808E0FE0EDB500D0804E064
:100B3000FE0EDB50090802E1010E01D0000E5BEF52
:100B4000C3F007019551D880945502E294C795F7F8
:100B500094079251922BEA6A000FE96E0C0EEA227A
:100B6000EF5012000101E251100B03E00401FA51B1
:100B70000AE1420EE66E460EE66E21ECA1F0E55269
:100B8000E5520101E2891200D9CFE6FFE1CFD9FF9A
:100B9000FE0EDB50D80805E1300EF36EFE0EF3CFEB
:100BA000DBFF060EAB1406E0AB980000000000006F
:100BB000AB8840D1FE0EDB50100805E0FE0EDB5086
:100BC000110801E037D10201050E146FFE0EDB5053
:100BD000110837E1020124510DE12050800B0AE198
:100BE000050105014751010B0AE1050105014751C6
:100BF000400B05E1100EE66E8FD9E55222D00501BB
:100C000005014751400B02E00F0E01D0060EE66EC3
:100C100083D9E552C0C1E6FF7FD9E552C1C1E6FFE5
:100C20007BD9E552C2C1E6FF77D9E5520A0E010130
:100C3000C303F3500101C425E66E6ED9E5520501E8
:100C400047910401F051496E4A6A4A3404E249501E
:100C5000D208000E4A5405E20701042B07010407DD
:100C6000E9D00501475104E10501485101E1E2D015
:100C70000201245101E0DED02050800B01E0DAD0E7
:100C80000490050148A10BD04E0EE66E420EE66EB2
:100C900021ECA1F0E552E5520501486BCBD00501EE
:100CA00047A11AD001010101E251080B03E0040140
:100CB000FA510DE1410EE66E460EE66E21ECA1F012
:100CC000E552E5520101E287050147B34BDF05011B
:100CD000479305014791AED0050147A304D042DFF9
:100CE00005014793A7D0050147A726D0440EE66E1D
:100CF0004D0EE66E21ECA1F0E552E5520480440E63
:100D0000E66E4D0EE66E21ECA1F0E552E552030EC3
:100D10000101D05D04E0030E0101D15D08E1540E34
:100D2000E66E440EE66E21ECA1F0E552E5520501B7
:100D30004797050147857ED0050147A524D0570E6A
:100D4000E66E420EE66E21ECA1F0E552E55204801B
:100D5000570EE66E420EE66E21ECA1F0E552E5522A
:100D6000530EE66E490EE66E21ECA1F0E552E55217
:100D70004A0EE66E460EE66E21ECA1F0E552E55213
:100D80000501479557D0050147A90BD0410EE66EE6
:100D9000500EE66E21ECA1F0E552E55205014799AF
:100DA00049D0050147AB0BD0410EE66E520EE66E00
:100DB00021ECA1F0E552E5520501479B3BD005012E
:100DC00047AD13D04F0EE66E520EE66E21ECA1F049
:100DD000E552E552540EE66E520EE66E21ECA1F09D
:100DE000E552E5520501479D25D0050147AF22D0C8
:100DF0004E0EE66E4C0EE66E21ECA1F0E552E55289
:100E0000560EE66E440EE66E21ECA1F0E552E55278
:100E1000420EE66E530EE66E21ECA1F0E552E5526D
:100E2000570EE66E430EE66E21ECA1F0E552E55258
:100E30000501479F200EF36EFE0EDBCFF4FFF3504B
:100E4000F45C04E3FE0EDB507E0807E2FE0EDBCF0F
:100E5000E6FF5FDEE552000944E00401F051496E0F
:100E60004A6AD8904A5004E6FF0E495C000E4A5880
:100E700038E2FE0EDB503B0804E0FE0EDB507C083F
:100E800002E10401F92BFE0EDB50210804E0FE0E06
:100E9000DB5040080AE13B0E0401FE5D04E07C0EDD
:100EA0000401FE5D02E10401F92BFE0EDBCFFEF42E
:100EB0000401F151EA6A000FE96E0B0EEA22FE0E00
:100EC000DBCFEFFF0401F12B0401F02B0401F05103
:100ED00008E10401FE6BFEC4F9F4FEC4F1F4FEC4A3
:100EE000F2F4E552E7CFD9FF1200ACA212000401E0
:100EF000F851EDECCEF0006E0050E66E40ECC8F01C
:100F000000C0EFFF3B0E005C03E07C0E005C01E1E3
:100F100029900401F82B12005FECC3F0ACA2FED7BD
:100F200051ECCEF040ECC8F0FE0EDBCFEFFF5BEFF4
:100F3000C3F0C4EC10F0010EE66ED9EC10F0E552EF
:100F400084948C908D9A8D9CF29E0000F66A080E17
:100F5000F76EF86A940E7F6E550E7E6EAA0E7E6E48
:100F60007F82000000EC00F012000401F007F25153
:100F7000EA6A000FE96E0B0EEA22EF50006EF22BC8
:100F800012002EECC4F00AE11F50020B07E102012F
:100F90008951020B04E18951010B01E1000C010CA4
:100FA000D9CFE6FFE1CFD9FFE6522050200B01E177
:100FB00076D08250010B03E18250020B03E02F50E8
:100FC000400B6DE00101E3890601880EFD6F130EF1
:100FD000FE6F33AC45D0C4EC10F00601880EFD6FF7
:100FE000130EFE6F010EE66ED9EC10F0E55252ECD6
:100FF00096F033AC2DD00601880EFD6F130EFE6FF8
:101000000101016B320EE66EC10EE66E010EE66E58
:101010007EECDAF0E552E552E552CAECD7F0010E6B
:10102000E66E0CECDDF0E552000901E0FF00500E29
:10103000E66E62ECFDF0E5528250010B08E1825051
:10104000020B05E10101E39952EC96F0FF00D1D7C4
:101050000601880EFD6F130EFE6F09EC11F01FD014
:101060002F9CC4EC10F0010EE66ED9EC10F0E552A6
:10107000C8ECD3F0D8ECD3F02A0EE66EC10EE66EC3
:10108000010EE66E7EECDAF0E552E552E552CAEC6E
:10109000D7F00101E39952EC96F009EC11F0E5521A
:1010A000E552E7CFD9FF120014ECCEF0DF6AD00E84
:1010B0004C6ED40E4D6E010E4E6EFD0EDBCF4FF01A
:1010C000506A516A090E416E426A436A4FC03CF051
:1010D00050C03DF051C03EF091ECF9F039C04FF0F6
:1010E0003AC050F03BC051F09EECC9F0DFCF52F057
:1010F000536A546A9BECC7F00800F5CF00F0F55036
:101100000DE0090EDF5C0AE2FE0EDB5003E145EC68
:10111000DAF002D068ECDAF0DF2AC9D7E5525BEFEB
:10112000C3F02750200B06E00501105102011911F0
:101130002D1101E1000C010C0101E251400B0CE00A
:101140000201685109E1080E155C07E0290E155CE3
:1011500004E00A0E155C01E0000C010CBEEC21F06D
:10116000D9ECCCF02D6B3751381102E020944BDADA
:1011700015EF65F00701BE51010B07E07DECC5F0EE
:1011800004E0050ED05D01E0000C010C0101269D7C
:10119000010E0D6E26BF0D681200030E0DECC4F09B
:1011A000258E12006A0ECEEFC3F06B0ECEEFC3F0A9
:1011B00001018E51010B08E06BEC0FF0000904E017
:1011C00001013B51800B01E0000C010C040E0DEC01
:1011D000C4F001013C0EA86F12000101A8510DE1FD
:1011E0002DAC08D0570EE66ED80EE66E010E5AEC06
:1011F000C6F001D0EBDF258E2D8C1200258E050E5A
:101200000DEFC4F0F0ECC5F000010E6EE66A82EC62
:10121000CFF00F6E120087C1E6FFA80EBEECC3F040
:1012200093C100F0B4ECCDF007E10A0E0101950383
:10123000F350FE0BE842006E0050E66EA90EBEEFC2
:10124000C3F05FECC3F0FE0EDB505DECC4F0EF507A
:101250000AE122ECCBF007E340ECCAF05DECC4F00D
:10126000100EEF6EF0D75BEFC3F05FECC3F0FE0E35
:10127000DB50D5ECC4F0EF5030080AE122ECCBF0A3
:1012800007E340ECCAF0D5ECC4F0200EEF6EEFD7C8
:101290005BEFC3F0830E096EFA0E2FECC5F0005021
:1012A0000E6E0EC00FF00E6AFB0EA2ECD3F00050D3
:1012B0009AEFC5F03AC18BF2120001013A511308BE
:1012C00004E2010E3A6F2BA63A6BDAEFBBF035EC75
:1012D000CEF0020802E1BAC7B9F7FE0EDB0402E164
:1012E000B9C7BAF75BEFC3F082ECD0F025EFCBF0D3
:1012F00042C1ABF242C1AAF282ECD0F0EF50400BF7
:1013000003E00201020EAA6F0101D1519BECC4F06F
:10131000EF50400B03E00201020EAB6F120014EC21
:10132000CEF02850010B17E146ECCAF016E14A5006
:1013300014E11750010B03E01C0E155C0CE0175074
:10134000100B03E0150E155C06E01F50100B05E0B6
:101350000C0E155C02E1000E01D0010EDF6E2C5068
:10136000800B03E12C50400B02E0010EDF6E289051
:10137000DF50E5525BEFC3F01A9C238A1200010193
:10138000DF8B11C512F50501106B279A1200CEEC08
:10139000C9F01EE00901E6511BE0CCECCFF0E6C934
:1013A000E6FFAEEC10F0E5520901E75105E0E7C9B0
:1013B000E6FFAEEC10F0E5520901E76BE7C9E6F98C
:1013C000010136990450010B01E03689D2EF08F093
:1013D000010136AF05D004A002D01A8812001A8A83
:1013E00012005FECC3F0CEECC9F00CE0FE0EDB5057
:1013F00009E0C5DF49ECD0F00901E6AF02D00101F8
:101400003689D0DE5BEFC3F05FECC3F0CEECC9F001
:1014100011E0FE0EDB500EE0FD0EDB500BE0AFDF07
:1014200049ECD0F0F1ECCBF0FE0EDBAE02D00101C6
:101430003689B8DE5BEFC3F05FECC3F0010136AD77
:1014400012D0CCECCFF049ECD0F0FD0EDB5002E036
:10145000F1ECCBF001013699FE0EDBBE3689DB5094
:1014600008E0A0DE06D0FE0EDBAE02D01A8801D066
:101470001A8A5BEFC3F026ECD3F0DBCFFBF6020158
:10148000D25101E105D80201190ED26F5BEFC3F012
:1014900018ECCEF0010EFBC6DBFFCEECC9F062E02B
:1014A0002050200B5FE00601FB51FC5D5BE067DF35
:1014B00079DE01013689890E47ECC4F00101DFA510
:1014C0000BD0530E47ECC4F0570E47ECC4F0520E4D
:1014D00047ECC4F00101DF95640EAFECCEF065EC93
:1014E000D1F0DF50300805E2DFCFE6FFAEEC10F0C0
:1014F000E552640EA8ECC9F03AC0DBFFFAECC3F089
:1015000065ECD1F00101E3A503D0520E47ECC4F025
:10151000DF50300808E30601FB51630804E30101D2
:10152000E351040B08E0300EDF5C02E1540E01D001
:10153000DF5047ECC4F00101E3A303D0520E47ECA7
:10154000C4F0FAECC3F0010EDBCF3EF0A0ECCBF020
:10155000300FDF6E300EDF5C02E1540E01D0DF5041
:1015600047ECC4F0FBC6FCF6020EE15C02E2E16A65
:10157000E552E16E5BEFC3F0690ECEEFC3F0060EED
:10158000C7ECC6F0280E9EECC3F0BCEF0AF00101D8
:1015900036BFF5DF12000601980ED880B0553A0E1E
:1015A000B15509E20E50B05D0101D46F0F50060134
:1015B000B159010108D0B0510E240101D46F0601C8
:1015C000B1510F200101D56F1200190E3D6E3E6A18
:1015D0000EC042F00FC043F073ECF9F03BC037F29D
:1015E0003CC038F2180E426E436A37C23DF038C232
:1015F0003EF0BDECFDF03DC037F23EC038F21200C7
:10160000EB0ECEEFC3F00101E293199A139229EC8D
:1016100019F0F6DF0201376B386B199409EF0DF002
:101620009DECA7F00A0E9EECC3F0E30EE3ECC4F0D1
:10163000006E0050F5E112005FECC3F0F1DFEC0E3C
:1016400086ECD0F028EC74F000C709F0FC0E016EB7
:101650000FC000F0B1EC3AF0012A0EC000F0B1EC7E
:101660003AF0096A5BEFC3F0660ECEECC3F0198066
:101670001200670ECEECC3F01990120014ECCEF0FD
:1016800038EC20F0DF6EA4ECCBF007E019A00ED010
:10169000F0DFDF500BE1006A07D019B007D0E4DFBC
:1016A000DF5004E1010E006E63EC75F0E5525BEF74
:1016B000C3F00EEFD2F012ECC4F003E03450400B54
:1016C00004E001015751040B01E1000C010C14EC82
:1016D000CEF001018AA10AD038EC20F0DF6EDF04E1
:1016E00003E0020EDF5C02E1010E01D0000EE552C4
:1016F0005BEFC3F0ECDF000905E138EC20F00408F3
:1017000001E0000C010CF6DF000904E1A8ECCBF0CD
:1017100001E0000C010C14ECCEF01E50010B0EE0A9
:101720009CECC6F00BE012ECC4F003E0D2ECC9F084
:1017300005E11950020B02E1000E01D0010EDF6E2F
:10174000DF5002E08CEC04F0DF50E5525BEFC3F0B9
:1017500014ECCEF01D50040B1AE01D50080B17E0DE
:101760001E50010B14E09CECC6F011E00501105175
:101770000EE12050040B0BE12050010B08E112ECAC
:10178000C4F003E0D2ECC9F002E1000E01D0010E7A
:10179000DF6EDF5002E08CEC04F0DF50E5525BEFCF
:1017A000C3F08A0ED2ECC7F0010136AD05D0410E70
:1017B000E66E4E0EE6EFC3F036BF258E120018EC33
:1017C000CEF0C20EDE6E010EDD6E38EC20F00108A8
:1017D00004E038EC20F002080BE1F40EDE6E010E9E
:1017E000DD6E0101345104E0260EDE6E020EDD6E68
:1017F000B3ECCEF00CE08AECD0F002010051495C71
:1018000001514A5804E2DECF00F2DDCF01F201C2FD
:10181000E6FF00C2E6FF740E85ECC3F0020EE15C49
:1018200002E2E16AE552E16E5BEFC3F01D9CB2ECAF
:10183000CAF0BBDCEC0ED2ECC7F0258E120035EC02
:10184000CEF00A0DF3CF5AF3F4CF5BF3000E030191
:101850005A27030E5B235BEFC3F06B0E005C05E2BF
:101860000201AA510101245F12007FECCFF004E6CF
:10187000990E495C000E4A5804E20201AA51010186
:10188000242712001200280E0101D8806855040D8B
:10189000F328016E0150E66EAA0EBEEFC3F05FECB6
:1018A000C3F02AA40AD052ECC5F0B1EC26F0CBEC80
:1018B000D2F00101500EA86F2A945BEFC3F0149E82
:1018C0000A01DA51800B03E12EECC4F001E1148E21
:1018D00012000101D051080D15ECC6F0010ED89090
:1018E0004B364C36E806FBE10250080D4B50F32412
:1018F000496E4C50F4204950016E12000A01DA8FF3
:10190000DEDF02018051CEECC4F01CE249509608A3
:10191000000E4A5417E202687F0501E1026A030ED5
:101920007F5D02E1010E026EFF0E025C16E0670EA3
:10193000096ECFDF080EE66ED40EE66E0A0E4EEC90
:10194000D0F00BD031EC75F01EAC03D00201098948
:1019500002D00201068B0501478502017F6B010160
:10196000B18F500EA86F2496318C12000201996934
:1019700099C28BF799C28AF799C289F799C288F7F9
:1019800099C287F70701906991698E698F698EC73F
:101990008CF78FC78DF71200040E0101805D03E103
:1019A0008150100B07E0050E805D03E18150100BA4
:1019B00001E1000C010C120014ECCEF00101A45165
:1019C00003E19A51200821E2DF6A090EDF5C10E290
:1019D000DF505CECC5F0EF50040B08E0100EDF2484
:1019E000E66EF1EC2CF0E552000902E1DF2AEDD7BA
:1019F000090EDF5C0AE2100EDF262986DFCFE6FF44
:101A0000AFEC2CF0E552DF5001D0000EE5525BEF59
:101A1000C3F01F86B2ECCAF0B199B19B2582238A2C
:101A20001200D9CFE6FFE1CFD9FFE6528C96000035
:101A30000000FE0EDBCFE6FF2DEC5CF0E55200006F
:101A4000C950DF6E00008C86030EE66E32ECFEF0AD
:101A5000E552DF5000D0E552E552E7CFD9FF120042
:101A60003AEC5CF0F00EC616C680C68A1200800EF4
:101A7000E66EE66A010EE66EC6ECFCF0CBECD2F048
:101A800030EF0DF0128212800601019102011E0E4C
:101A9000306F120012901FA2128012921FB2128297
:101AA000120026ECCFF09BECC4F0EF50E840E84089
:101AB0003F0BDF6E000EDF94DF96DF98DF9ADF9C2E
:101AC000DF9E0A0E006EFE0EDB5009E1030EDF5CA6
:101AD00002E2050E006EDF5044E1010E41D0FE0E21
:101AE000DB50030804E1DF5002E1010E006EFE0E40
:101AF000DB5004080EE1DF0402E1320E006E020E3C
:101B0000DF5C02E15A0E006E030EDF5C02E1640E40
:101B1000006EFE0EDB50050810E1320E006EDF0491
:101B200002E1640E006E020EDF5C02E17D0E006ECB
:101B3000030EDF5C02E1FA0E006EFE0EDB0404E031
:101B4000FE0EDB5002080DE1DF5002E1010E006ED7
:101B5000DF0402E1050E006E030EDF5C02E1190EE8
:101B6000006EE5525BEFC3F087ECD2F0C0C100F02D
:101B7000000406E10101C151460802E2020E006EB6
:101B8000030E005C06E10101C151280802E2040EC7
:101B9000006ED5CA03F0FFECCAF005E03751080B20
:101BA00002E0040E036EE00E4A6ED00E4B6E010E84
:101BB0004C6E00504CECC4F003506AECC8F0EF508F
:101BC0004924016E170E4A6ED10E4B6E010E4C6EFB
:101BD00000504CECC4F0035070ECC8F0EF504924B6
:101BE000026E025097ECC7F0E66A7D0E8CECC5F0F1
:101BF00087ECD2F0280E026E016EFFECCAF00EE008
:101C00003751080B0BE01CCA01F021CA02F0015049
:101C100002E0025003E1280E026E016E025097ECC2
:101C2000C7F07C0E85ECC3F087EFD2F0129A1FB29A
:101C3000128A30DFDEECCCF0DCEC69F01F50020BD6
:101C400006E00101D151D05D02E01A8C12001AACFD
:101C500002D0BCEC09F01200080E0B5C04E3B3ECFC
:101C6000CEF001E1000C010C095004E00701010E67
:101C7000A7ECCFF0096AB2EC04F0000907E0710E9E
:101C8000E66E280EE66E010E12ECD2F01200B2ECF7
:101C900004F0000909E07E0E096E080EE66EB60E2D
:101CA000E66E020E12ECD2F0096A120026ECD3F0B6
:101CB000DBCF48F116ECD2F0B7ECCAF0D9ECCCF09F
:101CC00013985BEFC3F00101485112E0060EAFEC30
:101CD000CEF048C13EF055ECD1F0006E005001E16D
:101CE000002A00500101485F48C15BF249EFC5F08E
:101CF0006DEFC7F007015A5106E1080EE3ECC4F09E
:101D00000501261501E1000C010C2C9E2C9C64ECB5
:101D10002EF0A6EF96F05FECC3F0E2ECCCF007E11A
:101D20002B50010B04E101018A51200B09E140C253
:101D300043F23FC242F23EC241F2F8ECCBF009D08E
:101D4000FE0EDB5006E043C240F242C23FF241C207
:101D50003EF204802BA002D004902B90BEEC40F009
:101D60000101320EA86F5BEFC3F025B41200189A80
:101D700017B8188A12000301916B926B936B946BE6
:101D800091C38DF392C38EF393C38FF394C390F3F7
:101D9000030E016EFF0E015C32E0056A030E026E57
:101DA000FF0E025C22E00250EA6A890FE96E030E20
:101DB000EA22EF504B6E4C6A0150EA6A850FE96ED9
:101DC000030EEA22EF50D1ECC6F0EAECC9F0EF5076
:101DD0009AECC5F005509AECC5F0EAECC9F00EC0DB
:101DE000EFFF0FC005F00206DBD70150EA6A8D0F46
:101DF000E96E030EEA2205C0EFFF0106CBD7120001
:101E000035ECCEF0006E00AE04D0006C01010E0E79
:101E1000116F0101040EE7ECCCF012510AE111C17F
:101E200012F1100E116F135104E112C113F1100ED3
:101E3000126F130E156F5BEFC3F07DECC5F003E17D
:101E4000030E0A5C01E0000C010C7DECC5F005E11D
:101E5000020E0A5C03E00A0401E0000C010C7DECB8
:101E6000C5F003E1020E0A5C01E0000C010C7DEC00
:101E7000C5F007E10A5005E1CB51040B01E0020C6B
:101E8000010C000C7DECC5F005E1020E0A5C03E0DC
:101E90000A0401E0000C010C0601EC5106E07DECA7
:101EA000C5F003E10A50000801E3000C010C7DECD1
:101EB000C5F004E10A0403E00A5001E0000C010C43
:101EC0007DECC5F006E1020E0A5C04E0030E0A5C3C
:101ED00001E0000C010C12ECC4F003E0B0ECCBF01C
:101EE00001E1000C010C0101D05104E10A01DA51B9
:101EF000040B01E1000C010C0101D05104E10A01C5
:101F0000DA51080B01E1000C010C03ECCBF009E005
:101F10000301B851A6ECD3F0B0ECC5F0210E85EC6E
:101F2000C3F0120003ECCBF002E085EF0FF0E66A9D
:101F3000E66A210E85EFC3F07DECC5F010E1CC51CF
:101F4000040B05E00A040CE0020E0A5C09E0CB5128
:101F5000040B05E00A5004E0030E0A5C01E0000CEB
:101F6000010C0101D05103E1CC51400B04E1E4DF4D
:101F7000000901E1000C010CD6ECC9F001E0030CF2
:101F8000B8ECCDF001E0080C07ECCBF001E11B0C44
:101F9000D05109E0030ED05D05E10A5004E0030EC4
:101FA0000A5C01E0030C010CD6ECC9F001E00A0C5C
:101FB000B8ECCDF001E0380C07ECCBF001E1640C9B
:101FC000D05101E0500C380CEFDFE66ED5DFE66E45
:101FD000D60EE66E0A0E98EFC3F05AEC41F0190ED9
:101FE00001240A01D880D75503E2190E0124D76FC6
:101FF000B4ECCBF0D75D03E2B4ECCBF0D76FD46B8D
:10200000338876EFC8F0D6ECC9F004E1B8ECCDF037
:1020100001E1000C010CEF0E896E8A6A8B6A9E0E3C
:102020008C6E900E8D6E8E6A8F6A010E906E916A24
:10203000EF0E926E070E936E930E946E600E956E79
:10204000030E966E7F0E976E060E986EFE0E996EBC
:102050009A6812001F98258A0101B19B02011A514A
:102060001FE0020E685D03E1B8ECCBF019E0070158
:10207000BE9BBE9B32BCBE8B74EC09F00601EA0528
:10208000EB6F020EEA5D01E2EB6BEBC600F00101C3
:10209000D05102E0EDC600F00050E66E17ECCFF034
:1020A00002011A6B25821200C08EA70E99ECC6F0B1
:1020B000ECECCCF0A70E99ECC6F0C3500E26C45041
:1020C0000F220EC04DF00FC04EF0D8904E324D3260
:1020D0000EC04FF00FC050F0D89050324F32D89011
:1020E00050324F324D504F244B6E4E5050204C6E5C
:1020F0000EC051F00FC052F0040ED890523251323F
:10210000E804FBE151504B5C496E52504C584A6E0A
:102110000EC053F00FC054F0060ED8905432533214
:10212000E804FBE1495053240E6E4A5054200F6ED0
:102130000EC0CDF20FC0CEF2C09E1200CDC20EF086
:10214000CEC20FF0E66A6EEC26F0E5520101200ED9
:10215000166F1C6F188F410E1B6F12005FECC3F0DF
:1021600005011151EA6A000FE96E080E8FECD0F0FC
:10217000112B1151F0ECC3F002E6F1ECCCF001E3CD
:10218000116B102B5BEFC3F0B2EC04F0000910E010
:102190008AECC6F0020E0101395D02E1010E396FD1
:1021A00063DD5AEC48F073DD65EC48F041EC79F002
:1021B00012005FECC3F00101E3890601880EFD6F98
:1021C000130EFE6F9EEC16F08A988A8624EC25F09A
:1021D0000101766B140EE66E76ECC2F0E552FE0E4F
:1021E000DB500CE039EC0BF0BCEC0AF0A3ECF6F0A1
:1021F00037ECF7F0DFECDAF029ECD9F00601506BA0
:102200002AEC3DF00601516B0101B56B89985BEF3B
:10221000C3F0F29E3DECFEF0F26AF06AB96A9D6A84
:10222000000EA66EA16E9E6E8D8C8D8A8C9084841D
:10223000070E936E0000000000008A9A0000000064
:1022400000000000270E936E4E0E996E00000000F5
:10225000000003000000000000000000FF0012006A
:1022600014ECCEF020AA3BD0F6ECCCF006E359EC0F
:10227000D1F035E2BCECCAF032E21B50080B2FE182
:10228000F6ECCCF006E359ECD1F029E2BCECCAF054
:1022900026E2F6ECCCF006E359ECD1F020E2BCECFF
:1022A000CAF01DE20050DF6EDF50CEECC4F013E246
:1022B000BCECCAF010E2DF50FBECCCF004E6B40E4C
:1022C0004B5C000E4C5807E2220EE66EC10EE66E25
:1022D000010EFFECCBF0E66A6CDFE5529ADFE552C7
:1022E0005BEFC3F05FECC3F0D8ECD3F052ECC5F079
:1022F000ECECC3F0CAECD7F054ECD0F054ECD0F0D6
:1023000054ECD0F070ECC7F070ECC7F05BEFC3F0AA
:10231000ECECCCF00BECCBF00BECCBF0460EF3EC92
:10232000C9F00F50496E4A6A9F0E00ECCDF049503B
:10233000006E0050800801E2006A0201FC0ED880A5
:10234000CD55080ECE5502E2040E0FD0080ED880EF
:10235000CD55070ECE5502E2030E07D0140ED880DD
:10236000CD55050ECE5503E2020E002607D0200EF5
:10237000D880CD55030ECE5501E2002A00508008CA
:1023800001E2006A080ED880CD55070ECE5502E254
:10239000030E07D0140ED880CD55050ECE5503E29E
:1023A000020E00261200200ED880CD55030ECE5509
:1023B00001E2002A120018ECCEF0C08EAF0E99ECAC
:1023C000C6F0010157A9C5D0500ED880C354050EE0
:1023D000C45401E3BAD0D00EC35C0A0EC45801E362
:1023E000B4D03C0E496E4A6ACDC23DF0CEC23EF03A
:1023F000F7ECD2F000503C0802E23C0E006E0EEC0E
:10240000D3F007014950C35CD06F4A50C458D16F14
:10241000140ED05F050ED15B010157AB9AD0D0C727
:10242000D4F1D1C7D5F105ECCDF0070E53ECC9F0CE
:10243000FDE16A0E4924096E05ECCDF0E2ECD0F026
:1024400009ECC7F00101E3AF10D0E39FC80E93EC95
:10245000C9F004E3840E57ECC9F002E2070119D079
:102460000EC0D2F70FC0D3F76DD0C80E93ECC9F0F1
:1024700004E3840E57ECC9F011E20701C80ED25DE7
:10248000000ED35906E3840ED880D255030ED355DF
:1024900060E2260ED26F020ED36F54D0010E0701F8
:1024A0004A6AD225496ED3514A2294ECD0F00CE30B
:1024B000D2C74BF0D3C74CF04B06000E4C5A4B50D2
:1024C0000E5C4C500F5845E20101D0510CE1070160
:1024D0000E50D25D0F50D35903E2D22B000E1CD008
:1024E000D207000E2ED007010E50D25D0F50D359E7
:1024F00015E2D2510E5C0101D46F0701D3510F5880
:102500002DECCBF003E2050ED46FD56BD45107014F
:10251000D2270101D5510701D32314D00E50D25D2B
:102520000101D46F0F500701D3592DECCBF003E21A
:10253000050ED46FD56BD4510701D25F0101D5517F
:102540000701D35B02EC32F004D00701060EA7ECC2
:10255000CFF032ECC4F00701A7274A50A823A7C741
:1025600049F0A8C74AF0ABECCFF00701A75F4A508B
:10257000A85B080ED880C354090EC45462E3ECEC87
:10258000CCF00B0EF3ECC9F0040E0BECCBF0E8042E
:10259000FCE1360ED8800E56060E0F56CDC249F01D
:1025A000CEC24AF053ECC9F0FDE149500E264A5024
:1025B0000F2220BA0ED0B2C249F0B3C24AF0ABEC3F
:1025C000CFF00201B25F4A50B35B0E50B2270F50FA
:1025D00013D0B2C249F0B3C24AF0640E79ECC3F032
:1025E00049500201B25F4A50B35B2AECCFF0ABEC2A
:1025F000CFF00201B2274A50B323020E4A6AB42533
:10260000496EB5514A22B251495CB3514A5813E35D
:10261000020ED880B455000EB55513E2B4C24BF08B
:10262000B5C24CF0020E4B5E000E4C5A4B50B25DE0
:102630004C50B35906E202EC32F0B2C2B4F2B3C26B
:10264000B5F2C09E63ECC4F002E2E16AE552E16ECD
:102650005BEFC3F018ECCEF0C08EAB0E99ECC6F079
:1026600032ECC4F00701A9274A50AA23A9C749F0B0
:10267000AAC74AF0ABECCFF00701A95F4A50AA5BAA
:10268000C09E63ECC4F002E2E16AE552E16E5BEFEA
:10269000C3F018ECCEF0070114A108D0149123EC7C
:1026A000CEF07D0E976E060EE9ECD0F0C08E9B0E3C
:1026B00099ECC6F032ECC4F00701AB274A50AC23CA
:1026C000ABC749F0ACC74AF0ABECCFF00701AB5F4A
:1026D0004A50AC5BC09E63ECC4F002E2E16AE55292
:1026E000E16E5BEFC3F035ECCEF007E1C00E016E9A
:1026F00001015FA304D0E00E01D0B00E016E010114
:102700000D510126F4EC3AF0FE0EDB5013E00F0EF3
:10271000005C03E3005030080DE2230E006E090157
:10272000EB5108E0020E0101395D04E00901EB51B3
:1027300059ECCEF000505BEFC3F014ECCEF0B6ECE9
:102740000CF02EECC4F008E10701B16B0A01D56B67
:10275000DA9331EC75F012D02FECC7F0EFCFB1F770
:10276000D0C1DFFFD5CA00F0080EE66EE66ADF5082
:1027700006ECCFF01AECD2F05FECC6F0149C01012D
:10278000D05103E0030ED05D06E1030E0A01D45DD3
:1027900007E1148C05D0020E0A01D45D01E1148C0E
:1027A000DAA304D0D8CAB6F7D9CAB7F73CEC19F007
:1027B00082ECD0F0EFCFBEF70701BE9F0101D051F0
:1027C00003E0030ED05D02E10701BE8F2FEC1FF086
:1027D000B5ECC5F0DFECD7F02FEC25F078EC09F084
:1027E000E5525BEFC3F012ECD3F006ECCFF05FEFF5
:1027F000C6F082ECD0F025ECCBF02EECC4F00FE06C
:102800000A01DAA306D0B6C7D8FAB7C7D9FA3CECA2
:1028100019F0E9DF01012FECC7F0B1C7EFFF12009B
:1028200014ECCEF0DF6A080EDF5C04E26CECD1F051
:10283000DF2AF9D7E5525BEFC3F014ECCEF0DF6A84
:10284000080EDF5C0CE2B6ECC4F0EFCF49F0FE0EF0
:10285000DB50495C02E1010E03D0DF2AF1D7000E04
:10286000E5525BEFC3F05FECC3F018BE08D051EC4B
:10287000CEF073EC04F0E5527F0B01ECC4F05BEF9B
:10288000C3F05FECC3F018BE13D029A003D075ECE1
:1028900007F0FBD74CECC8F00BE04CECC8F001ECB7
:1028A000C4F073ECD1F0EE2A000EEE22EE22F2D745
:1028B0005BEFC3F05FECC3F018BE25D029A003D0B6
:1028C00075EC07F0FBD7A0ECC5F0E80E426E030EE6
:1028D00081ECC5F0492401ECC4F075ECC4F080EC47
:1028E000D1F0A0ECC5F0640E10ECD0F0640E7AECE0
:1028F000D1F00A0E10ECD0F00A0E7AECD1F0300EC6
:10290000492401ECC4F05BEFC3F05FECC3F018BEE8
:102910000FD01EAE0DD01D0EE66EC10EE66E010E7E
:10292000C4ECC3F052ECC5F0ACDFE552E552E55221
:102930005BEFC3F014ECCEF00201CF2B1EAE19D02A
:10294000060EE66ED00EE66E010EBDECC4F051EC44
:10295000CEF089DFE552FE0EDB28E66E84DFE5521D
:10296000FE0EDB50020FE66E7EDFE5523B0E01EC01
:10297000C4F051ECCEF061DFE552000915E1DF6AE9
:10298000080EDF5C11E2B6ECC4F0EF50FF080AE17C
:10299000B6ECC4F0FE0EDBCFEFFF36ECC7F026C777
:1029A000EFFF02D0DF2AECD707012669E5525BEF83
:1029B000C3F014ECCEF0DF6A080EDF5C0FE2B6EC79
:1029C000C4F0EF50FF0808E036ECC7F0EF50016E9E
:1029D000B6ECC4F0EF5005D0DF2AEED70201CF6B82
:1029E000FF0EE5525BEFC3F018ECCEF0DF6A080E85
:1029F000DF5C0FE2B6ECC4F0010EEFCFDBFFDB5083
:102A0000FF0805E06CECD1F0010EDB5005D0DF2AA9
:102A1000EED70201CF6B000EBCECCBF002E2E16A14
:102A2000E552E16E49505BEFC3F014ECCEF032504A
:102A3000100B04E1020E07015A5D02E1DF6A03D0C8
:102A4000F0ECD0F0309ADF50E5525BEFC3F018ECB9
:102A5000CEF03250100B04E1020E07015A5D03E183
:102A6000DE6ADD6A08D0F0ECD0F0E66A82ECCFF0E6
:102A70005CECC9F0309A63ECC4F002E2E16AE55222
:102A8000E16E5BEFC3F014ECCEF007015E6B5F6BA1
:102A90002DA802D0010E2AD0080EE3ECC4F0DF6EA0
:102AA00007015E2B000E5F23200EDF1405E0580E99
:102AB0005E5D020E5F59F0E35E51605D5F516159EA
:102AC00004E25EC760F75FC761F7580E5E5D020EF5
:102AD0005F590BE301018B5105E15CC726F7360E08
:102AE00080ECC4F02D88000E01D0010EE5525BEFA2
:102AF000C3F05FECC3F003ECCCF05BEFC3F05CEC35
:102B0000CFF003E2C0ECCBF004D0FE0EDB50F60FAA
:102B1000410F5BEFC3F0020E006E020178B9008E28
:102B200035C101F00150280802E2280E016E005064
:102B3000E66E060E0102F350E66E780E85ECC3F0E9
:102B400040EC20F0016A01013551280807E27C0EB3
:102B50000FECCDF003E2280E355D016E0150E66EFC
:102B60003A0EBEEFC3F014ECCEF038EC20F0DF6E7E
:102B70000F0EE66EDF5007E0030EDF5C04E001019C
:102B80008A51020B02E1000E01D0010E000905E09E
:102B90000A0E01017A03F35001D0000EE66E7E0E9C
:102BA00085ECC3F0E5525BEFC3F064C178F2B0ECA2
:102BB000CBF002E165C178F21200B0ECCBF003E19A
:102BC00078C265F102D078C264F1EFDF8BEF15F0C7
:102BD0008DC20EF08EC20FF086ECD1F05E0E85EC49
:102BE000C3F08FC20EF090C20FF086ECD1F05F0EF2
:102BF00085ECC3F092C2E6FF91C2E6FFE66A7B0E67
:102C00008CEFC5F00601B46BB56B020EEDECC6F0AF
:102C10000601B42B000EB523B451B65DB551B759BA
:102C200004E2B4C6B6F6B5C6B7F6E80ED880B45519
:102C3000030EB5550BE201018B5105E15CC726F788
:102C4000390E80ECC4F02D883186010C84B0DDD7BC
:102C5000000C14ECCEF0FE0EDBCF5CF72D50100B09
:102C600003E13150100B02E1000E20D031A604D058
:102C70000A0EEDECC6F001D0C5DF51ECCEF011EC40
:102C80000DF0E552DF6EE66A11EC0DF0E552010140
:102C90003851100B0AE03050200B07E1E3A102D0BD
:102CA0002E0E01D0210E8BECCEF0DF50E5525BEF03
:102CB000C3F04CECCEF00101E3915BEFC3F04CECC0
:102CC000CEF0FC0EFDECC3F00101E3915BEFC3F02D
:102CD0004CECCEF08CECD1F00101E3915BEFC3F052
:102CE0004CECCEF08CECD1F0FA0EFDECC3F0F90E0A
:102CF000FDECC3F00101E3915BEFC3F019ECD3F0FD
:102D0000D4C1E6FF82ECCFF0D5C1E6FF82ECCFF074
:102D10000EC0E6FF82ECCFF00FC0E6FF82ECCFF0F2
:102D20000101E3915BEFC3F01D0E86EFD0F01E0EA4
:102D300086EFD0F0D9CFE6FF5BEFC3F02AB203D025
:102D4000600ECEECC3F02A8212002AA203D0610EDC
:102D5000CEECC3F02A9212002AB203D0600ECEEC61
:102D6000C3F02A8212002AA203D0610ECEECC3F077
:102D70002A9212005FECC3F031B206D0620ECEECA4
:102D8000C3F0FE0EDBCF1BF25BEFC3F05FECC3F0D2
:102D9000B00ECEECC3F0FE0EDBCF1CF25BEFC3F047
:102DA0005FECC3F007018651320D14ECCDF0BCECA2
:102DB000CDF012E1FE0EDB500FE10101D05104E134
:102DC00029510A0D14ECCDF0DAECC9F005E001014F
:102DD000E80ED46F030ED56F5BEFC3F014ECCEF0AA
:102DE000D6CA85F707011E0E866F0101D05105E195
:102DF00011ECC7F03EC086F710D0030ED05D0DE198
:102E0000030E0A5C03E10701140E06D0F2ECC6F0D3
:102E100004E059ECD0F00701866FD7CA00F0070133
:102E2000BEAF10D0190E006E0A01D75D06E2C4ECE9
:102E3000CBF099ECD0F0005E05D0190ED75D99EC7F
:102E4000D0F00026190E005C05E3190E005C0701A6
:102E5000862705D0190ED88000540701865F080E1A
:102E6000006E21A20FD00101D05102E1020E18D054
:102E7000D00506E0020ED05D03E0040ED05D11E146
:102E8000010E0ED00101D05102E1080E09D0D0058B
:102E900006E0020ED05D03E0040ED05D02E1070EF5
:102EA000006E07018551FE0BE8420024056EDF6AC3
:102EB0000550865D13E2DF2A8551FE0BE842862528
:102EC000016E01500024FE0BE842866F0050015C49
:102ED00002E20050016E0050015C856F2EECC4F0E0
:102EE00005E10701320E856F1F0E866F07ECCBF0F0
:102EF00004E2DFCFE6FF54DFE552C0ECCDF05EE048
:102F00000701BE51800B27E0DF5025E154DB21ECA7
:102F1000C8F00A01D751190808E2190ED75DFFEC75
:102F2000CEF00101D4274A50D523BCECCDF008E205
:102F3000C4ECCBF0FFECCEF00101D45F4A50D55B7E
:102F400001010A0ED503F3CFD5F1D403F3CFD4F1A9
:102F5000F450D52704D0DFCFE6FF22DFE55207018A
:102F60008551320D29ECC4F07DECC5F001E1D58F1F
:102F7000200E006E07018851005C10E18C510101A8
:102F8000D4190CE107018D510101D51907E10701A1
:102F90008E510E1802E18F510F180DE000C088F716
:102FA000D4C18CF7D5C18DF70EC08EF70FC08FF747
:102FB0000050F8ECD0F067DD85EC0FF0B4EC0DF0CC
:102FC00025EC4EF0E5525BEFC3F0F6ECC6F0005096
:102FD00001E11200C0ECCDF065E00101DC0ED46F20
:102FE000050ED56FF00E0E6E0A0E0F6E030E005C0E
:102FF00001E1D58F000403E0020E005C45E167ECBF
:103000000BF0000915E001018951640D29ECC4F0B1
:1030100021ECC8F0010E0F0B05E0D890D533D43366
:10302000E806FBE1640E0101D427000ED5232CD065
:103030000101345129E03451080DF3CFD2F1F4CF1E
:10304000D3F15C0ED227000ED323D2C149F0D3C1F5
:103050004AF0F00ED88049560A0E4A56010E0F0B60
:1030600003E06BECC9F0FDE149500101D225D46FBA
:103070004A50D321D56FD2C10EF0D3C10FF0F00E5C
:10308000D8800E560A0E0F56050ED05D08E10E0EC2
:10309000D46F060ED56FC40E0E6E090E0F6E300E75
:1030A000F8ECD0F043EF15F0320EE66E730EBEEF83
:1030B000C3F0640ECEEFC3F018ECCEF012ECC4F007
:1030C00001E192D08AECC4F001E08ED007015A51A0
:1030D00001E08AD00FECCBF001E086D0195101E07D
:1030E00083D001013B51800B04E1050ED05D01E06E
:1030F0007BD0080EE3ECC4F0DF6E2EECC4F06EE182
:10310000E09FDFB8E08FE251040B68E094510108C2
:1031100065E20201D95162E1D85160E10101E25159
:10312000010B5CE1E051800B54E0EDECC4F051E0A8
:103130001D50400B4EE1020168514BE12050200B25
:1031400048E0195146E1245144E12C50800B41E103
:103150002C50400B3EE12F50200B3BE12350800BC5
:1031600038E13050400B35E12450010B32E1D2EC14
:1031700008F0E4DD0101030E9A6F280E9B6F440EE8
:103180009C6F9E6B9EC19DF130ECF1F00701148F96
:10319000149323ECCEF00701159128ECCEF0070133
:1031A0000B8907ECF7F0E00E07010A150609E66E39
:1031B000120EE66E420E6EECC3F00701099FCEECD4
:1031C000CEF0820ECEECC3F001019405190DF3CFC1
:1031D000D8F20101E0BF02D0D5EC08F001013BAF0D
:1031E00003D0010EDF1401D0000EBCECCBF002E2E4
:1031F000E16AE552E16E49505BEFC3F001013B51DA
:10320000800B06E012ECC4F003E08AECC4F001E0AD
:10321000000C010C53C1E6FFF1DF000903E00101DE
:103220006E5101D0000EE66E340E85ECC3F06FC116
:10323000E6FF350EBEEFC3F0650ECEEFC3F02050B3
:10324000400B06E00101E151040B02E1E18501D8E8
:10325000120014ECCEF054C1DFFFB0ECCBF002E171
:1032600058C1DFFF080EDF02F350E66E750EBEECAC
:10327000C3F0E5525BEFC3F00701B6510C0803E35E
:10328000B7510C0805E2B66B0C0EB76F0A01DA9362
:103290001200016A0D0E015C07E058ECC8F002E074
:1032A00001501200012AF6D7000C0C0E016E0150DD
:1032B00007E058ECC8F002E0015012000106F7D711
:1032C000000C0701B46BB56BD7DFB6C701F007017F
:1032D000B751D880015409E36FEC04F0F3500701B3
:1032E000B413F450B513012AF2D71200016AD6ECD8
:1032F000C9F00BE0EAECCEF006E249500508000EFA
:103300004A5401E2012A420E0DD0B8ECCDF012E091
:10331000EAECCEF006E249501408000E4A5401E2ED
:10332000012A440E0124CFECCCF0F3CFB4F7F4CF54
:10333000B5F71200EAECCEF014E249504608000E50
:103340004A540FE20701F40EB46FB5692EECC4F0D5
:1033500001E1AFD00701B66B0C0EB76F0A01DA833B
:10336000A8D0006AD751CEECC4F006E249500D084F
:10337000000E4A5401E2002AD751CEECC4F006E216
:1033800049501308000E4A5401E2002AD751180888
:1033900001E2002AD751190801E2002AD751CEECE8
:1033A000C4F006E249501F08000E4A5401E2002A08
:1033B000D751CEECC4F006E249502508000E4A541D
:1033C00001E2002A0101D05103E0030ED05D1CE1AF
:1033D000EAECCEF006E249500508000E4A5401E23C
:1033E000012AA9ECD3F006E249500A08000E4A541B
:1033F00001E2012AA9ECD3F022E249501308000EA1
:103400004A541DE2012A1BD0EAECCEF006E24950F4
:103410001E08000E4A5401E2012AA9ECD3F006E28C
:1034200049502808000E4A5401E2012AA9ECD3F0C1
:1034300006E249503208000E4A5401E2012A460EC3
:103440004C6EDF0E4D6E010E4E6E00504F6E506A88
:10345000516A030ED8904F3650365136E806FAE1DD
:103460009EECC9F00150526E536A546AD89052369D
:10347000533654369BECC7F00900F5CFB4F70A0079
:10348000F5CFB5F703ECCBF005E00701B485B589BE
:10349000B49DB59B030E0A01D45D02E0D45109E14D
:1034A000F8DE0701B66F01DF0701B76F0A01DA83A3
:1034B000E3DE0A01D40514E10701B705056E0A0E23
:1034C000B75D01E20506E5DE0701B66F0550D8805D
:1034D000B65502E205C0B6F7F4DE0A01DA8312003F
:1034E000020ED45D12E10701B629056EB65102083D
:1034F00001E2052ADADE0701B76F0550B75D02E287
:1035000005C0B7F7DEDE0A01DA8312001E0E006E78
:103510000101D05104E111ECC7F03E500AD0DAECC1
:10352000C9F002E0140E05D0F2ECC6F003E059EC4D
:10353000D0F0006E0A01D651FE0BE842056E120073
:10354000050E7CECC4F0050E0A01D803F350006EA2
:103550000101012B64ECC8F01B8F1200080E7CECFB
:10356000C4F00A01D951050D9DECD0F00101200EE7
:10357000196F19C118F11B8F12003DECC8F0DEEC79
:10358000C9F03B51200B06E18FECC9F003E00101CB
:103590001E0EA86FC2EC63F0FFECC5F0300E010107
:1035A000195D02E1200E196F1B8F016B2A0E006E50
:1035B0002388E1EF25F00101D05102E129510BD020
:1035C000030ED05D11E1030E0A5C02E1640E03D02C
:1035D0000A5004E1960E0E6E0F6A1200240E2E257C
:1035E000E8ECC4F00E6E0F6A120090DF0701BEAF68
:1035F00015D092ECD1F00A01D751190804E2190E46
:10360000D75D9AECC5F0190ED75D1CE2C4ECCBF087
:10361000FFECCEF00E5E4A500F5A12000A01D7514D
:10362000190803E2190ED75D0026190ED75D03E2D3
:10363000C4ECCBF0005E0050A6ECD3F0190ED75DC1
:1036400001E1B9DF1200570E7CECC4F09CECCBF02A
:1036500006E18FECC9F003E001011E0EA86FC5DF83
:1036600003ECCBF00BE00101410E166F500E176F0B
:103670000301B8510F6AE8307F0B0E6EFFECC5F006
:103680000101200E196F19C118F103ECCBF009E00C
:103690000101460E186F2951E8240301B85D07E1C6
:1036A00003D0BCECCDF003E101012A0E196F01013A
:1036B0001B8F12005FECC3F0070EE126BCEC0FF08D
:1036C0000A01D65D04E2BCEC0FF00A01D66FD4EC1F
:1036D0000FF00A01D880D65504E2D4EC0FF00A01AD
:1036E000D66F03EC10F0000903E00A01190ED76F42
:1036F0000DDFBCECCDF004E3190ED75D002603D03E
:10370000C4ECCBF005260550005C03E30550005ED9
:103710000AD0006AD40507E1DC51D75D04E2DCCAB7
:10372000D7FADDCAD6FA00C0D8FAF0DE0550002676
:10373000BCECCDF004E3190ED75D002609D0C4EC33
:10374000CBF0056E0550D880005402E20550005EB3
:1037500059ECD1F00BE249505408000E4A5406E2ED
:10376000540E006EDCCAD7FADDCAD6FA00C0D9FA08
:1037700000C0C5F7190ED75D03E3190ED75D03D05E
:10378000190ED880D7550701B26FB36BBEAF02D008
:103790000A0E01D0320EB303F3CFB3F7B203F3CF67
:1037A000B2F7F450B327FE0EDB501DE02050800B23
:1037B0001AE10A01D45102E1E0DE0AD0D40502E1A7
:1037C000BFDE06D0020ED45D02E1C8DE01D03BDFD1
:1037D000DEECC9F03B51200B06E18FECC9F003E0B1
:1037E00001011E0EA86F3450040B0DE10A01DA51DD
:1037F000020B09E0D6ECC9F006E1B8ECCDF003E12C
:1038000003ECCBF003E072DD349401D05ADD070104
:10381000010EB06F01012AA303D00701070EB06F9C
:10382000D5CADFFF0A01D56B0701B051010853E289
:10383000C8ECCBF050E1CE51010B4DE1050ED05D4F
:103840004AE0040ED05D47E0D00503E0020ED05DF3
:103850000FE1AEEC04F00A01D95D0AE2D52B8AEC47
:10386000D2F004E61E0E495C000E4A5834E21ED027
:103870000101D0511DE10A018AECD2F004E61F0ECD
:10388000495C000E4A5801E2D52B8AECD2F004E6DE
:103890000F0E495C000E4A5809E3D651FBECCCF000
:1038A00004E60B0E4B5C000E4C5815E2D52B13D0E2
:1038B0000A018AECD2F004E62D0E495C000E4A584B
:1038C00001E2D52B8AECD2F004E60F0E495C000E23
:1038D0004A5801E2D52BDF500A01D55D0AE0D5CA6E
:1038E000DFFFDFECD7F0D5CAE6FFAB0EBEECC3F0CE
:1038F000248A1EAC03D00201098902D00201068B82
:10390000050147858EEC39F0070EE15C02E2E16AC1
:10391000E552E16E5BEFC3F0006A800E066E056E45
:1039200005500502F350015CF4500258D8B008D09D
:1039300000C005F006420650051206BE09D0F0D7B9
:1039400005C000F006420650051206BE01D0E8D7B9
:1039500000D012005FECC3F02A8448C102F0D2EC20
:10396000C4F03FE05A0E025E010EE66E73EC13F0F7
:10397000E552016E02504B0817E24B0E025C036EDB
:10398000060E4A6E4AC043F001C03EF017ECFEF04E
:103990003EC049F049C043F003C03EF017ECFEF0D2
:1039A0003EC003F00350015E0F0E015C02E20F0EF9
:1039B000016E0150300802E2300E016E01C0C1F705
:1039C00002500A0D29ECC4F00150496E4A6AE6EC37
:1039D000CEF03D50026E23B604D00250E82402011E
:1039E000D56F19ECCDF00701C06FFE0EDB50020859
:1039F00001E189D0C0C701F00101E2A502D0040EA7
:103A0000016E01504B6E4C6A0250D1ECC6F0030EB1
:103A1000D8900E360F36E806FBE108ECCCF00A0E23
:103A20004F6E4FC043F00BC23EF055ECD1F04D6EDF
:103A30004E6A00504B6E4C6A800E3D6E3E6AA1ECA1
:103A4000D0F0AEECC8F07DECD3F066ECC6F0036AC3
:103A50000FDB016E1C50040B31E0010403E0020E89
:103A6000015C2CE13450400B29E1FE0EDB5026E0D6
:103A700001C202F0025022E00250F0ECC3F004E672
:103A8000800E495C000E4A5819E20250FE0BE842D3
:103A9000D880005413E20250E824005C0FE2FE0ECE
:103AA000DB0406E10C0E02010027000E012305D005
:103AB0000C0E0201005F000E015B032A03500EE1B1
:103AC000880ED8800E54130E0F5404E2880E0E6E2A
:103AD000130E0F6E0EC000F20FC001F22450020B45
:103AE00006E12250400B03E03150800B0AE0036AEC
:103AF000006A31AE06D0000E0201026F036B006F48
:103B0000016BDFEC0BF05BEFC3F05FECC3F0B0ECEC
:103B1000C5F051ECCEF05FEC16F0CBECD2F05BEFE1
:103B2000C3F05FECC3F05EECD0F0770EC1ECCAF0EE
:103B3000FE0EDB5003E0100EC1ECCAF05BEFC3F0E9
:103B4000F6ECC6F0050E005C09E0CCECCBF006E12B
:103B500067EC0BF0000902E1000E01D0010E000934
:103B600002E0000E03D001013451E824E66E3C0E61
:103B7000BEEFC3F063EC3FF0E3DF0201A85103E0C6
:103B80000101345106E00201A85105E1010134515F
:103B900002E0E5EC17F02A84120026ECCFF003E0F7
:103BA0000101285101D0000EDF6E21B204D0040EB5
:103BB000DF02F3CFDFFFDFCFE6FF760EBEECC3F010
:103BC000DF90DF42DF5005E1FE0EDB5002E0010E28
:103BD000DF6EDFCFE6FF790EBEECC3F0E5525BEFA0
:103BE000C3F05FECC3F0016A080E015C16E2FE0E42
:103BF000DB5001241EECCDF0026E100E025C040DB1
:103C0000F350006E7DECC5F001E1006AACECD3F03E
:103C10000050CEECC3F0012AE7D7140E9EECC3F09F
:103C20005BEFC3F0C0ECCDF00CE0220ECEECC3F0A5
:103C30000101D05102E1180E01D0080EE66ED1DF6D
:103C4000E55243EF15F0C0ECCDF00DE0310ECEECB7
:103C5000C3F083EC0BF0000902E0100E01D0000E5F
:103C6000E66EBFDFE55243EF15F0260E0101B55DAC
:103C700002E112EF1EF023EF1EF002019951010143
:103C8000625D18E062C199F26251020B05E1CC510C
:103C9000200B02E1000E01D0010E000902E0000E2F
:103CA00001D0380EE66E0F0EE66EC80EE66EA10E5F
:103CB0008CECC5F01200120005ECC6F0840ECEECC0
:103CC000C3F02A929EEC16F0E66A720EBEECC3F0C8
:103CD0003C0EE66E710EBEECC3F0EEEC16F01CEC82
:103CE00019F043EC0CF00BEC09F0B9D861ECCFF013
:103CF000E66A130EBEECC3F0010162855C95BDDF80
:103D00006AEC4EF0E668B30EBEECC3F03DD825EC8D
:103D10004EF08EEC4FF0D5EC08F0E8EC15F0D5EC59
:103D200015F08BEC15F029EC19F08DDF49ECC5F09E
:103D300007DFB3EC15F00AEC19F0010EE66EF1DEC8
:103D4000E55205ECC6F00601B26B090EB36F6ADFEF
:103D500001015F51200B02E0640E01D0320EE66ECD
:103D60001F0EBEECC3F0010EE66E0F0EBEEFC3F0E9
:103D70001200046A01015FAF04D011BC048011BEBF
:103D800004823CB904841200010112983B51100BCB
:103D900001E012883B51100B0FE02150020B0CE0A8
:103DA0001E50200B09E0050ED05D06E0040ED05D2C
:103DB00003E0030E006E06D031C100F0CCECCBF076
:103DC00001E0006A0050E66EA60EBEEFC3F0016A85
:103DD0000701BEB302D04BC101F04CC102F0BE518D
:103DE000020B09E00101D05104E10601EA5101088A
:103DF00002E34DC102F00F0E0101D8804155E66E7D
:103E0000025097ECC7F07DC1E6FF47C1E6FFA00E68
:103E1000E66E70EC16F0496E060EE15E495070C118
:103E2000E6FF6E0EBEECC3F00701BEB10FD001017C
:103E3000CEAD03D0CE9D25EC4EF01450100B06E015
:103E40001450200B03E114988EEC4FF00701BE5183
:103E5000010B02E0AE0E01D0AD0ECEEFC3F0E7EFE6
:103E60001EF014ECCEF0F6ECC6F0000403E0020EF7
:103E7000005C08E1E66A3350040B02E0030E20D038
:103E8000000E1ED0005005E1010EE66E4ADEE5523E
:103E900038D0050E005C16E102018951040B08E1DF
:103EA0002050400B03E0330E875D02E0000E01D08E
:103EB000010E000902E0875101D0000EE66E040EEB
:103EC000E66E21D0030E005C1CE18AECC4F019E020
:103ED000020E0A5C03E14BECCAF00CD0E80E0E6E49
:103EE000030E0F6EB0ECC5F03E0E85ECC3F0E66A33
:103EF000020EE66E140E85ECC3F00501040E266F6B
:103F000005D0E66AE66A140E85ECC3F0E5525BEF75
:103F1000C3F014ECCEF002012F6B0601BF6BBFC6DD
:103F2000BEF6329E0101D05124E10601EA5101089A
:103F300003E31350010B17E0016AEA05EB6F020E71
:103F4000EA5D03E302011A5102E00601EB6BEBC6E6
:103F5000E6FF17ECCFF0E66A030EE66E120E85EC74
:103F6000C3F0328E04D061ECCFF00601EB6B77DF4B
:103F700055D0030ED05D50E162991350010B06E15C
:103F8000D6ECC9F003E1C4ECCDF042E0F2ECC6F0AF
:103F90000AE02D0EDF6E010E016E026A13A00ED034
:103FA00002012F6F0BD0DAECC9F006E0020E016EB1
:103FB000026A1F0EDF6E02D0016A026AE66A0150D1
:103FC000E66E120E85ECC3F0EDC6E6FF17ECCFF0FF
:103FD000328ED6ECC9F002E0010162890701200EA1
:103FE000516F3F0EDF5C02E1100E516F640EDF5C1B
:103FF00002E10A0E516F4B0EDF5C02E10D0E516FB4
:104000002D0EDF5C02E1160E516F4E6B526B02D02B
:1040100061ECCFF032DE02D061ECCFF00DEC39F084
:10402000E5525BEFC3F0BF0E83ECD2F0E840E8400E
:104030003F0B005C02010B6F060E00C0E7FF070B91
:1040400004E0E742E79EE806FCE1E75002010B5F6F
:104050000B076E0E0B5D09E22150100B06E101010A
:10406000395103E1218816ECD2F00BC200F01200A6
:104070001FB203D00101D05112000101D151120031
:104080000C0ECEECC3F0F0ECC5F00E6E0F6AFF0E16
:104090000E1804E10F5002E10E680F681200416B28
:1040A000426B436B446B400E456FD8903C373B37B7
:1040B0003A37393738373737363735374437433774
:1040C000423741374051445D3F5143593E51425977
:1040D0003D51415909E34051445F3F51435B3E51DB
:1040E000425B3D51415B3C2B452FE0D71200010163
:1040F000CC9711BECC87CD9911BCCD8912000A0E88
:1041000023ECCDF001010490CC51080B01E00480B8
:104110000492CD51100B01E00482119E04B0118E67
:10412000119C04B2118C07010A970A990A8504A010
:104130000ED00101CC5107010A99010B01E00A8957
:104140000101CC5107010A97020B01E00A870A51CD
:10415000100B06E10101775103E10450020B02E06C
:1041600007010A9507010A9104B20A8108ECF7F0E9
:10417000B9EF1EF014ECCEF096ECD1F0200ED4EC9A
:10418000D0F00050026E0F0ED4ECD0F001012B5194
:10419000005C29E1250E025C26E1050E18ECD0F04A
:1041A0007DECC5F013E2010EE66E0A0EDF246EEC24
:1041B000CEF0D1ECC3F00F0E01010617D051065D11
:1041C00005E0288206C1D0F11FECC6F02EECC4F049
:1041D00007E1030EE66E100EDF24E66EFFECD0F072
:1041E000096A010E02D0096A000EE5525BEFC3F0C6
:1041F0005FECC3F01EAC03D00201098102D00201C2
:1042000006830501478147872B8C2C8A75ECC4F007
:10421000EE50ED1013E00101442B640E445D03E207
:10422000A9DF00091DE101014407FF0E445D03E021
:10423000A1DF0009F8E10101442B12D0010144077C
:10424000FF0E445D03E096DF00090AE10101442B03
:10425000640E445D03E28EDF0009F8E101014407CA
:104260005BEFC3F05FECC3F0140E496EDA0E4A6EDA
:10427000010E06ECC4F0FCECD2F07F0B006EFE0EDB
:10428000DB50040806E1FD0EDB50310802E2020EAD
:10429000006EC8ECCDF006E1FD0EDB50310802E205
:1042A000040E006E5BEFC3F0040E0101435D01E3F9
:1042B000436B395102E0190E04D0160E4325E8EC89
:1042C000C4F0006E0050E66EE66A3C0EE66E9DECB1
:1042D000FBF01DEFCEF021900201320E246F295128
:1042E00002E0140E246FC80E366F1DAC2998D95108
:1042F00002E0D5EC08F01D50400B03E02A50800B83
:1043000002E19EEC16F00201098709850983098103
:104310007A6B0901EB6B12005FECC3F0FE0EDB5011
:104320000EE029A006D0FE0EDB50030B02E175EC77
:1043300007F0280EEDECC6F0FE0EDB06EFD75BEFC4
:10434000C3F011C512F50501106B279C0101E09126
:10435000120027BA09D013C549F114C529F12492D6
:1043600023BC2482B9EC64F0278A01013699D5EC8C
:1043700008F00201216B239A259212001FECD2F063
:10438000E0DF2750200B05E08AECC4F002E0080EC5
:10439000076EDFDF2F98120027AA02D00101E48BFD
:1043A0000750220A01E19ED1030A01E17FD1010AEF
:1043B00001E1EFD03F0A39E0010A01E0ADD1278CDD
:1043C00049C113F529C114F5239C24B2238C27BAC3
:1043D00015D0010136AD11D0E3B706D03651070B29
:1043E000050DF3500A0F496F640E296F36B902D0DC
:1043F000430E296FA3EC64F001D0C0DFC4ECCDF014
:1044000007E0200E06014A5D03E0200E8FECC6F0A7
:104410001D901F0E076E02012D5101E17ED1275024
:10442000200B01E17AD1076A23D10501105101E186
:1044300088D08AECC4F016E02750200B13E0050169
:10444000235107E1020E265D0DE17AEC0EF0000922
:1044500009E102012D5101E12D2B080E076E1F0EFF
:10446000086E1200050110071251EA6A000FE96E8A
:10447000080EEA22EFCF02F7122B1251F0ECC3F034
:1044800002E6F1ECCCF001E3126B8AECC4F00BE035
:104490002750200B08E002C7E6FF0DEC3CF0E55288
:1044A000200E076E12003C0E0701025D04E124821B
:1044B000238C229C32D13E0E025D06E12492239C85
:1044C0001EBC2BD1228C29D1740E025D01E125D1B5
:1044D0000601EA510AE02750200B07E0298A02C7AB
:1044E000E6FFE4EC6FF0E552299A800E0701025DC9
:1044F0000FE2380E496EDE0E4A6E010E4B6E200E34
:10450000025DCAECC6F064ECC3F00800F5CF02F718
:10451000800E025D03E10201040E526F0701025199
:10452000800805E2800E025DFD0F0201526F800ED1
:104530000701025D01E3B4D0025101E1EED0200E8B
:10454000CFD027AAE9D0C6ECCAF007E00701025194
:10455000800803E3200E8FECC6F010DF8AECC4F075
:1045600005E0279C080E076E100E086E2750200BE2
:1045700001E1D3D00201555101E1CFD0189A55BFC6
:10458000188A196B010EE66E7F0E551535ECCBF0CF
:10459000C4D01750800B06E02750200B09E10B0E0A
:1045A000155C06E01D50040B03E01D50080B58E19C
:1045B0002750200B09E01750800B06E013ECCBF0DE
:1045C00003E00B0E155C1CE115EC65F0D7DE2094C2
:1045D00027AAA3D08AECC4F003E00201010E2D6FDC
:1045E000D9ECCCF00601EA5101E197D00701025164
:1045F000800801E292D02F88200E8FECC6F08DD07B
:10460000230E155C10E1010EE66E8BEC0EF0E55208
:104610001EAC03D00201098702D002010681050108
:10462000478D179E7AD05BEC96F0000914E0275076
:10463000200B11E00C50006E020E6FECC9F00C5014
:10464000026E00500C6E0250E66E88EC74F0E5527B
:104650000201196B62D027AA60D0C5EC98F05DD03A
:104660008AECC4F008E02750200B05E0080E076E26
:104670001F0E086E52D0FE0E070102150EE0228EAC
:10468000010E016F02A102D0030E016F02910243DD
:10469000210E076E0501200E07D00201020E526F97
:1046A000220E076E05011F0E156F37D0070101514D
:1046B00012E001072380CFEC64F0076A1DA006D04A
:1046C000020E076E27BA02D024ECD2F0210E086E3B
:1046D0001D80229E22D00201010E526F228E220ED8
:1046E000076E1BD00201525114E023905207CFEC09
:1046F00064F0030E076E1DB007D0070E076E27BAD1
:1047000003D0006A63EC75F0220E086E229E1D90A5
:1047100004D015C507F001D031DE0101E49B120081
:10472000020171510101D880485502E271C248F17D
:104730002B510A0825E2100E2B5D5CECC5F0060E2D
:10474000AFECD3F0016EE251040B13E01B50080BE9
:1047500010E101501E0802E21E0E016E6E0E0201F3
:104760000B5D02E2140E016E5A0E0B5D02E20F0E9B
:10477000016E01500101D880485502E201C048F1A4
:10478000395121E10A0E2B5D05E14851640802E22E
:10479000640E486F02010B51F0ECC3F004E6820E88
:1047A000495C000E4A5806E201014851640802E2E1
:1047B000640E486F6E0E02010B5D05E2CCECCDF08D
:1047C00002E2320E486F2150100B05E0CCECCDF028
:1047D00002E2320E486FD2ECC4F014E101014851FC
:1047E0001E080AE26E0E02010B5D0CE3CCECCDF06C
:1047F00009E3D0ECCBF006E001015FB309D05F83A1
:1048000037EFF7F001015FA303D05F9337ECF7F0C8
:104810001200DACFE4FFE2CFDAFFE9CFE4FFEACF1C
:10482000E4FFE652FC0EB36EF30EB26E0201110706
:104830000201115105E10201320E116F01012181C6
:104840000101E3A92CD00601FD07000EFE5B060165
:10485000FD51FE1124E1F29EF26AF06AB96A9D6A86
:10486000000EA66EA16E9E6E8D8C8D8A8C908494A7
:10487000070E936E0000000000008A9A00000000FE
:1048800000000000270E936E4E0E996E000000008F
:10489000000003000000000000000000FF001E8078
:1048A0001D861D8481B20BD001014FA302D01E9042
:1048B00006D001014FA102D01D9601D01D9481B4F4
:1048C0000BD001014FA302D01E9006D001014FA1D1
:1048D00002D01D9401D01D9687B60BD001014FABBD
:1048E00002D01E9006D001014FA902D01D9601D022
:1048F0001D9481B00BD001014FAB02D01E9006D0A9
:1049000001014FA902D01D9401D01D96020112078A
:104910000201125137E10201050E126F0101AC5183
:1049200016E00101AC07020102015151020B05E042
:104930001D50040B02E1020151810201020151519B
:10494000080B05E01D50080B02E102015185010131
:10495000AD5106E0FF0E0101AD5D02E00101AD2B9E
:104960001FAE04D00601DE2B000EDF2307015051DD
:1049700009E0070150070701505104E151C750F702
:10498000010121830101AB5102E00101AB070101EB
:10499000269701012695010126A102D00101268555
:1049A000010126A302D001012687010126930101FE
:1049B000269188A202D00101268188A002D001019F
:1049C00026830F0E010126150101236F01012351DA
:1049D000EA6AC50FE96E060EEA22EFCF22F1010E58
:1049E0000101221513E01F50080B05E00101010130
:1049F0003B51010B0BE12050200B08E0010122AFDD
:104A000003D00101240702D00101242B9EAA11D05A
:104A10000701942B07019351932BEA6A000FE96E6B
:104A20000C0EEA22AECFEFFF0701945102E192C7CC
:104A300093F7A19207014607E552E5CFEAFFE5CFDC
:104A4000E9FFE5CFDAFF110001013BAB07D03B9B4B
:104A5000238A0601425102E0426B436B12000701B8
:104A6000BEB103D0119A119812001198BEA31188FB
:104A7000119ABEB3118A12000B0E7CECC4F0258E85
:104A8000120012ECC4F003E08AECC4F006E01394C8
:104A9000010156A30ED013840CD0139402013D5192
:104AA00007E10101E251800B03E13B51040B01E0FE
:104AB0001384139613A4138613981350040B04E164
:104AC000D2ECC4F001E013881200E8C1E9FFE9C1AB
:104AD000EAFFEECF49F0EECF4AF0EECF4BF0EECF4B
:104AE0004CF0EFCF4DF0E6C1E9FFE7C1EAFF49C066
:104AF000EEFF4AC0EEFF4BC0EEFF4CC0EEFF4DC0D4
:104B0000EEFF12005FECC3F0A5ECC7F0FB0EDBCFAD
:104B1000E8F1FC0EDBCFE9F101019F0EE66F010E1B
:104B2000E76FD3DF9FEC31F0D8A002D0010E01D0A7
:104B3000000E5BEFC3F018ECCEF00050E66ED3EC45
:104B4000FDF0E552140EE66E32ECFEF0E55247EC55
:104B5000FEF042ECFEF00009FCE1C450006E005093
:104B6000F80812E2C20410E0050EC25C0DE0090E66
:104B7000C25C0AE00D0EC25C07E0110EC25C04E0EC
:104B8000390EC25C01E00006020EE15C02E2E16A5D
:104B9000E552E16E5BEFC3F014ECCEF00050DF6E37
:104BA000460E496ED20E4A6E010E34ECD3F001501F
:104BB000006E009E45ECDAF001AEF2D7E5525BEFF5
:104BC000C3F014ECCEF00050DF6E2350100B1DE14B
:104BD0000050E66E73EC04F0E552800B16E01B0EFD
:104BE000DF5C08E10101200E166F500E176F410EB9
:104BF000186F07D00101450E166F520E186F18C1BD
:104C000017F1200E196F040E016F2A8823A808D00F
:104C1000420E496ED40E4A6E010E34ECD3F007D02A
:104C2000DFCFE6FF73EC04F0E552016EDF2A2AA81D
:104C300002D0019E2A980150006E009E68ECDAF0C6
:104C400001AEE4D72398E5525BEFC3F05CECCFF004
:104C500003E2C0ECCBF004D0FE0EDB50410FF60FA8
:104C6000006E45ECDAF05BEFC3F05CECCFF003E2F2
:104C7000C0ECCBF004D0FE0EDB50410FF60F006EFF
:104C800068ECDAF05BEFC3F028ECD2F0DFDFE5523E
:104C900066ECC9F0DBDFE5525BEFC3F028ECD2F045
:104CA000E4DFE55266ECC9F0E0DFE5525BEFC3F00C
:104CB0005FECC3F00EECCCF0020E01010027BAEC61
:104CC000D9F0DF50006E050E0101005FBAECD9F09B
:104CD000030E0101005FE5525BEFC3F05FECC3F030
:104CE0000EECCCF0FE0EDB50020F0101016FD7EC91
:104CF000D9F0DF50006EFE0EDBCF01F1D7ECD9F01A
:104D0000E5525BEFC3F000C059F2C8ECD3F0FF0EE0
:104D1000005C01E041DF0101B189120000C05AF2DC
:104D2000D8ECD3F0FF0E005C01E04BDF0101B18B4A
:104D30001200C8ECD3F0FF0E005C01E02DDF010192
:104D4000B18D640EA86F24961200D8ECD3F0FF0E3C
:104D5000005C01E036DF0101B18F640EA86F24967C
:104D600012005FECC3F03DECC8F052ECC5F0ECEC87
:104D7000C3F05BEFC3F05FECC3F03DECC8F051EC67
:104D8000CEF0010EE66E54EC08F0E552E5525BEF12
:104D9000C3F05FECC3F091EC6FF00101190EAA6F44
:104DA000FC0EDBCFAEF1FD0EDBCFAFF1FE0EDBCFA5
:104DB000B0F15BEFC3F0830E096EE00EA2ECD3F00E
:104DC000800E005C08E291EC6FF00101190EAA6FF1
:104DD0000201E00EA96F120026ECD3F0DBCF4AF0FF
:104DE000800E4A1407E0A0ECC5F0496C4A1E000E84
:104DF0004A2202D0A0ECC5F009ECD2F05BEFC3F080
:104E00005FECC3F012A60FD0060150B503D001012C
:104E1000FBECC7F0288ABCBF289AFE0EDB5001E0ED
:104E2000287ACEEC40F05BEFC3F026ECD3F0DBAE9B
:104E300008D0DB50FF0DFE0EF3CFDBFFFCECC9F01A
:104E400007D0FCECC9F0DB50FF0DFE0EF3CFDBFF0B
:104E5000DB505BEFC3F014ECCEF007015A5101E0D8
:104E60005DD11D50400B01E059D13250040B01E1DE
:104E700054D10101D05104E18450020B01E14DD124
:104E80000B0EE3ECC4F00601BC6FF2ECC6F001E0DF
:104E9000A5D0140E0601E76EBC19E8AE02D0BC35F1
:104EA00003D0E750D880BC5502E2140EBC6FEC0E64
:104EB000E76EBC19E8AE02D0E73402D0E750BC5D23
:104EC00002E2EC0EBC6FBE51E76EBC19E8AE02D038
:104ED000BC3503D0E750D880BC5502E2BE2B0BD0C6
:104EE000BE51E76EBC19E8AE02D0E73402D0E750FD
:104EF000BC5D03E2BE07BEC6BCF6200E496E4A6A20
:104F0000C1C63DF0C2C63EF015ECCCF03DC0C0F6C7
:104F1000C0C649F04A6A49BE4A6849500601C15FA5
:104F20004A50C25BBCC649F04A6A49BE4A68495009
:104F3000C1274A50C223C0C6E6FF77DFE552016EA3
:104F4000010EE66E0E0E01240BECC6F002011A51A2
:104F500001E1E3D01BAA05D0BCC6E6FFBEEC75F0AC
:104F6000E552C3ECC5F02AE01250080B03E1040E31
:104F70001A1528E0B3ECCEF001E0010E496ED051D5
:104F800003E1CC51400B07E0D05103E0CB51040BBF
:104F900002E0000E01D0010E491809E012A602D06D
:104FA000E66A09D00601BC51010124270BD012A6E4
:104FB00005D0010EE66E24DFE55204D00601BC5197
:104FC0000101245F0601BC5101E0A7D002011A5182
:104FD000320801E3A2D0320E1A6F9FD01B0EE66E8C
:104FE00027EC15F0E552F3CFBCF6F4CFBDF6026A1C
:104FF000016A0601BC51E76EBD19E8AE02D0BD35AD
:1050000003D0E750D880BD5505E2BC51BD5DB2EC80
:10501000C8F0026E0601BD51E76EBC19E8AE02D0C1
:10502000BC3503D0E750D880BC5505E2BD51BC5D0E
:10503000B2ECC8F0016E0601BF51D880025402E202
:1050400002C0BFF6BE51D880015402E201C0BEF6D4
:10505000000EE76EBF19E8AE02D0BF3503D0E750AF
:10506000D880BF5505E2010EE66E0D0E0BECC6F0C2
:10507000010E0601E76EBF19E8AE02D0BF3503D0BE
:10508000E750D880BF5505E2010EE66E0C0E0BEC22
:10509000C6F0020E0601E76EBF19E8AE02D0BF35BA
:1050A00003D0E750D880BF5505E2010EE66E0B0E27
:1050B0000BECC6F0000E0601E76EBE19E8AE02D09A
:1050C000BE3503D0E750D880BE5505E2010EE66E2E
:1050D0000F0E0BECC6F0010E0601E76EBE19E8AE2E
:1050E00002D0BE3503D0E750D880BE5505E2010E90
:1050F000E66E100E0BECC6F0020E0601E76EBE194E
:10510000E8AE02D0BE3503D0E750D880BE5505E2E8
:10511000010EE66E110E0BECC6F03294E5525BEF19
:10512000C3F018ECCEF0FC0EDB506AE102012A510C
:1051300067E10490FE0EDB50140804E2140E26EC26
:10514000C8F00480FE0EDBCF49F05651D880495498
:1051500003E2FE0EDBCF56F201012A51100B03E0F1
:10516000050ED05D05E10450010B02E0FE0EDB2AC6
:10517000010E67C1DBFF050ED05D02E1010EDB6AA7
:10518000010EDB50280803E2DE52280EDD6E050E0C
:10519000A8ECC9F03EC0DBFFDF6A150EDF5C22E23F
:1051A000006AFE0EDB5004E0FE0EDB50DF5C13E312
:1051B00001012A51100B07E0050ED05D04E0020149
:1051C0005651DF5C08E001016751040806E2010E58
:1051D000DB50DF5C02E1010E006E005003ECC8F012
:1051E000DF2ADBD71350010B69E00201215166E190
:1051F0000101D05103E0030ED05D60E132845ED046
:10520000FC0EDB0430E102012A5106E0FD0EDB500A
:1052100003E12250400B55E1C8ECCDF003E2080E4B
:1052200026ECC8F0FD0EDB500C0805E20C0EF36E08
:10523000FD0EF3CFDBFFB2ECC7F0150EDF5C3EE2F4
:10524000FE0EDB5004E0FE0EDB50DF5C07E3090ED0
:10525000DF5C07E3FD0EDB50DF5C03E2010E03ECD5
:10526000C8F0DF2AEAD7FC0EDB50020827E1C8ECC1
:10527000CDF003E2080E26ECC8F0FD0EDB500C0862
:1052800005E20B0EF36EFD0EF3CFDBFFB2ECC7F0C1
:10529000150EDF5C13E2FE0EDB5004E0FE0EDB5069
:1052A000DF5C07E3090EDF5C07E3FD0EDB50DF5C2C
:1052B00003E2010E03ECC8F0DF2AEAD7FE0EDBCFD3
:1052C0000AF2020EE15C02E2E16AE552E16E5BEF96
:1052D000C3F00101D1510AECC8F02AECC6F001502C
:1052E000080D4950F3240A01DF6F4A50F420E06FA3
:1052F00012000101C551C05D0CE1C651C15D09E15B
:10530000C751C25D06E1C851C35D03E1C951C45D27
:1053100001E0000C010C0101D151D05D01E0000C55
:10532000D0510BE1CC51400B01E0010E496ED95137
:10533000400B01E0010E495C2DE0030ED05D23E13E
:10534000D851C2ECC4F00A5C1EE1F2ECC6F00CE0ED
:105350000101CC51040B01E0010E4A6ED951040B3E
:1053600001E0010E4A5C16E0F2ECC6F00CE101012E
:10537000CB51040B01E0010E4B6ED851040B01E040
:10538000010E4B5C07E00101D05103E0030ED05D3C
:1053900001E1000C010CADDF000903E0BCDF0009F6
:1053A00001E1000C010CF7DF000928E02EECC4F04D
:1053B00001E1010CD1510AECC8F0080EE66EE66A74
:1053C000D15163ECD0F00150F2ECD2F0D051100D7D
:1053D000F3CF4FF0F4CF50F02A0E4F260A0E502292
:1053E0000701B151080DBAECC8F04FECFAF0516E5C
:1053F000060EE15E5150000901E1010C000C1AB2E9
:1054000002D0C5ECC8F0D0C1D1F134AA17D0010147
:1054100038A306D0DA93CDB3DA83DA95CDB5DA8541
:10542000D99DCCBDD98DD995CCB5D985D895CBB5DD
:10543000D8858DECD2F01EECCFF01AD00101D151FD
:1054400003E1D99DCCBDD98D030ED15D11E18DEC69
:10545000D2F01EECCFF0F2ECC6F006E00101D995D7
:10546000CCA506D0D98504D00101D895CBB5D88577
:1054700034AA0DD0500EE66EE66A2A0EE66E0A0ECB
:10548000E66E7A0EE66E0A0EB2ECC6F00FD0050E8E
:10549000D05D0CE0100EE66EE66A3BECD3F0D15125
:1054A00063ECD0F032ECCDF05FECC6F0050E0101FC
:1054B000D15D08E0D151EA6ACF0FE96E0A0EEA2207
:1054C000B1C7EFFF1200C5C1C0F1C6C1C1F1C7C16C
:1054D000C2F1C8C1C3F1C9C1C4F1D1C1D0F134AA6C
:1054E00008D03DECCBF02A0EE66E0A0EB2ECC6F008
:1054F00014D02EECC4F011E0100EE66EE66A2AEC31
:10550000C6F0A1ECC4F0D051100D15ECC6F00AECB9
:10551000CDF032ECCDF05FECC6F02EECC4F004E040
:105520002FECC7F0B1C7EFFF12005FECC3F03BDF19
:10553000000916E1F9EC13F0FE0EDB5002E15FDF2B
:1055400001D0C1DFCBECCAF0248A1EAC04D002012A
:105550000983098102D0020106830501478347813F
:105560005BEFC3F0F9EC13F00101C0510CE0C00592
:1055700003E13C0EC15D07E3C55105E0C50514E13B
:105580003C0EC65D11E28AECC6F0348A10D8349A1B
:105590009DEC13F01C8A8AECC6F01C9A188488ECE7
:1055A000C7F0189451EFCAF002D89DEF13F00DC167
:1055B00003F0C5C19AF2C6C19BF2C7C19CF2C8C133
:1055C0009DF2C9C19EF2D1C100F037ECCDF0DAC135
:1055D000DEF134AA08D03DECCBF0540EE66E060E98
:1055E000B2ECC6F011D0050E005C0EE0100EE66EB7
:1055F000E66A01012AECC6F0A1ECC4F0540EE66E96
:10560000060EE66E18ECCCF0016A050E005C03E0B5
:1056100000500AECC8F0F3DE03C00DF19AC2C0F1ED
:105620009BC2C1F19CC2C2F19DC2C3F19EC2C4F132
:1056300000C0D0F134AA1ED0010138A30ED0CD9302
:10564000DEB3CD83CD95DEB5CD851296CDB3128672
:105650001294CDB51284CBECA0F00101CC9DDDBD40
:10566000CC8DCC95DDB5CC85CB95DCB5CB85F1EC7F
:10567000CEF018D00101D05103E1CC9DDDBDCC8D21
:10568000030ED05D0FE1F1ECCEF0F2ECC6F006E0D7
:105690000101CC95DDA506D0CC8504D00101CB95C8
:1056A000DCB5CB8534AA09D0500E1FECCCF02A0E05
:1056B000E66E0A0EB2ECC6F00AD0050E005C07E0FA
:1056C000100E1FECCCF03BECD3F018ECCCF001C08A
:1056D000B1F72EECC4F004E02FECC7F001C0EFFFEF
:1056E00004903BB104803B913BB33B813B9304B0BE
:1056F0003B83129C3BB1128C129E3BB3128ECBECBF
:10570000CAF0248AABDB1EAC06D0020109870985EA
:105710000983098102D00201068305014881BF0E79
:10572000476F12005FECC3F0010162853DEC1EF093
:105730005BEFC3F0370E005C02E2370E006E0050E4
:105740009F0802E29F0E006E630E005C08E2370EB7
:10575000005CE824496E090E43ECC4F005D0630EEA
:10576000005C99ECD0F0090F006E0201D05102E00C
:10577000030E00260050150802E2150E006E1200FE
:10578000B0ECCFF00201215110E12050010B0DE1EE
:1057900024510BE13250100B08E12750200B05E09B
:1057A000D85103E130A003D03090000E70D0FE0E2F
:1057B000DB5002E0990E01D00A0EE3ECC4F05CEC81
:1057C000C9F08C0E3CECCDF00201D05103E0790E13
:1057D0003CECCDF02C5129E1020EDB50A7ECC5F0DA
:1057E00024E30A0EE3ECC4F0496E020EDB50495C80
:1057F0001CE311AE0DD0119E77EC20F00201068D56
:10580000090E0DECC4F026ECCCF0D0ECCDF00DD0B0
:105810000201D05107E107010A9308ECF7F0EBEC25
:1058200052F011840201FA0ED06F010EDB50006EAF
:1058300000509F0802E29F0E006E00504B6E4C6AB3
:1058400005011851070D2CECCCF0030E0F0B03E0F3
:105850006BECC9F0FDE149C018F56CDF0050DF6E5C
:1058600000C0A2F7090E016E01012AB9010613500A
:10587000010B06E00150D880005402E20150006E96
:10588000E66AE66A0050E66E73ECC7F0DF50496ED8
:10589000030EE15C02E2E16AE552E16E49505BEF22
:1058A000C3F035ECCEF0020B1CE00101E251400BDD
:1058B00018E00201685115E1080E155C06E0290E9A
:1058C000155C03E00A0E155C0CE1080E155C02E1A4
:1058D000010E20D0290E155C02E1020E1BD0030E32
:1058E00019D0016A0A0E015C19E2FE0EDB50010BB1
:1058F00006E0230E0124BAECC5F0155C0AE0FE0EAA
:10590000DB50020B09E02D0E0124BAECC5F0155C4A
:1059100003E101500C6E02D0012AE4D75BEFC3F023
:105920005FECC3F0800E0C6E17AE17D0179E1750A9
:10593000010B03E11750100B10E0100E0C6E51EC30
:10594000CEF0AFDFE5522C0E155C02E1200E0C6E9E
:105950000B0E155C02E1400E0C6E5BEFC3F05FECCA
:10596000C3F0D0ECC8F051ECCEF01FEC0CF0E552D7
:10597000ABECD0F00101A46FA451640D29ECC4F08C
:10598000A6ECD0F05C0FE8ECC4F0006EB5ECCFF004
:1059900033ECCCF000504B6E4C6A01014B50495C2B
:1059A000D46F4C504A58D56F29A60BD09A5133EC7E
:1059B000CCF00101D451495C0E6ED5514A580F6E9E
:1059C00006D09A510F6AD4250E6ED5510F22ADEC38
:1059D000CDF0E6ECCEF03DC0A4F139C09AF15BEF1A
:1059E000C3F05FECC3F0D0ECC8F0DB505CECC5F06A
:1059F000030EAFECD3F00101A45D02E0000E1BD05A
:105A0000FE0EDB505CECC5F0020EAFECD3F09A5DFD
:105A1000006E00BE006C040E005C0AE32FECCFF0B9
:105A200009E0945107E0A45105E0190E005C02E280
:105A3000010E01D0000E5BEFC3F0010EE66E70DFC9
:105A4000E55200680A0E0C5C02E20C501DD0200EDC
:105A50000C5C02E10E0E18D0400E0C5C02E10F0E41
:105A600013D0100E155C02E10A0E0ED0180E155C54
:105A700002E10B0E09D0110E155C02E10C0E04D0F0
:105A8000190E155C02E10D0E006EFF0E005C1DE0AC
:105A90000050E66E8E0EBEECC3F0300EE66E8F0E3A
:105AA000BEECC3F0C80E9EECC3F017A808D057ECAC
:105AB000CAF0000904E0140E9EECC3F0F8D7E66AC1
:105AC0008F0EBEECC3F0179E010C000CD7ECD0F08B
:105AD000920E491810E14A500EE1006A83EC26F05C
:105AE000B80E17ECCBF00101A86B21860201776B91
:105AF000696B289E072AD7ECD0F0930E49185CE119
:105B00004A505AE1010EE66E0BDFE5520A0E0C5CBC
:105B100032E202017751050833E36951020830E3AC
:105B2000772B28BE692B010E016E070E015C13E274
:105B300001285DECC4F0EF50006E060E015C05E13B
:105B4000800E010115150C10006EDBECD0F000C0CA
:105B5000EFFF012AEAD70101159F36AD2DD00C5079
:105B600002E1540E02D0300E0C24006E800E0010A4
:105B70002BECC8F010D0200E0C5C12E128AE02D045
:105B8000258E1AD0288E0101158FD20E2BECC8F06D
:105B9000010136AD11D00501930E4B6F1E0E0BD0D7
:105BA000400E0C5C04E1980E076E1A8805D0100EAA
:105BB0000C5C02E19A0E076ED7ECD0F0980E4918F3
:105BC00075E14A5073E1010E016E070E015C0DE2B2
:105BD000DBECD0F0EF9EDBECD0F0EF500E0803E1F1
:105BE000DBECD0F0EF6A012AF0D70FC1A4F10A0E66
:105BF00001011003F35011259A6F0A0E1203F3509E
:105C000013259B6F0A0E1403F3CF9CF19E6B9EC16C
:105C10009DF1040E0201775D0DE269510BE112C1A5
:105C2000A4F10A0E01011303F35014259A6F9C6B23
:105C30009CC19BF10201690508E111C1A4F19BC15E
:105C40009AF19CC19BF101019C6B020E0201695DFE
:105C50000EE110C1A4F10A0E01011103F350122547
:105C60009A6F0A0E1303F35014259B6F9C6B9A0EC8
:105C7000076EDCEC0CF0006E005013E10101A45142
:105C800003E19A51380802E2258E120018ECC7F0A1
:105C90000A0E005C06E10101DF51010B02E0FEEF9C
:105CA00008F000C02BF129840EECD2F0D7ECD0F034
:105CB0009A0E491808E14A5006E10101B19BB199D9
:105CC00003D80C0E076E120041ECCDF02582238A1A
:105CD00012003EC2A3F13FC2A2F140C2A1F10101F4
:105CE000A06B9F6B1FA402D07BEF31F09FEF31F0D0
:105CF00004902C50100B01E00480ADECF7F02C5018
:105D0000100B01E0010E496E0450010B495C02E0EA
:105D100030ECC8F01200B3ECD3F001018DA715D020
:105D2000FE0EDB5008E0FD0EDB5005E1DF68CBA185
:105D300002D0010EDF6EFE0EDB5007E1FD0EDB50E0
:105D400004E0010EDF6ECBB1DF68DF5021E06AECCA
:105D5000C4F0A36BA3C1A0F1A3C19FF12CECD2F0BE
:105D600001E0010E496EDF0402E0000E01D0010ED9
:105D7000491802E0C0DA01D0E2DA7CEC04F01EAC93
:105D800003D00201098102D0020106830501478187
:105D9000E5525BEFC3F00101A36BA26BA16B0201A3
:105DA0008851E824496E640E68ECD0F017ECFEF0E0
:105DB0003AC0A0F1320EAFECCEF088C23EF017EC44
:105DC000FEF03EC09FF1020189A102D07BEF31F0CD
:105DD0009FEF31F030ECD2F09AC23BF03C6A3D6A62
:105DE0003E6A45ECCBF0D6ECFBF037C0DEFF38C0A6
:105DF000DEFF39C0DEFF3AC0DDFFDD52DD529BC25F
:105E000049F0D4ECCDF0100E406E270E416EA6EC9A
:105E1000C4F09CC249F0D4ECCDF0640E406E416AEF
:105E2000A6ECC4F00A0E02019D03F3509E25496EB4
:105E3000D4ECCDF086ECCFF0DECF3BF0DECF3CF003
:105E4000DECF3DF0DDCF3EF0DD52DD52040EE15CF1
:105E500002E2E16AE552E16E5BEFC3F007AE6ED09D
:105E60002B50400B03E02C50200B31E0800E010141
:105E7000C01505E1C0510CE11F0EC15D09E2C06B08
:105E80001F0EC16FC46BC4C1C3F1C4C1C2F11FD026
:105E9000100E2B5D1CE2360E006E0050C05D03E359
:105EA00000C0C0F10DD0200EC05D11E32C0EC05D0E
:105EB0000EE2260EC05D02E2200E01D02C0EC06F55
:105EC000C46BC4C1C3F1C4C1C2F1C4C1C1F12B5080
:105ED000400B03E02C50200B31E1800E0101C51571
:105EE00005E1C5510CE11F0EC65D09E2C56B1F0E31
:105EF000C66FC96BC9C1C8F1C9C1C7F11FD0100EA7
:105F00002B5D1CE2360E006E0050C55D03E300C041
:105F1000C5F10DD0200EC55D11E32C0EC55D0EE25E
:105F2000260EC55D02E2200E01D02C0EC56FC96B96
:105F3000C9C1C8F1C9C1C7F1C9C1C6F12B50400BD5
:105F400003E02C50200B1DE02050400B03E11250C9
:105F5000080B0FE12050400B12E01F50020B03E131
:105F60001250040B06E11F50020B09E01250080BFF
:105F700006E06AECC4F0ADDEDBECC8F002D0E6EC83
:105F8000C8F02B50400B03E02C50200B16E11F50A3
:105F9000020B11E01250040B0EE033ECC6F099DE58
:105FA0009AC1BBF19BC1BCF19CC1BDF19DC1BEF1C9
:105FB0009EC1BFF102D0F1ECC8F01F50020B18E1F6
:105FC00002018951010B03E18951020B11E02EEC12
:105FD000C4F006E02050800B0BE0050E995D08E14F
:105FE0002050400B05E03EECC6F0D5DEDBECC8F0FF
:105FF00001013BA974D0B6C19AF2B7C19BF2B8C1F6
:106000009CF2B9C19DF2BAC19EF2E4DE3BC0C8F772
:106010003CC0C9F73DC0CAF73EC0CBF7BBC19AF23E
:10602000BCC19BF2BDC19CF2BEC19DF2BFC19EF23C
:10603000D1DE3BC0CCF73CC0CDF73DC0CEF73EC073
:10604000CFF70701C851CC5FC951CD5BCA51CE5BB8
:10605000CB51CF5B0101CEA108D0400E0701CC2768
:106060001F0ECD23000ECE23CF23049C1E50200BE9
:1060700001E0048CD8800701CF51FF0A08E6680EC2
:10608000CC5DC50ECD59FF0ECE59FF0ECF5919E389
:10609000CF35000ECF1909E6D880980ECC553A0EB0
:1060A000CD55000ECE55000ECF550BE3CCC70EF0EC
:1060B000CDC70FF0B0ECC5F0A50E85ECC3F01E8A7D
:1060C00001D01E9A0450400B01E0010E496E1E5093
:1060D000200B01E0010E495C02E0B5ECC5F02BACF1
:1060E00096D0800E071401E192D0100E01012B5DB5
:1060F00001E38DD02CBA0DD0FCECC8F0C5C19FF1E6
:10610000C6C1A0F1C7C1A1F1C8C1A2F1C9C1A3F123
:106110000CD03EECC6F0C0C19FF1C1C1A0F1C2C11C
:10612000A1F1C3C1A2F1C4C1A3F118ECC7F02C5076
:10613000200B2EE0005001012B5D2AE000C00DF184
:1061400000C02BF12BC1CFF13AECCCF012ECC8F02F
:10615000056E2CAA06D0050EE66E0524CFECCAF01B
:1061600005D0050EE66E055074ECC9F0D1ECC3F015
:106170000E0E05242FECC5F00101CE9B00BACE8B8C
:10618000096A97EC35F020820201010E246F01D0DC
:10619000AFDD0701C2510101C05D04E0B4EC0DF0B8
:1061A000C0C1C2F701012B5132E12B50080B2FE087
:1061B000020E3A5D2CE1D5ECCFF004E00BECCBF015
:1061C000E806FCE10701C6510E1802E1C7510F189D
:1061D0001EE0006A5A0E0E1807E10F5005E1590E35
:1061E000C61901E1C7510AE0590E0E1808E10F5017
:1061F00006E15A0EC61903E1C75101E1002A0EC09B
:10620000C6F70FC0C7F70050E66E02D8E55212007D
:106210005FECC3F0010139516CE12B516AE12B5065
:10622000080B67E0FE0EDB5003E1020E3A5D61E110
:10623000D5ECCFF004E00BECCBF0E806FCE10EC0AF
:10624000C6F70FC0C7F7190E93ECC9F003E2036855
:1062500002681DD0410E93ECC9F015E22AECCFF094
:10626000190E495E000E4A5A4950016EB7ECCEF045
:106270000800F550026EB7ECCEF0F62A79ECC9F0C2
:10628000F550036E04D069C302F06AC303F0010144
:1062900096A904D069C302F06AC303F0FE0EDB5076
:1062A00007E10701C351025C03E1C451035C21E033
:1062B00002C0C3F703C0C4F7410E93ECC9F011E26A
:1062C00001019651100B0DE1010EE66EE66A0350D6
:1062D000E66E0250E66E3DECC7F00B0ED4ECCAF051
:1062E00005D0FE0EDB5002E040ECCCF00A0E23ECB1
:1062F000CDF05BEFC3F00101A3519E279E51090829
:1063000003E20A0E9E5F9D2BA2519D279D51090815
:1063100003E20A0E9D5F9C2BA1519C279C516308B0
:1063200003E2640E9C5F9B2BA0519B279B5163084B
:1063300003E2640E9B5F9A2B9F519A271200010182
:10634000A3519E5F9E510A0803E20A0E9E279D07F5
:10635000A2519D5F9D510A0803E20A0E9D279C07EA
:10636000A1519C5F9C51640803E2640E9C279B072B
:10637000A0519B5F9B51640803E2640E9B279A0720
:106380009F519A5F12000101E2A53BD0E1A902D022
:10639000310E01D05E0E9A2707ECC9F01BDD21EC0F
:1063A000C7F0030E406E416A426A06ECD1F0F6EC8B
:1063B000C5F045ECCBF0ECECFCF03BC09AF105EC01
:1063C000CAF0F6ECC5F0100E406E270E416E426A20
:1063D000436AECECFCF03BC09BF137C00EF038C0D8
:1063E0000FF0ADECCDF0E6ECCEF03DC09CF1FAEC58
:1063F000C3F039C03EF017ECFEF03EC09DF13AC04C
:106400009EF1120018ECCEF02BBC03D01AD82F9EB0
:1064100010D02CAA07D02050400B0AE01F50020BCE
:1064200008E106D02050400B04E01F50020B01E0B1
:1064300008D8020EE15C02E2E16AE552E16E5BEF30
:10644000C3F018ECCEF00101E451010BDE6EDD6A01
:106450001F50020B06E02050400B03E0FCECC8F09C
:1064600002D03EECC6F0A36BA3C1A2F1A3C1A1F17F
:10647000A3C1A0F1A3C19FF120ACE4912050400B37
:1064800010E1D0510EE12CECD2F001E0010ED9EC7C
:10649000C6F002E0000E01D0010E491801E081D0E3
:1064A0007CD02050400B12E03450400B0FE02CEC1D
:1064B000D2F001E0010E496E020ED05D02E0000E46
:1064C00001D0010E49186DE13ADF6CD02050400B2D
:1064D00019E1D00503E0020ED05D14E145ECCDF0EA
:1064E00011E201010F0EA16FE251040B01E0010E58
:1064F000496E020ED05D02E0000E01D0010E491877
:106500004CE04FD0D4ECCBF014E00101090EA16FA8
:10651000010EA26F050EA36FE251040B01E0010E04
:10652000D9ECC6F002E0000E01D0010E491835E0AA
:1065300038D02050400B13E1DAECC9F010E0010133
:106540000A0EA16FE251040B01E0010ED9ECC6F076
:1065500002E0000E01D0010E49181FE022D02050A9
:10656000400B20E12EECC4F003E0040ED05D1AE1F4
:10657000010EA06F0A0EA16F040ED05D03E1E2A52B
:1065800010D00BD0E251040B01E0010E496EE15135
:10659000800B01E0010E491804E0D1DE0101E48125
:1065A00001D0A9DE0101E251010B2DE02050400B8A
:1065B0002AE1020114511DE00101E451010B496E71
:1065C0004A6ADF50491813E1DE52DD504A180FE1E4
:1065D0000201A0510101A05D0AE10201A1510101E6
:1065E000A15D05E10201A2510101A25D02E00501E8
:1065F00047859FC19FF2A0C1A0F2A1C1A1F2A2C193
:10660000A2F2A3C1A3F2FFECCAF015E02050400BA8
:1066100012E1050ED05D0FE0040ED05D0CE09F6B23
:10662000A06B500EA16FA36BA3C1A2F1E2A502D093
:1066300062DE01D084DE0101E2B5A5DED5ECC7F053
:106640001BE2100E2B5D34ECC8F00101A06BA0C161
:106650009FF135ECD2F0A16F3AECD2F0A26FA36BB0
:10666000E251040B01E0010E496E3FECD2F04918F3
:1066700002E065DE01D03FDE010196B374D057A978
:1066800043D057AB70D0D2C70EF0D3C70FF0260E51
:10669000D8800E54020E0F5406E20480260E0E5EC1
:1066A000020E0F5A06D00490260ED8800E56020E07
:1066B0000F569B51496E4A6A9A51640DF350492412
:1066C000D46FF4504A20D56FD4C14DF0D5C14EF0EF
:1066D000F5ECC4F037C03BF038C03CF039C03DF0B9
:1066E0003AC03EF0880E406E130E416E426A436A15
:1066F000ECECFCF03BC00EF03CC00FF0A0ECC6F0A0
:1067000004A030D01CDE2FD09AC100F0000405E1B7
:106710009B51310802E2020E006E030E005C05E19F
:106720009B51310802E2040E006E98514F6E506A80
:1067300000504D6E4E6A0A0E4B6E4C6AB2C23DF06E
:10674000B3C23EF0A1ECD0F0BDECFDF07DECD3F097
:10675000AEECC8F04FC042F050C043F066ECC6F05B
:10676000A0ECC6F0C8DDC3ECC5F003E1B8ECCBF09B
:1067700019E00601F05101019C5D14E10601EF51A1
:1067800001019B5D0FE10601F15101019D5D0AE1EF
:106790000601F25101019E5D05E10601EE51010184
:1067A0009A5D0CE09AC1EEF69BC1EFF69CC1F0F643
:1067B0009DC1F1F69EC1F2F630ECF1F0020EE15C03
:1067C00002E2E16AE552E16E5BEFC3F0D9CFE6FF8A
:1067D000E1CFD9FFB6C19AF1B7C19BF1B8C19CF125
:1067E000B9C19DF1BAC19EF10101A46BFE0EDB504F
:1067F0000A0807E22996FE0EDBCFE6FFAFEC2CF08D
:10680000E5520101006B800E01011315036E800E2D
:1068100001011015026E010EEA6E9A5105D89B51C6
:1068200003D89C5101D814D0076B066F0A0E065D81
:10683000D8A003D0066F072BF9D700510E0FE96ED1
:106840000751EF6EE92A0651EF6E002B002B000C6A
:106850009DC114F19EC115F10101A45107E10A0E79
:1068600001019A5D03E20101100E0E6F0701BEBB2C
:1068700003D00101100E156F0701BEAD05D0010157
:10688000100E146F14C115F11DBC03D00101108F3F
:1068900003D00250010110130101138F0101A45113
:1068A00009081AE20201365117E0C8ECD3F00101E1
:1068B000020E006F9AC100F0BAECD9F0A4C100F04A
:1068C0000101006BBAECD9F0010EE66EE66A21EC2C
:1068D00009F0E552E55223D00101A4511FE0070160
:1068E0000701BE51200B1AE1288C14C115F113C108
:1068F00014F112C113F111C112F110C111F10FC144
:1069000010F10EC10FF10A0E496E49C043F0A4C147
:106910003EF017ECFEF03AC00EF101D0289CE55293
:10692000E7CFD9FF1200D9CFE6FFE1CFD9FF020EA2
:10693000E126010EA4C1DBFF2BC1DFFF0101D15114
:10694000EA6AB80FE96E070EEA22EFCFBFF7BBC1C4
:106950009AF1BCC19BF1BDC19CF1BEC19DF1BFC10B
:106960009EF10101A46BDF500A0806E22996DFCFF1
:10697000E6FFAFEC2CF0E5520101016B800E010146
:106980001B15026E010EEA6E9A5105D89B5103D871
:106990009C5101D816D0076B066F0A0E065DD8A071
:1069A00003D0066F072BF9D70151160FE96E075177
:1069B000300FEF6EE92A0651300FEF6E012B012BDD
:1069C000000C300E01019D2501011C6F0101A45135
:1069D00007E10A0E01019A5D03E20101200E166F24
:1069E0000701BFAD03D00101200E1C6F0101188FFC
:1069F00001011B8F0101A4511DE007010701BF51D7
:106A0000200B18E11BC11CF11AC11BF119C11AF1AD
:106A100018C119F117C118F116C117F10A0E496E04
:106A200049C043F0A4C13EF017ECFEF03A50300FDD
:106A30000101166FA4C1A5F1010EDBCFA4F1020E76
:106A4000E15C02E2E16AE552E16EE552E7CFD9FF8F
:106A5000120014ECCEF0830E096E0A0EE66E0101F0
:106A60000D03F350E66E5E0EE66E020ED1ECC3F03F
:106A7000DE0E2FECC5F00050DF6EFE0EA2ECD3F060
:106A80000101E19D2E9EB90E005C16E1FF0E020190
:106A90005E5D12E02E8E020E01012B5D0DE1050EF2
:106AA0000201635D09E1210E5F5D01E1606B280E6B
:106AB000645D02E13C0E656FA30EDF5C02E1010143
:106AC000E18DE5525BEFC3F08C0E02018D1909E1F7
:106AD0000A0E8E1906E18C0E8F1902E10A0E90192A
:106AE00007E0800E8E1504E1800E901501E1000C88
:106AF000010C0201915102E1925107E0FF0E915DFC
:106B000004E0FF0E925D01E0000C010C2B50080B1D
:106B10000DE0B3ECCEF00AE12B5106E1010EE66E7A
:106B200008EC31F0E552120040ECCCF0120018B045
:106B30003DD00DC1E6FF57EC5AF0E552C5DF000924
:106B400002E0B1ECC9F00DC1E6FF73EC5AF0E5527A
:106B5000D0DF000903E00201916B926BE8EC15F0C5
:106B600078DF01015651080B03E12B51090809E2B6
:106B7000FF0E02018A5D02E1320E8A6F8AC248F17D
:106B800008D0FF0E8C5D03E1320E8C6F02D08CC1F9
:106B900048F18DEC41F001015F8DE2B55F9D59EC4C
:106BA000F6F049ECC5F0B7ECCAF0B0DFCBEFCAF0B5
:106BB00014ECCEF0FD0EDB50100DF350DF6E010E25
:106BC000096E0201680E986FFD0EDB500A080AE29A
:106BD000020E096E690E986FFD0EDB50F00F100D5E
:106BE000F350DF6EFE0EDB50FF0802E0DFECCFF06B
:106BF000DF50E5525BEFC3F00201875103E087519C
:106C0000330802E20D0E876F8851CEECC4F007E224
:106C10004950FA08000E4A5402E21E0E886F89BFDE
:106C2000896B93510E0803E2936B0101CC9B120018
:106C300026ECCFF0FF081BE0DFECCFF00F0ED4EC1A
:106C4000D0F00A0E005C07E10101DF51010B03E007
:106C5000096A000EBCD100C02BF101018A51100B52
:106C600006E00A0EDBECC3F002E2FE0EDB682BC18D
:106C70000DF10201756B0101E295E1992B510A08B2
:106C800038E2100E2B5D006E00509CECCFF029E036
:106C9000A6ECD0F001010D6F8AECC3F0EF380F0BBA
:106CA0000201756F2FECCFF024E01B50020B0EE0B9
:106CB0002B50080B03E12250080B08E00101E2858C
:106CC000B5ECCFF0460815E1E18913D00701020EBB
:106CD000266F1BA202D0050E266F180E80ECC4F0A2
:106CE00008D0FE0EDB680101090E0D6F0DC12BF1FE
:106CF000258E0101E2A50FD02BA605D00701139721
:106D0000140E4AECCDF022A603D0010E4AECCDF0D1
:106D10000701149F0FD02BA605D007011387140E6F
:106D2000D4ECCAF022A603D0010ED4ECCAF00701BD
:106D3000148F149323ECCEF001014FECCDF001E061
:106D4000098FCEECCEF0840ECEECC3F007010B8998
:106D50000101E2A502D007010B9907ECF7F002014F
:106D6000D86B07ECC5F0100E18ECD0F029A403D0B6
:106D70007CEC04F029940F0E0101CA15D06FCA39BA
:106D80000F0BD16FD151060802E2D0C1D1F1D0056D
:106D900001E1CB91020ED05D01E1CB818DECD2F00F
:106DA0000A6E040EE66E0B0EDF24E66ED80EE66E5B
:106DB000010ED1ECC3F007ECC5F0FE0EDB50FF086E
:106DC00003E198C209F002D0100EDF26100E2AEC63
:106DD000D3F0FFECD0F0FE0EDB50FF0852E012ECD7
:106DE000C8F0DF6E0B0ED4ECD0F07DECC5F008E0FF
:106DF0001F0ECB17E00E0014CB138DECD2F00A6EF1
:106E00000C0ED4ECD0F0440E0101CC17BB0E0014D4
:106E1000CC1390ECD2F0470E0101CD17B80E001440
:106E2000CD1390ECD2F09E0E0101CE17610E00142E
:106E3000CE1398C209F00A0EE66E030EDF24E66E4A
:106E40008A0EE66E020ED1ECC3F012ECC8F0DF6ED3
:106E50000C0ED4ECD0F0440E0101D917BB0E001477
:106E6000D91390ECD2F0470E0101DA17B80E0014D6
:106E7000DA1390ECD2F09E0E0101DB17610E0014C4
:106E8000DB13096AC0C119F5C1C11AF5C2C11BF5EE
:106E9000C3C11CF5C4C11DF5C5C11EF5C6C11FF592
:106EA000C7C120F5C8C121F5C9C122F518B41CD04D
:106EB00012941296129A1F92010138A30CD0CDA100
:106EC00002D0128A1F821296CDB312861294CDA5DB
:106ED00009D0128407D0F8ECCBF00101DA95DA93EF
:106EE000CD95CD93CBECA0F0D5ECC7F03DE25C0E98
:106EF0000D25E8ECC4F0006E00500101C05D016E8C
:106F000001AE03D0C051005C016EE251040B03E1FD
:106F10000150030803E3015019080AE2050EE2ECF0
:106F2000C9F0C00EE66E010E21ECC4F000C0C0F145
:106F300000500101C55D016E01AE03D0C551005C7A
:106F4000016EE251040B03E10150030803E3015019
:106F500014080AE2050EE2ECC9F0C50EE66E010E59
:106F600021ECC4F000C0C5F1D9ECCAF041EC25F029
:106F70004AEC0DF0129C01013BB1128C129E3BB306
:106F8000128E1CEC64F0129801013BB912887FEC60
:106F900020F00101CC9F119011825DEC09F06AECA8
:106FA0004EF025EC4EF0096A010137A702D001EC42
:106FB00048F0E6ECC8F0F1ECC8F0B9DD0101246B53
:106FC0001DBC04D00701A16B3AECCCF0010EE552D8
:106FD0005BEFC3F014ECCEF00B0E01012B5D11E260
:106FE000C1C1E6FFC0C1E6FF32EC21F0E552E55237
:106FF000005001012B5D05E00701020EA7ECCFF068
:107000006ED00A0E2B5D02E248C18CF107ECC5F090
:1070100077EC20F00101CC9F38A30DD0F80ECD17EE
:10702000CD911FB2CD81CD9312B6CD83CD9512B443
:10703000CD85B6EC40F02BC1CFF1E8ECCFF0050EDA
:1070400074ECC9F02AECD3F0C9ECC3F00A0EDF24CB
:10705000016E0101D139F00BD01197ECC9F0050E8A
:10706000E66ECB0EE66E010EE66E0B0EDF2403EC31
:10707000CFF0050ECFECCAF0E66E050EDF2403EC70
:10708000CFF01CBA24D007ECC5F001015651080B13
:1070900003E12B51090802E248C18AF2DAECBBF0A5
:1070A0003AC18BF2FE0EDB50FF0803E198C209F0F3
:1070B00002D0100EDF26100EE66E870EE66E020E70
:1070C0002AECD3F0C9ECC3F0096AF9EC13F0010122
:1070D00037A702D07CECC8F0096A0201206BE552A8
:1070E0005BEFC3F014ECCEF00F0EDF6EF40E060172
:1070F0000017F00E0517DF500617E5525BEFC3F0DF
:10710000060106910095019102990199149913992C
:107110000499039112005FECC3F0B3ECCEF001E0F0
:10712000010E496EFE0EDB5002E0000E01D0010E92
:10713000491803E00601058502D006010587010113
:107140008AA102D00601068D5BEFC3F00050050A4C
:107150004FE0010A4AE0070A22E0010A1BE0030AA5
:1071600017E0010A01E0120006010583B3ECCEF03E
:1071700001E0010E496ECC51400B01E0010E4918AF
:1071800002E0060105810601EA5146E0068B120085
:10719000E66A02D0010EE66EBEDFE552120006017D
:1071A0000081B3ECCEF001E0010EBBECC9F002E0CF
:1071B000060105810A5003E0030E0A5C02E10601A4
:1071C0000571C4ECCDF002E00601068B32A024D09C
:1071D000B3ECCEF001E0010EBBECC9F003E0060118
:1071E00005871200060105851200060100831200C2
:1071F0000601008702018951040B04E03A5102E1C3
:107200000601068B020189A102D00601068D02014A
:1072100089A302D00601068F1200800E071406E033
:107220002050010B03E1D0C100F003D038EC20F076
:10723000006E58DFA6EF38F012005FECC3F07DEC73
:10724000C5F00DE10A0403E0020E0A5C04E1CC5132
:10725000040B16E10BD0CB51040B08E011D0D00584
:1072600007E145ECCDF002E2420E21D0450E1FD0E1
:10727000020ED05D07E145ECCDF002E2400E17D0E2
:10728000440E15D0050ED05D07E1E151800B02E000
:10729000480E0DD0470E0BD0040ED05D02E1460E15
:1072A00006D0CC51400B02E1430E01D0410ECEEC92
:1072B000C3F0F6ECC6F0030E005C12E10A0403E032
:1072C000020E0A5C05E10101CC51040B05E106D078
:1072D0000101CB51040B02E0540E1CD0550E1AD004
:1072E000000402E1520E16D0020E005C02E1500EC4
:1072F00011D0050E005C02E1570E0CD0040E005CAC
:1073000002E1560E07D00101CC51400B02E1530EB1
:1073100001D0510ECEECC3F05BEFC3F0B0ECCFF078
:107320002EECC4F00CE12A50020B01E0010EE66ED7
:10733000D950010F4DECCBF02A929EEC16F033B8E9
:1073400042D02050800B12E11450100B0FE014506B
:10735000200B0CE10101D05106E0030ED05D03E0EB
:10736000050ED05D03E114988EEC4FF02050800B99
:107370000AE11450200B07E02EECC4F004E1149A4B
:1073800014988EEC4FF07DECC5F003E0050ED05D57
:1073900001E1CE9D1390D05103E113908AB5138083
:1073A000030ED05D05E10A5003E013908EB5138003
:1073B000139A13A0138A5FEC0CF01CEC64F00AEC37
:1073C00019F041EC25F0258202EC32F0010EE66E58
:1073D00034DFE552EEEC16F012EC1EF033B85FD05D
:1073E000D5CAE6FFAB0EBEECC3F01CEC19F08EEC78
:1073F0004FF092EC0FF089EC1FF0C4EC1EF028B2B5
:107400004ED01C9834902450010B05E12750200BDE
:1074100002E0D5EC08F00E6A0F6A07ECCBF004E14D
:10742000100E0E6E270E0CD0050ED05D04E1240E5A
:107430000E6E2C0E05D0CEA104D0400E0E6E1F0E87
:107440000F6EB0ECC5F0A40E85ECC3F02EECC4F0CA
:1074500003E0050ED15D02E143EC0CF0B9EC1EF047
:107460006F0ECEECC3F0EBEC52F031EC1FF0A0EC61
:107470001DF029EC19F08BEC15F012ECC4F002E0D1
:1074800023EC1EF0B3EC15F0050E005C02E10BECF2
:1074900009F090EC23F07FEC64F037ECF7F02EEC81
:1074A000C4F00AE1010EDB502A92E8B02A822AB227
:1074B00003D02A82A5EC16F03398030EE15C02E2B9
:1074C000E16AE552E16E5BEFC3F08C9800000000CA
:1074D000030EE66E2DEC5CF0E552040E095CE66EE0
:1074E0002DEC5CF0E5520150E66E2DEC5CF0E552BF
:1074F00090ECFDF0006E00008C881200D9CFE6FF02
:10750000E1CFD9FF8C9800000000060EE66E2DEC4E
:107510005CF0E5528C880000000000008C980000B0
:107520000000020EE66E2DEC5CF0E552040E095CE4
:10753000E66E2DEC5CF0E5520150E66E2DEC5CF051
:10754000E552FE0EDBCFE6FF2DEC5CF0E5528C88B9
:10755000040EE66E62ECFDF0E552E552E7CFD9FF8E
:10756000120018ECCEF00050DF6E010EDB6A3CD842
:10757000DF50005C31E0680E095C02E1012A01067F
:10758000040E095C16E2F29EA6980950636E015043
:10759000626EDF50616E7F9E7F9C7F84550E7E6E93
:1075A000AA0E7E6E7F82F28E040E44ECD2F07F949F
:1075B00013D0010EDB2ADFCFE6FFA0DFE55285DF27
:1075C000DF50005C02E037EC0DF0DF50005C04E0BF
:1075D000050EA7ECC5F0EDE3020EE15C02E2E16A04
:1075E000E552E16E5BEFC3F018ECCEF0010EDB6A02
:1075F000040E095C0AE20950636E0150626E7F9EC0
:107600007F9C7F806150006E12D0010EDB2A5DDF0F
:107610000050DF6E5ADF0050DF5C02E037EC0DF007
:107620000050DF5C04E0050EA7ECC5F0EEE3020EAF
:10763000E15C02E2E16AE552E16E5BEFC3F05FEC10
:10764000C3F046ECCCF013E0FC0EDBCFF3FFDB2AFB
:10765000F3502FECC5F0FD0EDBCFE9FFDB2AFE0E69
:10766000DBCFEAFF01E3DB2A00C0EFFFEAD75BEFE5
:10767000C3F05FECC3F046ECCCF01BE0ADECCAF01D
:1076800018E359ECD1F005E24950A408000E4A5421
:1076900010E340ECCAF0016EFC0EDBCFE9FFDB2A01
:1076A000FD0EDBCFEAFF01E3DB2AEF5097ECC9F0D8
:1076B000E2D75BEFC3F05FECC3F01F0E0501235D63
:1076C0000DE2232B2551EA6A270FE96E050E8FEC98
:1076D000D0F0252B25511F0801E2256B5BEFC3F08D
:1076E0005FECC3F0030E0A5C54E10E6A0F6AFE0EF3
:1076F000DB500D0803E11F0E0E6E0F6AFE0EDB500D
:107700000A0803E11D0E0E6E0F6AFE0EDB5009081B
:1077100003E1EF0E0E6E0F6AC8ECCDF003E10E68C8
:10772000020E0F6EFE0EDB507F0804E1B50E0E6EEA
:10773000030E0F6EFE0EDB501F0821E27F0EDBEC06
:10774000C3F01DE2410EDBECC3F00CE3FE0EDB5098
:107750005A0808E3200E496EFE0EB0ECD0F0FE0E83
:10776000E7CFDBFF540E496ED10E4A6E010E4B6E11
:10777000FE0EDB50E00FDCECD2F0A2ECD1F00E50AC
:107780000F1049E00FC0E6FF96DFE5520EC0E6FF9E
:107790003DD0FE0EDB50090803E1200E26ECC8F0B8
:1077A000016A400E015C37E2060E4A6EDF0E4B6E38
:1077B000010E4C6E01504CECC4F0FE0EDB50495CE7
:1077C00028E1030E066E01B0068C01B2068A01B4F0
:1077D000068801B6068601B806842350040B09E129
:1077E000200E011406E06F0EE66E65DFE55223847D
:1077F0000BD02350040B08E0200E011405E17F0E8E
:10780000E66E59DFE55223940650E66E54DFE552EA
:1078100002D0012AC6D75BEFC3F014ECCEF0800E85
:10782000DBECC3F003E3200E26ECC8F00201050EEA
:107830002D6FFE0EDB50740810E1010E2D6F030E4C
:107840000A5C07E1050123515CECD1F0020F020153
:107850002D6F0501106B1D822BD0FE0EDB5028E032
:10786000DF6A150EDF5C11E2A9ECD1F00BE1DF2A33
:10787000C1ECC6F054ECCDF0DF2AC1ECC6F054ECFC
:10788000CDF003D0030EDF26ECD7150EDF5C04E14C
:1078900051ECCEF025DFE552200EDBECC3F003E225
:1078A000200E26ECC8F051ECCEF0E4EC6FF0E5527F
:1078B000E5525BEFC3F018ECCEF023A012D01DB060
:1078C00009D00201535D1CE30701016B026B53C237
:1078D00054F216D00201532B535180081BE2800E44
:1078E00018D01DA010D0070E0701015D09E2012B81
:1078F00002910243020E0201535D02E30701028F6F
:107900000201010E06D00201532B5351800802E2FE
:10791000800E536F1D9023B01D802350010B03E197
:10792000020E535D04E01D50020B01E18AD01DA23E
:1079300004D00701CC0E026F0FD007010291024361
:10794000028F070ED8800155016E01500106000913
:1079500003E002910243F9D700C709F00101B1A782
:10796000E48B0201545107081DE254513F0802E222
:107970003F0E546FC6ECCAF006E0200E8FECC6F046
:10798000200E54ECCDF09AECC9F00CE00701035145
:1079900009E0800E02015425006E03C701F00701C3
:1079A0000307DFDD780E0701025D18E2298A02C7AE
:1079B000E6FF3CEC04F0E552DF6EDF500EE0C6EC73
:1079C000CAF00BE02D5104E0DFCFE6FF26DF04D044
:1079D000DFCFE6FFE4EC6FF0E552299A0101E49B6A
:1079E000B1A72FD00701035105E002C700F003C77C
:1079F00001F0B7DD0701035106E01D50020B03E162
:107A00001C0E025D1BE103510AE01C0E025D07E142
:107A1000CC0E006E030703C701F0A3DD1D82010138
:107A2000B19715EC65F0230E155C03E1410E0DECEA
:107A3000C4F0249223AC03D0248201D003070701B1
:107A4000026B096A020EE15C02E2E16AE552E16E54
:107A50005BEFC3F0C3ECC5F00CE11B0E0101B55D9B
:107A600008E11850400B05E084848C808D8A8D8C51
:107A7000120006015051040B02E08D8C01D08D9C48
:107A80005051080B02E08D8A01D08D9A5051010BA4
:107A900002E08C8001D08C905051020B02E0848473
:107AA000120084941200000012000601D99D885033
:107AB000800B01E0D98DD99F8850400B01E0D98F10
:107AC000D9918850100B01E0D981D9938850200BAF
:107AD00001E0D983D9998850080B01E0D989D99B55
:107AE0008850040B01E0D98B12005FECC3F0FD0E4F
:107AF000DB50DBECC3F008E3FE0EDBCFE6FFFD0E50
:107B000055ECCBF00AE207D0FD0EDBCFE6FFFE0E10
:107B100055ECCBF002E2010E01D0000E5BEFC3F09A
:107B2000B0ECCFF02EB254D082B003D00701290EB2
:107B300076D082B203D007012C0E71D0DF6A060E18
:107B4000DF5C43E2DF50040DF35083095CECC9F0C5
:107B5000050EDF5C03E1DE52BB0EDD6E49ECD2F0B8
:107B600000C047F700501A082EE2F00E005C2BE22E
:107B7000FE0EDB5002E1010E56D049ECD2F000C0FF
:107B800048F700501A081FE2F00E005C1CE249ECB6
:107B9000D2F000C049F700501A0815E2F00E005C60
:107BA00012E2080EE66E48C7E6FF47C7E6FF42EC62
:107BB000C7F009E0080EE66E49C7E6FF48C7E6FFD2
:107BC00042ECC7F002E1DF2ABAD7060EDF5C02E121
:107BD000000E29D0010E3CECCDF05DECCBF010E2B4
:107BE0000C0EE66E020EDB50370FBAECC5F0E66EF7
:107BF00048C7E6FF42ECC7F003E1020EDB2AEDD7EF
:107C00005DECCBF00FE247C74AF748C74BF749C7CF
:107C10004CF7020EDB50080DF350DF1007014D6FDB
:107C20004D5101D0800E496E030EE15C02E2E16A23
:107C3000E552E16E49505BEFC3F03DECC8F09CECBF
:107C4000CBF006E18FECC9F003E001011E0EA86F36
:107C500001012D0E176F1FA402D02B0E176F02010A
:107C6000405107E13F5105E13E5103E10101200E82
:107C7000176FFAECC3F040C23EF011ECC6F0010100
:107C8000186F300E3A24196F300E02013F250101A2
:107C90001A6F0701BEAB05D0300E02013E2501016F
:107CA0001B6F0101198F120026ECCFF09BECC4F082
:107CB000EFCFDFFF01019F6BA06BA16BA26BA36BEA
:107CC0001DAE03D0050EA16F3BD05DECCAF0400B9A
:107CD00003E12750040B1DE051ECCEF051EC0DF008
:107CE000E55200C0A1F10050630825E20101A16B3B
:107CF000A02B7D0E005C02E1190EA16F0EECD3F0FB
:107D0000FA0E491818E14A5016E1A02B320EA16F65
:107D100012D05DECCAF0200B02E0A32B0CD05DEC7E
:107D2000CAF0100B07E0020EA26F57A704D0050E91
:107D3000A26F01D0A22B2AAE03D0020E9EECC3F09C
:107D4000E5525BEFC3F0AC0E006E0050D2ECC7F012
:107D500035C100F0D8ECCDF001011A5D05E1B5ECBC
:107D6000D0F002E1200E1B6F0201060E3D6F41EFC5
:107D700025F05FECC3F0B10E496EE10E4A6E010EC4
:107D80004B6E050E4F6E4FC043F0FE0EDBCF3EF044
:107D900017ECFEF03EC04CF04D6A66ECCFF0006E82
:107DA000C8ECD3F00101020EE7ECCCF0128F0C0E00
:107DB000DBECC3F003E20E0E0F6F0ED00E0E106F51
:107DC000FE0EDB50630802E2100E106F0F0EDBECAC
:107DD000C3F002E2090E116F140E146F120E156F2C
:107DE0005BEFC3F05FECC3F0D8ECD3F00101012BE3
:107DF000FE0EDB50006ED7ECD9F02B50100B07E1D4
:107E0000640EDBECC3F003E20101200E176F2BA818
:107E100007D001014D0E1B6F570E1C6F188F16D027
:107E2000FD0EDB5003E10101198F07D00A0EDBECD8
:107E3000C3F003E20101200E186F0101570E1B6F02
:107E400033B602D02A0E1C6F5FB31C8F5BEFC3F0FA
:107E50005FECC3F041EC25F0FE0EDB5003E0B1EC2B
:107E6000CDF003D00068A5EC26F0D2ECC4F01AE007
:107E7000020E0101395D0FE1A50E485D0CE1D8EC61
:107E8000D3F0150EE66EC10EE66E010EE66E7EECC8
:107E9000DAF0E5520BD0010EE66E6FEC05F0A60F9E
:107EA000E66E03D0E66A48C1E6FF9CDFE552E55284
:107EB0002BA807D0006899EC26F048C1E6FF59DFEF
:107EC000E5525BEFC3F014ECCEF041EC25F0B40EBC
:107ED00017ECCBF034C1DFFFB0ECCBF003E0A8EC43
:107EE000CBF001E1DF6ADF50006ED7ECD9F0640E11
:107EF000DF5C03E20101200E1A6F0A0EDF5C03E271
:107F00000101200E1B6FE5525BEFC3F03DECC8F0A2
:107F10009CECCBF008E18FECC9F005E00101D051F9
:107F200002E0A891A84349C100F0D7ECD9F0640E53
:107F30000101495D02E2200E166F0A0E495D02E260
:107F4000200E176F8F0E006EE1EF25F0270E0DEC5F
:107F5000C4F00101500EA86F3B51200B06E18FECDD
:107F6000C9F003E001011E0EA86F1200F20E006EB0
:107F700012ECC4F002E0F50E006E8EEC26F032C179
:107F800000F012ECC4F002E053C100F00101040E55
:107F9000016FD7ECD9F001011B8F12005FECC3F029
:107FA00012ECC4F003E08AECC4F003E028C100F056
:107FB00008D0CCECCBF003E058C100F002D054C1A3
:107FC00000F05BEFC3F0CD0E17ECCBF0010EE66EC8
:107FD000E5DFE552D8ECCDF001011A5D05E1B5EC25
:107FE000D0F002E1200E1B6F12005FECC3F093ECA7
:107FF000D2F0400B03E12750040B05E001018E5144
:10800000020B01E191D093ECD2F0200B03E027505A
:10801000040B02E001019E6B93ECD2F0400B03E1F4
:108020002750040B5AE00101A0510EE0A1510CE1D0
:10803000FE0EDB5005E19C5102E19D5101E0A06B79
:108040009C6B9CC19DF170D05A0EA15D16E1FAECBB
:10805000C3F09CC13EF0A0ECCBF0006EFE0EDB50F6
:1080600007E1005003E101019D5102E00101A16B14
:1080700001019D6B00509C5F57D09C5102E19D51C6
:1080800053E09D51496E4A6A9C510A0D6DECC6F051
:10809000A1510A0D14ECCDF025ECC5F0D4C142F08D
:1080A000D5C143F0BDECFDF039C0D2F13AC0D3F1F7
:1080B0000101D251D31138E0D2510E5ED3510F5A83
:1080C000FE0EDB5001E1A16BFBECCAF0E6ECCEF05A
:1080D0003DC09CF139C09DF127D093ECD2F0100B3C
:1080E00023E093ECD2F0200B1FE1020E016E0101A0
:1080F00057A702D0050E016E01C0A2F101C043F0E6
:108100009DC13EF0A0ECCBF0006EFE0EDB5004E112
:10811000005002E000C0A2F1FE0EDB5005E000506E
:1081200003E000500101A25F5BEFC3F05FECC3F01E
:1081300051ECCEF0E66A59DFE552E55207ECC9F0A2
:108140009FEC31F001019A510DE11F0E9B5D0AE297
:108150009AC29AF19BC29BF19CC29CF19DC29DF177
:108160009EC29EF102016F2B5BEFC3F00101DA9317
:10817000CDB3DA83DA95CDB5DA851200010138A3E3
:1081800006D0CD9312B6CD83CD9512B4CD85EEDF5A
:1081900004B053DDCBECA0F064EF2EF00A0E020128
:1081A0003F03F3504B6E4C6A4051640D2CECCCF005
:1081B0003E5101014924D66F000E4A20D76F0A0EA6
:1081C000006E0701BEAB02D0010E08D0BEA907D0D9
:1081D000140E006E010157A702D0320E006E1FB4BC
:1081E00003D00101DDECCAF028AA1AD00EECD3F0BE
:1081F000100ED8804956270E4A560101D7514A1809
:10820000E8AE02D04A3404D04950D65D4A50D7591E
:108210001FE20050FFECCEF0D6274A50D72318D0EB
:1082200000504A6AF00F496ED80E4A2201014A50A6
:10823000D719E8AE02D0D73504D0D651495CD75112
:108240004A5806E20050FFECCEF0D65F4A50D75BAA
:108250001F84800ED71503E01F94DDECCAF00EECEE
:10826000D3F0D6C13DF0D7C13EF015ECCCF04AAE0C
:1082700004D0396C3A1E000E3A2239500101D65F03
:108280003A50D75BADECCDF0B0ECD1F03DC040F250
:1082900039500101D66FD76BFBECCAF0B0ECD1F0CE
:1082A0003DC03FF239C03EF256EF41F02F8E0480C0
:1082B000BEEF40F00A01DA9F5FEC0CF0016A0101A9
:1082C000D0510EE10701BEBF11D00A0E016E11ECB4
:1082D000C7F03E50006E0150005C18E2005015D00F
:1082E000030ED05D11E10701BEAF02D0160E0DD016
:1082F000030E0A5C02E1140E08D00A5002E11E0EC1
:1083000004D059ECD0F001D0160E016E01501608C1
:1083100002E2160E016E1200000CFEDF000903E0FF
:108320000101500E486F12005FECC3F000AE14D094
:10833000FF0E0002F3CF6FF26F0EE96E020EEA6ECF
:10834000EFCF3EF0FE0EDBCF43F017ECFEF03EC069
:10835000EFFF02016F6D09D000C03EF0FE0EDBCFD3
:1083600043F017ECFEF03EC06FF25BEFC3F014EC8D
:10837000CEF02F50200B56E12350800B53E13050AC
:10838000400B50E12450010B4DE11FA618D062ECC8
:10839000CBF00101269902016F5102E0010126890B
:1083A0000101269B02016FAF02D00101268B010162
:1083B00026A938D01DAC36D016EC0CF033D024C131
:1083C00000F001012699005001E02689269B00BE9D
:1083D000268B26BB006CC3ECC5F016E12E50100BAB
:1083E0000DE01E50040B0AE11B50080B07E1005082
:1083F00002E0EDEC08F0006A0101246BB8ECCBF070
:1084000006E0440EB55D03E000380F0B006E00502F
:1084100007E00101268D269F26BB268F246B02D004
:1084200001012699010126A902D08CEC04F001017A
:108430002651100B06E02B50200B40E01D50400B46
:108440003DE11F50080B16E03B51200B13E13BB3FD
:1084500032D06AECCBF00101279902016F5102E0A2
:10846000010127890101279B02016FAF27D001017C
:10847000278B24D025C100F02799005001E02789DF
:10848000279B00BE278B279927BB006C32A005D005
:108490000038E8461F0B006E04D0D8900032D89008
:1084A000003200500AE00701460EA66F0101278D39
:1084B000279F27BB278F256B01D027992B50200B97
:1084C00003E01D50400B10E001012651100B02E0AB
:1084D000ABEF46F02751100B02E0ABEF46F0205017
:1084E000200B02E1ABEF46F0D7CADCFAD6CADDFAC0
:1084F0000601D551D595010B01E0D585D551D5970C
:10850000020B01E0D587D5918650040B01E0D5819F
:10851000D5938650020B01E0D5830F0ED51564EC80
:10852000C5F000A019D08CEC04F006015051040BEA
:108530000CE03250010B09E13050040B06E100AEB3
:1085400002D0DA0709D0DA2B07D000AE03D0010140
:10855000250702D00101252BDAC600F00601D599C6
:10856000005001E0D589D59B00BED58BD5A92ED072
:10857000D5BB006C00900042005028E0DA6B50A59B
:1085800025D001013751010B06E01250080B03E121
:108590001250040B0FE0288A0601D5BB289AFEDD95
:1085A0001EAC03D00201098702D002010681050139
:1085B000478D0CD0AAC224F10601D5AB04D0AAC2C3
:1085C00024F10101246D0101268927840601D65179
:1085D000D695010B01E0D685D651D697020B01E066
:1085E000D687D951D691020B01E0D681D951D693C5
:1085F000010B01E0D6830F0ED61564ECC5F000A088
:1086000009D063ECCAF000AE03D00601DB0702D04C
:108610000601DB2BDBC600F0D699005001E0D689BD
:10862000D69B00BED68BD6A9CBD0D6BB006C30BCB7
:1086300002D000900042005001E1C2D0DB6B010E7D
:108640000D6ED6BB0D68EDECC4F001E1B0D0D0ECFE
:10865000CDF02EECC4F003E1D1EC0BF0A8D031BC8E
:10866000A6D030AC0ED0D00EE66E0F0EE66E840EA5
:10867000E66E070E98ECC3F0F5EC04F0C3EC4FF097
:1086800096D0D0510BE0030ED05D08E08D51100B59
:108690003EE0020ED05D02E0D00539E114BC1CD0F2
:1086A0003484E4EC0FF0EAECCEF007E24950140811
:1086B000000E4A5402E2E4EC0FF0EAECCEF009E2DC
:1086C00049503D08000E4A5404E2E4EC0FF0E4EC9B
:1086D0000FF0EDEC0FF06BD0348403ECCBF008E03E
:1086E000C80EE66E280EE66EB80EE66E030E0AD0D1
:1086F000E1DD190E0124E66EB4ECCBF0E66ED70E88
:10870000E66E0A0E98ECC3F00A01030E49D014BCC1
:1087100025D03484CFDD0D040BE14DECCCF008E224
:10872000190E0124D75D04E2020ED65FD72B11D0BB
:10873000800E0D140EE0D4EC0FF0FF0F0A01D65D91
:1087400008E2B4ECCBF0D880D75503E2020ED6276E
:10875000D7070A01010ED46F338825D03484AADDEF
:10876000800E0D140CE04DECCCF009E2B4ECCBF033
:10877000D880D75504E2020ED65FD7070FD00D047C
:108780000DE1D4EC0FF0FF0F0A01D65D07E2190EE0
:108790000124D75D03E2020ED627D72B0A01020E71
:1087A000D46F3388010EE66E5AEC1BF0E5521EAC16
:1087B00003D00201098902D00201068B0501478519
:1087C0000601D751D795010B01E0D785D751D7972F
:1087D000020B01E0D787D951D791200B01E0D78157
:1087E000D951D793100B01E0D7830F0ED71564EC46
:1087F000C5F000A009D063ECCAF000AE03D00601BA
:10880000DD0702D00601DD2BDDC600F0D799005050
:1088100001E0D789D79B00BED78BD7A9C5D1D7BBDD
:10882000006C00900042005001E1BED1DD6B010EF2
:108830000D6ED7BB0D681950100B04E12050800B52
:1088400001E1E0D001018DB592D133B631D020BE27
:1088500004D0740E006E99EC26F0FF0E0D5C0CE156
:108860000201050ED8800055000E01551EE2060ECD
:10887000005F000E015B19D071C201F02B50100B8C
:1088800007E102017151780803E25A0E015C016EA2
:1088900001500B5C0AE20201880E005D130E0159C3
:1088A00004E2060E0027000E0123DFEC0BF078D166
:1088B00002011D6B780E016E026ADCECCDF002E065
:1088C000C80E016E2BA804D0960E016E0A0E026E21
:1088D0000150E66E0250E66E480EE66E010E98EC10
:1088E000C3F0D2ECC4F00CE1010148510A0808E2DF
:1088F000010E481505E00D0402E1482B01D04807A0
:108900002A840901ED6BEE6BE9EC04F090EC23F0A6
:1089100059ECCDF0E5520201320E046F48C15BF212
:108920001AECCBF002E248C18CF1E383E395E397C4
:1089300048C102F0D2ECC4F004E00101E3935A0E06
:10894000025E0250E66ED8ECCBF0DCECCDF015E028
:108950002B50100B12E10D0404E1650E0101485D7E
:1089600007E0800E0D1409E0640E0101485D05E189
:10897000318EEDECC4F001E01C94F6ECC6F0315001
:10898000800B11E12050800B0EE1EDECC4F00BE107
:1089900000500BE0050E005C08E0030E005C03E1F4
:1089A000020E0A5C02E00D5001D0020EE2ECCAF0A9
:1089B00031AE25D0319E049819A006D0048839EC38
:1089C0000BF0050E9EECC3F00101395111E0D2EC21
:1089D000C4F006E00F0EE66EC10EE66E010E02D088
:1089E00069ECCAF0F2ECCFF003E1FA0E9EECC3F0B2
:1089F00004A802D034EC0BF00D50E2ECCAF00201F6
:108A0000078BCED00101E2AF28D08DB5B0D034C1F4
:108A1000A8F21FEC19F01E0EE66E340EE66E010E83
:108A200093ECC3F063EC3FF05DECCDF034C1E6FFB6
:108A3000D8ECCBF0A0EC1DF00201A85103E001013D
:108A4000345106E00201A85105E10101345102E070
:108A5000E5EC17F002010885A2D02CA426D0E3850E
:108A6000E393E39712ECC4F00EE1C80EE66E320E0B
:108A7000E66E010E93ECC3F032C1E6FFD8ECCBF00A
:108A80001CEC64F00FD0C80EE66E010EE66E530EBD
:108A9000E66E010E98ECC3F053C1E6FFD8ECCBF0C4
:108AA0000AEC19F0B6EC3FF07BD024A036D0D051C0
:108AB00012E1460EE66E280EE66E290EE66E010EF7
:108AC00098ECC3F001012951E8240301B86F010EAD
:108AD000C7ECC6F016D0F2ECC6F007E0E66A2E0E40
:108AE000E66E010E93ECC3F00ED02EECC4F00BE159
:108AF000330EE66E010EE66E870EE66E020E98EC01
:108B0000C3F0F5EC04F017EC4FF0B5ECC5F0E5EC74
:108B100017F005014785478F43D012ECC4F006E0FB
:108B20008AECC4F003E12750020B1CE0320E006E09
:108B30000050E66E080EE66E490EE66E010E98ECE9
:108B4000C3F086EC3FF00101E393E395E38749C16D
:108B5000E6FFD8ECCBF049C113F5B9EC64F00201A3
:108B600006871ED0F6ECC6F001018DA503D0E6EC19
:108B700008F016D01FEC19F0500EE66E350EE66EBA
:108B8000010E93ECC3F08BEC15F0A3EC3EF05DEC22
:108B9000CDF035C1E6FFD8ECCBF0020108832A8482
:108BA0002D8E02011E0E206F0601D851D895010BA3
:108BB00001E0D885D851D897020B01E0D887D95168
:108BC000D891800B01E0D881D951D893400B01E0B6
:108BD000D8830F0ED81564ECC5F000A009D063EC63
:108BE000CAF000AE03D00601DC0702D00601DC2B80
:108BF000DCC600F0D899005001E0D889D89B00BEAF
:108C0000D88BD8A9A8D0D8BB006C009000420050E7
:108C100001E1A1D0DC6B010E0D6ED8BB0D682CA656
:108C200031D012ECC4F003E08AECC4F00AE0280E64
:108C3000E66E280EE66E010E93ECC3F005ECC6F06E
:108C40001ED0B0ECCBF00BE11E0EE66E580EE66EB9
:108C5000010EE66E2EEC7AF0E552E5520DD01E0EB6
:108C6000E66E540EE66E010E93ECC3F05DECCDF0B3
:108C700054C1E6FF3BEC0AF0E55229EC19F0E3ECB5
:108C80003FF065D023AE23D021B661D0016A010147
:108C9000D05102E0010E016E3CECCFF00AE17FEC16
:108CA000CFF004E6E20E495C000E4A5802E2190ECB
:108CB0000026FF0E0D5C05E10050180802E2190EB7
:108CC000005E0150F5ECC3F000C0EFFF0BD02FAAFF
:108CD0000DD021B63CD00E0EE66E930EE66E020E5F
:108CE00093ECC3F0F5EC04F0238A31D021B00ED020
:108CF00021B62DD03C0EE66E660EE66E010E93ECAC
:108D0000C3F0D1EC52F01BEC05F021D021B61FD0FE
:108D10002EECC4F00CE1280EE66E680EE66E010E35
:108D200093ECC3F043EC0CF059EC05F010D0800E3E
:108D30000D1404E03C0E675D01E2672B0D0403E1B6
:108D4000675101E06707EBEC52F035EC05F02D8E32
:108D500002011E0E206F1DAC66D00701BE8374ECAD
:108D600009F001013B91129C3B51010B01E0128C77
:108D7000E66AC0EC2BF0E552006E00500F0802E2EC
:108D80000F0E006E100E0002F3CF0EF22BEC27F048
:108D90001D9A050E0701A1250201D8800E5501E29A
:108DA0001D8A2A50800B13E10D5111E0050E0701B9
:108DB000A15D02010E5D03E2D5EC08F01D881D5097
:108DC000100B31E01D50200B2EE0020109D02A507B
:108DD000800B0AE11D50800B07E11D50200B04E0C1
:108DE000FA0E0D6F1D981FD02ABE02D0D2EC08F0EB
:108DF0002BBA17D01E0EE66E050E74ECC9F0E66EA7
:108E0000BAECC6F00AE019C5C0F11AC5C1F11BC51C
:108E1000C2F11CC5C3F11DC5C4F1AAC224F10101F0
:108E2000269B010126891D50800B0DE10101265171
:108E3000100B01E17ED01F50080B01E17AD02050C9
:108E4000200B01E176D002011E0E206F1DAC02D076
:108E5000140E206F2BAA2FD01DBC16D00101445137
:108E6000630801E2446B800E241506E0FB0E245DCE
:108E700003E2246B000E12D0800E241559E1245118
:108E8000030856E2246B09D00101246B2AAE09D0F5
:108E9000050116514DE1320E166F010E54ECCCF067
:108EA00047D0A951030844E3010E54ECCCF0010172
:108EB000140EA96F3DD01E50400B03E00951010B69
:108EC00037E11EAC02D0098101D00683050147813C
:108ED0002B8C2C8A6AECC4F0D0C1E6FF54EC3EF037
:108EE000E55262ECCBF01D50800B06E001012451ED
:108EF00003E17BEC31F016D002016FAF0AD0BEC7A0
:108F0000E6FF96EC40F0E5520201AA510101242748
:108F100009D06F5107E0BEC7E6FF12ECC9F0AA51B5
:108F20000101245F02016F51DCE12D827CEC04F031
:108F30001D9E01012751100B4BE01F50080B48E00C
:108F40002050200B45E002011E0E206F1DAC02D008
:108F5000140E206F1EAC02D0098301D006830501D8
:108F600047832B8CD1C1DFFF2C9A33ECC6F0DFCFC7
:108F7000E6FF54EC3EF0E5526AECCBF002016FAF35
:108F80000DD0DF509BECC4F0EF50E66E96EC40F055
:108F9000E5520201AB51010125270CD06F510AE0C7
:108FA000DF509BECC4F0EF50E66E12ECC9F0AB5111
:108FB0000101255F02016F51DFE12D8249ECC6F00E
:108FC00024A606D00101010EA86F0701140E556FEB
:108FD0002BAC06D041ECCDF02B9C25822CAA238A09
:108FE0000101279926992794E5525BEFC3F03B0EC8
:108FF0007CECC4F00101320EA86F2F8833C119F246
:109000001200010137A70AD04D0E096E0F0EE66E51
:10901000100E0D03F350E7ECCAF010D0030E096EEA
:109020000F0EE66E140EE7ECCAF0D1ECC3F0030E9F
:10903000E66E230EE66E230EE66E0A0ED1ECC3F04A
:10904000096A12005FECC3F0030E096E140EE66E9F
:10905000000EE66E0A0E12ECD2F0040EE66E260E3C
:10906000E66E0A0EE66E260E03ECCFF0FE0EDB5027
:109070001EE0010137A70AD04D0E096E0F0EE7EC76
:10908000CAF0E66E100E0D03F3500ED00F0EE7EC93
:10909000CAF0E66E140E03ECCFF0030EE66E230E5C
:1090A000E66E0A0EE66E230EE66EC9ECC3F0096AA0
:1090B0005BEFC3F0030E096EAA0EE66E2A0EE66E93
:1090C0000A0EE66E300E82EFD3F0D3EFD2F0B3EC9F
:1090D000CEF003E10201D8511FE001014FECCDF0C9
:1090E00001E0098FCEECCEF0840ECEECC3F0060189
:1090F000EE6B21EC32F007010B9907ECF7F07FECF7
:1091000020F00701149F23ECCEF00701158128EC15
:10911000CEF0A5EC16F02D860201D96BD9C2D8F29B
:109120001200010121A148EF4DF0219102010F072A
:109130000F5101E01AD1640E0F6F2EECC4F016E14E
:109140002050400B13E1080EE3ECC4F0046E04ACB5
:109150000DD00101E1BF02D0E18F02D0E1BFE19F5C
:10916000E66A1DEC39F0E55202EC32F002013D51A5
:109170000CE03D51010803E3EDECC4F006E0020110
:109180003D073D5102E141EC25F03196150E0101FC
:10919000555D0BE002011651171103E01607000E92
:1091A000175B1651171101E12F8C0201145101E0D8
:1091B000140701018B5104E08B078B5101E13196BB
:1091C000020120510CE01F50080B09E0200720513C
:1091D00006E11DAC02D01D8E02D02DBE2D9E300E9C
:1091E0000401F75D06E10201066B076B086B096B72
:1091F00005D0340EF75D02E255ECA1F002011951E1
:109200001BE00501105118E12750400B15E10FEC50
:10921000CBF012E1190719510FE10C50006E5551B6
:1092200006E07F0E5515006E189A55BF188A010E7C
:10923000E66E005035ECCBF00201580758510BE1B7
:109240000101515102010B5D06E2410E7CECC4F0BC
:109250000101A869258EEDECC4F008E001018351FD
:1092600005E0765103E1A3ECDBF002D06FECDCF01B
:10927000FFECCAF008E0C3ECC5F005E1E0ECCDF08E
:1092800002E106011D79C8ECCBF011E01B50100B78
:109290000EE12150020B09E0050ED05D06E0040E40
:1092A000D05D03E01E50200B02E1060104790101AC
:1092B0003851100B06E11350020B05E01950200B3A
:1092C00002E106010D752850400B01E0010E020F6E
:1092D000016E2850400B01E0010E050F026E03687D
:1092E0001DAC08D0DBECD0F0EF7EDBECD0F0EF5023
:1092F000800B036E010183512BE014ECDCF00009BC
:1093000003E12E50200B24E02E9A9EEC16F0016A09
:10931000030E015C12E2026A040E025C08E2020E15
:10932000C7ECC6F0320E9EECC3F0022AF5D7E66811
:109330008CEC21F0E552012AEBD7A5EC16F00101E7
:109340005F99258205EC79F0FEECDBF0A3ECDBF015
:1093500002012D5101E02D077A5104E02250100B3B
:1093600001E17A07325101E03207D35109E0D30716
:10937000D35106E1D45102E1010ED46FCAECC1F021
:109380001EAC09D00201D107D15105E155ECA1F085
:109390000201030ED16F0FECCBF040E02050400BE8
:1093A0003DE01950400B3AE09AECC9F003E1195046
:1093B000200B34E002013707000E385B1950200BF8
:1093C0000AE0D2ECC9F009E19CECC6F004E101012D
:1093D000E051100B02E1000E01D0010E0490E8B044
:1093E00004800FECCBF003E00450010B17E0376B67
:1093F000386B0101E09904A006D00201196B19C273
:1094000055F215EC65F003EC0BF00101B1A705D0A6
:10941000249223BC2482C5ECC9F0209402013C5163
:1094200001E03C07335101E03307315101E03107DE
:1094300030510AE03007305107E177ECC7F001E125
:109440004A5002E04AEC0DF00201185109E01807F9
:10945000185106E130ECC8F00201D05101E111943D
:10946000100710513FE1280E106F1AAC0FD072ECAC
:1094700038F0D0C100F0A6EC38F00601017901A95E
:1094800031D0D1C100F0A6EC38F02CD01BA803D00D
:109490000601047927D01CA206D00101E2B522D032
:1094A000060114711FD01950200B06E0010138513C
:1094B000100B02E106010D752450020B03E1A4EC30
:1094C000CBF010E0020130510DE177ECC7F001E183
:1094D0004A5008E02C50800B05E12C50400B02E173
:1094E0000601017102012B5101E02B070701A65172
:1094F00005E0A607A65102E1B2ECCAF002012A512A
:1095000016E02A072A5113E112ECC4F003E1CEEC75
:10951000DAF00DD00701A351A41109E0A35101E035
:10952000A307A45101E0A4070201020E2A6F020161
:1095300029510CE02907295109E1178E1790178846
:10954000080E156E2CAC02D0290E156E0101AA5121
:1095500069E0AA07AA5166E10EECCAF0006E0201AA
:10956000A95107E0830E096EA9C201F0F4EC3AF0AC
:10957000096AFF0E0201845D28E084C24FF0506A40
:10958000516AE90E496EDC0E4A6E010E4B6EB5C192
:109590004CF04D6A4E6A00ECCEF00900F5504F24B5
:1095A000F36E0900F5505020F46E0900F55051207B
:1095B000E0ECCEF00800F550006E0201842B005064
:1095C00004E184690101B6ECD1F0005013E001011F
:1095D000190EAA6F0050E66EEFEC6FF0E552020133
:1095E000A95102E0A92B1ED00101AE2B000EAF2322
:1095F000B02318D02850080B03E13050080B04E0CA
:1096000028960101E4970ED00201A95105E0A96B4B
:109610000101FA0EA86F05D00101D890A833D890A7
:10962000A833E4970201285104E02807285101E1FA
:10963000259E275107E02707275104E106014169CC
:1096400041C640F60101A6510DE0A607A6510AE168
:10965000090E155C07E1C3ECC5F004E10101FA0E47
:10966000A76F1A8A0101A75101E0A7070701555109
:1096700001E0550702012F5123E02F072F5120E170
:10968000000E0601E76EBE19E8AE02D0BE3503D06B
:10969000E750D880BE5502E2BE0701D0BE2B000EB7
:1096A000E76EBF19E8AE02D0BF3503D0E750D880CF
:1096B000BF5502E2BF0701D0BF2B0201050E2F6F7D
:1096C000155105E01507155102E1DCEC69F00201C6
:1096D000215124E0210727AA21D020BC1AD01A50FA
:1096E000800B17E0800E071414E02050010B11E1ED
:1096F000216B1A9E0A01DA8F5FEC0CF031EC75F0E9
:109700001EAC03D00201098902D00201068B0501BB
:1097100047850201215102E1238A25820D5107E08C
:109720001D50400B04E00D070D5101E11D8E050198
:10973000165101E016070201355105E03507355194
:1097400002E1BCEC0AF00201B05101E0B007D051D7
:109750000DE0D007D0510AE107010A8308ECF7F0C9
:10976000EBEC52F00201185101E111942C5101E08F
:109770002C070101A85101E1A3D0A807A85101E0DD
:109780009FD0B19DB19F2F98E0951C921B9830AC53
:1097900002D0E2EC4FF02FBA07DB23BE98DA24B0F8
:1097A0005CDB2582238A279820BA02D0DBEC26F0E6
:1097B000208A0C0E155C29E12150200B26E00101C6
:1097C000A65123E11568C3ECC5F002E11E8417D051
:1097D00001013B71129C3B51010B01E0128C14EC16
:1097E00099F0540E0DECC4F001013BA108D04B0ED2
:1097F000E66ECC0EE66E1CEC0AF0E55204D0550E77
:10980000E66EBBEC26F0E5521A861D50400B11E0C7
:109810002A50800B0EE12150200B0BE02A8E130EF4
:10982000D2ECC7F0460EE66E410E6FECCAF0D5ECF6
:1098300008F00101E4A909D0E499E4877A0EE66E04
:10984000D80EE66E010E5AECC6F02550040B38E037
:109850000B0E155C35E12150200B32E00101A651C1
:109860002FE120982594B19BB199E27DE2AD1AD009
:10987000E4A30AD0010EE66EC10EE66E010E8FEC77
:10988000C3F00101198F09D0890EE66ED80EE66E7D
:10989000010E5AECC6F00101E487E483500EE66E37
:1098A000C60E0CD0F90EE66EC00EE66E010E8FEC01
:1098B000C3F00101198F500EE66E4E0EE6ECC3F0B8
:1098C00002011D5101E01D07045101E004071E5172
:1098D00001E01E071F5101E01F07345101E034076A
:1098E0000101A95101E0A9070201235101E0230769
:1098F000395101E03907D85108E0D807D85105E1BE
:1099000067EC48F002010E0ED96FD95101E0D9077A
:109910003A511CE02150200B0AE1110EAFECCEF0C1
:109920003AC23EF0A0ECCBF002E10601067B020158
:109930003A072150200B05E02050400B02E07DEC5F
:1099400005F002013A5102E1ABEC04F0060143518B
:109950000AE04307435102E15A0E436F25860F0E7A
:10996000435D01E225960201225108E022072251BF
:1099700002E174EC69F002011E0E216F3B5110E010
:1099800001012651400B0CE102013B073B5108E16C
:1099900044C100F0188673EC96F00201010E246FAA
:1099A0000201245142E0240724513FE101013951D1
:1099B00003E00901010EEB6F0901ED6BD0ECCDF076
:1099C0000101E38FADECF7F00201186BD05101E11A
:1099D000119430ECC8F020A204D0209264EC2EF058
:1099E00015D065ECCDF0249CA5EC16F0640E9EEC31
:1099F000C3F0A3ECDBF0CEECC9F008E02050200B64
:109A000005E0010EE66EAAEC99F0E55218B002D01E
:109A1000BDECD1F01890020106891EAC02D0098776
:109A200009850501BF0E476F48810201365104E0E8
:109A30003607365101E12582255101E02507D25133
:109A400009E00501105106E10201D207D25102E1FD
:109A500048EC0AF002011B5106E01B071B5103E111
:109A6000630ECEECC3F002011C5106E01C071C5132
:109A700003E1B10ECEECC3F002011A5105E01A0762
:109A80001A0502E12AEC10F002012E5101E02E0726
:109A9000120006014F6B4FC64EF64FC64DF64FC62D
:109AA0004CF64FC64BF6120018ECCEF0DE52010E0B
:109AB000DD6EFE0EDB501AE196ECD1F0050EE66E7F
:109AC000200EDF24E66E4B0EE66E060ED1ECC3F0E0
:109AD000050E2AECD3F0B60EE66E010ED1ECC3F003
:109AE0000F0ED4ECD0F00050DF6E096A0101B651C0
:109AF000630805E3B6510EE11F0EB75D0BE2360EAB
:109B0000006E83EC26F0FE0EDB5001E1C2DF010E99
:109B1000DB6A22D0FE0EDB501FE12C50800B07E0E9
:109B2000DF500A0804E20701BE9B74EC09F0DFCFA6
:109B3000E6FFE6EC33F0E55201018A51100B0CE030
:109B40000A0E445D09E2C8ECD3F0DEECD0F0DFCFC2
:109B5000E6FFA0EC80F0E5520201295115E1640E08
:109B60000101445D0BE2FAECC3F044C13EF011EC9C
:109B7000C6F00101166F300E3A2405D04D0E166F57
:109B8000030E4415310F176F016A050E015C2FE2B9
:109B90007E0E496EDF0E4A6E010E4B6E0150EA6A70
:109BA0004B0FE96E060EEA22EFCF4CF04D6A66ECE1
:109BB000CFF0026E2D0E025C05E10101B25102E10F
:109BC000200E026E0201295110E1020E0124D5EC93
:109BD000C4F002C0EFFF015008E12B9A2A0E025C8C
:109BE00004E12C50800B01E02B8A012ACED7020120
:109BF000295102E10101188F010EDB50BCECCBF0C2
:109C000002E2E16AE552E16E49505BEFC3F028ECF5
:109C1000CDF0016E44516EECC5F0050EE66E4B0EB4
:109C2000E66E060EE66E200E012482EFD3F00201EE
:109C3000050EB86FF00EB96FFA0EBA6F140EBB6F47
:109C4000F00EBC6FFA0EBD6F1200016A0101D05117
:109C500002E0010E016E01509BECCEF0EF50006E61
:109C6000CEAD006A0150F5ECC3F0EF50E66E015046
:109C70009BECCEF0010EAFECD3F0E66E0050E66E3A
:109C8000250E8CECC5F001011496CE51400B01E07D
:109C900014861200026A0101D05102E0010E026E28
:109CA0000250F5ECC3F0EFCF49F0190E43ECC4F0CD
:109CB000BEECC7F002E1200E1B6F4E0E186F520E65
:109CC000196F25EF4EF0238E1F964AEF4EF0239E1C
:109CD00017EFCAF0020EE66EBD0EBEECC3F0010136
:109CE000CCBB0FD0BB0ECEECC3F0010EE66E200E47
:109CF000E66EE66A2F0EE66E68EC16F0CBECD2F05C
:109D00003AD0070E0201935D19E29351E824496E9F
:109D10004A6AFF0E00ECCDF04950E66E060ED88080
:109D20009355070DF3500A0FE66EBC0E85ECC3F099
:109D3000010EE66E200EE66EE66A16D0F30EDCEC3F
:109D4000CBF0BC0E85ECC3F0020193510A0802E28D
:109D5000030E01D0010EE66E0F0ED88093550C0D48
:109D6000F350E66E800EE66E2F0E8CECC5F0B90E49
:109D7000E66E29EC16F0E55201011494CC51200B4B
:109D800001E01484120002019329BEECC7F002E145
:109D9000200E1B6F4E0E186F420E196F6AEF4EF0B9
:109DA0002F8A1F96C3EF4EF02F9A17EFCAF0D8EC08
:109DB000D3F02EECC4F017E1020E016F02018729E7
:109DC000CFECCCF09DECD0F0030EE66E020EE66E0A
:109DD00035EC09F0E552E55201011C8F500E166F6B
:109DE0004C0E176F1200030ED05D10E1F2ECC6F0BE
:109DF00006E0F10EE66EC00EE66E010E05D0E90E2D
:109E0000E66EC00EE66E010E0AEFD0F0016B29C1BE
:109E100000F0D8ECCDF00101165D02E1200E166FC6
:109E2000300E196F480E1B6F5A0E1C6F1200245013
:109E3000010B09E12EECC4F006E09EEC16F0030ED7
:109E4000006E63EC75F024802EECC4F003E0006833
:109E50008EEC26F01F96D7EF4EF02EECC4F005E105
:109E60000BEC09F031EC1FF004D0BCEC0AF0A5ECCF
:109E700016F024901A940101A86BB19F239809EC65
:109E80000DF034EF0EF0D8ECD3F03A0E496ED20E4E
:109E90004A6E010E4B6E0A5041ECD3F017C1E6FF3B
:109EA00016C1E6FF04EC0AF0E552E552010136ADB9
:109EB00002D0CAECD7F012003280B1ECCDF01F9680
:109EC000E2DF0DEF39F0329009EC0DF001DA2F9856
:109ED000120035ECCEF0140D29ECC4F0C0ECCDF03E
:109EE00005E0B0ECC5F0230E85ECC3F043EC15F0B3
:109EF000140E9EECC3F05BEFC3F05FECC3F0B6C290
:109F000000F0FE0EDB5001E1006AB7C2E6FF005030
:109F1000E66E240E85ECC3F05BEFC3F007018B51B6
:109F2000845D15E11450100B01E0010E496E3350B1
:109F3000010B495C0CE11450200B01E0010E4A6E4C
:109F40003350020B01E0010E4A5C01E1120084C7AC
:109F50008BF7339014B83380339214BA338214A839
:109F60000BD014AA03D084C7E6FF07D0E66AB1DF9E
:109F7000E552010EE66E04D0E66AABDFE552E66A12
:109F8000BCDFE552120007018451140D9DECD0F0A6
:109F900019C116F11AC117F11BC118F11CC119F131
:109FA0000101200E1A6F480E1B6F5A0E1C6F300EE7
:109FB000165D02E1200E166F8EEF4FF0308C1F966B
:109FC000C3EF4FF0309C2F980101A86B2398B19FED
:109FD00009EF0DF00101A85103E02450080B03E044
:109FE000B151200B01E02F8800508FECC6F0010129
:109FF000A85106E02F50100B03E1FA0EA86F24863B
:10A000001200010E0701D89056375737E806FBE1DA
:10A0100021AC02D0070156810D0E0701585D01E207
:10A02000582B1200219C8450020B01E0218C070167
:10A030004E5111E121AC78D04E2B010E566F576B6B
:10A04000586F3098596F5151FE0BE8425125506FAF
:10A05000010121931200010121A366D02193070180
:10A060004E0562E121BC52D030A84DD00C0E585D97
:10A0700047E2D89057335633006A5F0E005C1BE20C
:10A08000540E4B6ED10E4C6E010E4D6E00504E6E46
:10A0900032ECC5F0565149180CE157514A1809E104
:10A0A000200E0026610E005C02E3200E005E92DFAF
:10A0B00002D0002AE2D75F0E005C22E107011F0EEA
:10A0C000561901E157510AE01D0E561901E1575189
:10A0D00005E0EF0E561905E1575103E1200E006E21
:10A0E00079DFFF0E0701561902E1020E571906E04B
:10A0F000B50E561905E1030E571902E1ACEC6FF0ED
:10A1000007014E6B1200308801EF50F07ADF30A863
:10A1100004D00701010E596F06D00701592B595180
:10A120000C0801E24E6B3098120007AE06D0845046
:10A13000020B02E0219C01D0218C07014E5110E15D
:10A1400021BC75D00101219307014F6B07AE6FD081
:10A15000020E4E275151FE0BE8425125506F12005E
:10A160004E050BE14E2B51C750F70101219321AC55
:10A170005ED00701080E4E6F1200010121A357D0D7
:10A180002193070E07014E5D46E14E6B21AC40D096
:10A190000101A85103E02450080B03E0B151200B4A
:10A1A00001E02F88060E496EDF0E4A6E010E4B6EDF
:10A1B00007014F5152251FECCEF0006E810E005C5E
:10A1C00002E1526B1BD0800E005C03E1200E526F47
:10A1D00015D00D0E005C03E00A0E005C02E1200EBB
:10A1E0000BD00B0E005C02E12A0E06D00A0E005CBA
:10A1F00005E0005003E000508FECC6F00101A851CB
:10A2000009E02F50100B06E1FA0EA86F2486120009
:10A21000080E4E6F1200080E4E5D04E121AC07D00F
:10A220004E6B12004F914F4321BC4F894E2B1200B1
:10A23000D8ECD3F07DECC5F013E1C4ECCDF006E032
:10A24000E20E496EC00E4A6E010E05D03F0E496EF9
:10A25000D00E4A6E010E6EECD0F0ECECC3F018D0CC
:10A26000EAC600F00050020802E2020E006E120E72
:10A27000496ED20E4A6E010E4B6E005041ECD3F087
:10A280000601EA51020804E2EA05300F01011C6FE1
:10A2900089EC1FF0BCEC0FF0006E00500A01D65D97
:10A2A00004E200C0D6FAB5ECC5F012000101D051AD
:10A2B00005E13084B1ECCDF01F9603D00068A5EC29
:10A2C00026F018EF51F0309409EC0DF068EF51F0E2
:10A2D000040EE66EEA0EE66E060EE66EA00E03ECC7
:10A2E000CFF0140E016E3CC100F0B1EF3AF014EC67
:10A2F000CEF0E0C649F0E1C64AF0D89049364A3679
:10A30000060169ECCDF00CE3DEC64BF0DFC64CF085
:10A31000D8904B364C36E0514B5CE1514C5820E222
:10A32000DE51E0250E6EDF51E1210F6E0BECCBF01C
:10A33000E2C649F0E3C64AF0030E53ECC9F0FDE172
:10A3400049500601E25F4A50E35B2AECCFF0030E6E
:10A3500053ECC9F0FDE149500601E2274A50E323DE
:10A36000DEC6E0F6DFC6E1F675ECCAF049364A36DD
:10A37000D89049364A3669ECCDF00BE375ECCAF05B
:10A380004A32493297ECD2F04950DE5D4A50DF59EB
:10A3900002E2DF6A09D0E251DE5DE351DF5902E2F9
:10A3A000010E01D0020EDF6E75ECCAF049364A3656
:10A3B0004950E225E46F4A50E321E56FDF50E55252
:10A3C0005BEFC3F01DBC1200219C8450020B01E026
:10A3D000218C21AC03D002016C2B02D002016D2B29
:10A3E0001F9E0601E65109E121AC4BD0010EE66F3C
:10A3F000DE6BDF6BE76BE86B44D0E60515E121BC53
:10A4000040D0020EE66F73DF006E00500BE0070EC7
:10A410000601E85D07E2E82BE791E74300500108F9
:10A4200001E2E78F06011FD0020EE65D2AE121ACB2
:10A430001DD0E2C64BF0E3C64CF0030E0F0B05E057
:10A44000D8904C324B32E806FBE106014B50E25DFE
:10A45000496E4C50E3594A6E4950DE5D4A50DF590F
:10A460000EE2010EE66FDE6BDF6B0BD0E451E425EC
:10A47000496EE551E5214A6E69ECCDF002E2030E2A
:10A48000E66F030EE65D43E1E791E743E78F070ED2
:10A49000D880E855016E01500106000903E0E791FC
:10A4A000E743F9D7780EE75D30E20101A85103E0F8
:10A4B0002450080B03E0B151200B01E02F88E7C6C0
:10A4C000E6FF3CEC04F0E552006E200E005C03E376
:10A4D00000506E0802E22A0E0BD0298A00508FEC41
:10A4E000C6F00601DE51E45DDF51E55903E2200EBE
:10A4F0008FECC6F0299A0101A85107E02F50100BEC
:10A5000004E12486FA0EA86F30860601E66B1F8EE2
:10A5100012000101E183D05102E154DF07D01F9EF8
:10A52000DAECC9F002E07EDD01D0FFDD0101E1934C
:10A530001200800E071420E02A50020B1DE120506B
:10A54000200B1AE00201A95117E10101D05104E1E9
:10A550000601EA51010806E37DECC5F00DE1C4EC0B
:10A56000CDF00AE02A0E0101B11506E10C0E155CD2
:10A5700010E12150200B0DE0800E071409E18AEC58
:10A58000C4F006E00601EC5103E002012D5101E0A8
:10A59000000C010C0201395103E1120E0DECC4F064
:10A5A000120014ECCEF066C1DFFF21A205D001013C
:10A5B00066515CECD1F0DF5E1EBCDF6ADFCFE6FFE8
:10A5C000720EBEECC3F030800201078334B0E2DFCC
:10A5D000E5525BEFC3F014ECCEF067C1DFFF2EEC69
:10A5E000C4F002E1DF6A05D007010AB302D00F0E02
:10A5F000DF5EDFCFE6FF710EBEECC3F0020107871E
:10A60000E5525BEFC3F018ECCEF0D00EDE6E070E15
:10A61000DD6ECCECCDF004E28C0EDE6E0A0EDD6E4B
:10A62000E2A510D0080EDE6E070EDD6E38EC20F0CD
:10A63000010804E038EC20F0020818E16C0EDE6E30
:10A64000070E13D0090E2B5D0DE25F51020B0AE0DD
:10A650002250100B07E13450800B04E102010B5132
:10A660007D0804E2B80EDE6E0B0EDD6EAEECC4F0BB
:10A6700002E3000E01D0010EBCECCBF002E2E16A75
:10A68000E552E16E49505BEFC3F018ECCEF030ECD0
:10A6900011F091EC48F08FECC9F002E03ADF02D003
:10A6A0001FBE1F9E2450200B06E00201245103E12F
:10A6B00037ECF7F0249A02012B5102E055EC3DF003
:10A6C0000101B35111E1E66AC0EC2BF0E552006ED6
:10A6D0001DAC2AEF5AF00701A151F00BE83AA15D39
:10A6E0000024A16F2AEF5AF0B3050DE13CEC71F0A4
:10A6F0002BEC27F05CEC18F01E92E8A02AEF5AF041
:10A700001E822AEF5AF0020EB35D04E1FEECD3F094
:10A710002AEF5AF0030EB35D07E12EB42AEF5AF088
:10A7200029ECD9F02AEF5AF0040EB35D01E0B4D061
:10A730000201255102E02AEF5AF01750100B06E1F2
:10A740001750010B03E11750200B02E0000E01D05F
:10A75000010E2290E8B0228021AA45D057ECCAF021
:10A76000166E22A036D00101A6512AE1090E155C11
:10A7700017E1C3ECC5F014E10101A7510BE1A00EF4
:10A78000176E8FEC09F000093CE0CEECC9F039E11E
:10A790001A8637D0165035E1A76B900E176E1FD072
:10A7A000165002E1010E01D0100E8009176E8FECD9
:10A7B00009F0000926E0CEECC9F023E11A8421D08B
:10A7C00016501FE1A76BA7C1A6F1810E176E219A43
:10A7D00006D0165016E12250010B13E1219A020116
:10A7E000020E256F0ED031B40CD0E66A90EC3DF02D
:10A7F000E552000906E031840201020E256F07AE22
:10A80000256B3150040B02E12AEF5AF00201255169
:10A8100002E02AEF5AF0319457ECCAF0166E165047
:10A8200002E12AEF5AF08CEC04F00201A96B01015D
:10A83000280EA66F150E165C05E12050400B02E0B5
:10A840001E0EA66F080E165C06E0290E165C03E0CD
:10A85000100E165C02E12D0EA66F0201020E256F8E
:10A86000218A176A1650156E8FEC09F000090BE06B
:10A8700001013651800B07E00201355104E1040E5D
:10A88000006E63EC75F028B602D00101AA6BB6EC3D
:10A890000CF02A842AEF5AF0050EB35D21E1EDECAD
:10A8A000C4F00FE01B50080B0CE1C9ECC7F009E243
:10A8B000C9ECC7F006E202011E0E186F30ECC8F0BA
:10A8C000118401012651100B02E02AEF5AF02751A2
:10A8D000100B02E02AEF5AF055EC3DF02AEF5AF047
:10A8E000060EB35D07E120AA2AEF5AF0D0EC07F07C
:10A8F0002AEF5AF0070EB35D02E12AEF5AF0080E74
:10A90000B35D01E075D32550800B0AE002012851A8
:10A9100007E1020EC7ECC6F002011E0E286F259E4D
:10A9200025AC04D0010EC7ECC6F0259C25AA03D0A7
:10A93000BCEC0AF0259A01013651800B1BE00201A4
:10A94000355118E11AA404D0040EC7ECC6F01A94CD
:10A950001AA604D0070EC7ECC6F01A961AA804D09F
:10A96000060EC7ECC6F01A981AAA04D0050EC7EC5A
:10A97000C6F01A9A0101B1BD92D0B1A952D020AE51
:10A980000ED0A95167E12BA805D00B50E66EB9ECAB
:10A990003EF003D0E66A67ECBDF0E5525BD024A040
:10A9A00003D017EC4FF056D02C50400B03E12C5045
:10A9B000800B30E026AD4ED0C6EC08F00101B2515C
:10A9C0001AE1630EE66E440EE66E010E74ECC6F0FC
:10A9D00044C10CF202013B6B7EECC9F0000917E0A8
:10A9E0002C50800B14E001018E51100B10E102017C
:10A9F000100E3B6F0CD0290EE66EB2054A6A4B0F63
:10AA0000496E060E1EECD0F06EECCDF0E552010161
:10AA1000A96B20D021B61ED059C200F083EC26F0DD
:10AA200019D0B1A305D025A215D02592228212D02B
:10AA3000B1A110D025A206D025922BC1E6FFE6ECED
:10AA400033F0E5520201215105E11A50400B02E1B9
:10AA50000DEC39F0D9EC14F0006EFF0820E0570E31
:10AA6000005C07E1C8ECD3F0220E006E83EC26F008
:10AA700016D01B0E005C03E1ECECC2F010D0FF0E10
:10AA8000015C0DE0C8ECD3F00101140E116F0D0E46
:10AA9000126F050E006F0150006EBAECD9F0010183
:10AAA000B1BF8ED2B1ABF6D02CA603D0E3EC3FF011
:10AAB00071D230AC03D0C3EC4FF06CD22FAA05D0CA
:10AAC00023AA68D2C3EC4EF006D023AE06D023AA48
:10AAD00061D24AEC4EF0239AA8D024A003D0D7EC40
:10AAE0004EF058D22CA403D0B6EC3FF053D2E2AFD4
:10AAF00003D063EC3FF04ED219A803D059ECCDF04F
:10AB0000B1D03050040B1BE0D05119E127AD0DD06E
:10AB1000010E0D6E27BF0D680A0EE66EEA0EE66E98
:10AB2000060E93ECC3F0B5ECC5F02350200B04E106
:10AB300001012751400B3FE018EC51F03CD032A00E
:10AB40003ED027AD16D0010E0D6E27BF0D680AC08E
:10AB500006F1030E6EECCEF074ECC6F006C10AF0FE
:10AB6000E8ECCFF00A501EECCFF068EC51F0050194
:10AB700047852350200B03E0CEECC9F004E001012F
:10AB80002751400B18E0B6EC0CF0C3ECD1F043ECCD
:10AB90004FF002010881050147871EAC02D0020177
:10ABA00009851F50020B05E0DAECC9F002E07BECEE
:10ABB000CAF08EEC39F00101279D239A37D02C5032
:10ABC000400B03E12C50800B33E023AA04D0239ADE
:10ABD0006EECCDF047D027ADDDD1279D010E0D6E77
:10ABE00027BF0D68006A050EE66E0050E66EB20ED5
:10ABF000E66E010E98ECC3F00601030E426F0101F0
:10AC0000B2510EE0B229496E010E495204E0E84605
:10AC1000FE0B4906FCE10601426F1E0E436F02D097
:10AC200007EC4EF06EECCDF0E5520101A96BB2D10C
:10AC300020AE1AD0A95101E0ADD1D2ECC4F001E0B0
:10AC4000A9D10B50016E2250100B03E13450800B40
:10AC500002E0CAEC67F0006A005097ECC7F0F2EC33
:10AC60003EF0E552E55296D121B694D15AC200F099
:10AC70008EEC26F0A30E02015A5D01E08BD112EC9E
:10AC8000C4F001E187D18AECC4F001E083D1010175
:10AC9000320E20D0B1B37ED1B1A71ED01950400BD7
:10ACA00004E01950040B01E075D1D8ECD3F00A0E82
:10ACB000006EE1EC25F00101040E016F03C700F006
:10ACC00019AC02D094EC04F0D7ECD9F019AC62D1F5
:10ACD0000101200E1A6F5ED13BAB46D1070E006E0C
:10ACE0000050D880765501E2766B27AD10D0279DB5
:10ACF000010E0D6E27BF0D680050E66E760EE66EF3
:10AD0000010E93ECC3F00601426B0101A96BA9513E
:10AD100001E040D12050200B01E13CD10201A951BA
:10AD200001E038D1070E0101765D40E1D8ECD3F0A7
:10AD300097EC16F001012B0E166F00010FAE0BD031
:10AD400001012D0E166FFF0ED8800E560F56010E04
:10AD50000E26000E0F22E70E57ECC9F002E272EC4D
:10AD6000CDF00E500F1003E10101200E166F2AECFA
:10AD7000CFF0640ED6ECCEF039C049F03AC04AF0BC
:10AD80004950006E0101012BD7ECD9F082EC04F0A0
:10AD9000300F0101176F300E175D02E1200E176FA3
:10ADA000198F640E1A6F420E1B6FD0D0060E765D9F
:10ADB0001EE1D8ECD3F094EC16F0FFECC5F00101E5
:10ADC000410E166F460E176F560E186F300E195D36
:10ADD00001E0E0D0200E196F300E1A5D01E0DAD0EC
:10ADE000B5ECD0F001E0D6D0200E1B6FD3D0040E0E
:10ADF000765D03E0050E765D6CE1D8ECD3F0049847
:10AE0000050E0101765D09E14F0E166F530E176FA7
:10AE1000430E186FC9ECD1F026D0500E166F410EBC
:10AE2000176F0488D2ECC4F006E00101580E186FC9
:10AE3000EAC900F01AD00101E2A50DD0320E186F58
:10AE4000E1A902D0340E186FFBECCAF0ABC73DF09D
:10AE5000ACC73EF008D0490E186FFBECCAF0A9C78A
:10AE60003DF0AAC73EF0F7ECD2F0049000AE02D05D
:10AE7000006C04800101030E016F64ECC8F004A0B3
:10AE800002D02D0E196F430E1C6F04B8188F050EDB
:10AE9000765D0FE196A302D0230E09D05751100B17
:10AEA00001E178D05751200B01E174D02A0E196FBF
:10AEB00071D0E251040B6EE08A51400B6BE0EDEC77
:10AEC000C4F068E101014E0E1A6F2F0E1B6F410E88
:10AED0003ED0760514E1D8ECD3F0DE0EE66EC00E5F
:10AEE000E66E010E0AECD0F00BC200F0D8ECCDF00B
:10AEF0000101195D02E1200E196F1B8F27D0020E90
:10AF0000765D27E1D8ECD3F0D60EE66EC00EE66E85
:10AF1000010E0AECD0F0010183513CE033AC02D0C9
:10AF20002A0E186F060EE66E820E5BECCCF0005017
:10AF300002010B5D006E0101030E016FD8ECCDF034
:10AF40000101195D02E1200E196F1B8F560E1C6F57
:10AF500021D0030E765D03E19EEC10F01BD07651FC
:10AF600019E143ECDCF016D0020119510BE0275037
:10AF7000400B10E1140E0101A85D0CE23B0E7CECCD
:10AF8000C4F008D00101B1A105D023AA03D0239AAF
:10AF900093EC34F0D9EC14F0006EFF0811E0570E7A
:10AFA000005C0AE1B1ECCDF0CE0EE66EC00EE66EAE
:10AFB000010E0AECD0F004D00050006E8EEC26F0AA
:10AFC0000101A95101E046D2140EA96F02015651A8
:10AFD00001E05607020E685D01E03CD2320E01012D
:10AFE000B55D04E00D0EB55D01E034D2258232D2AC
:10AFF000090EB35D0AE106015051515D01E12AD20B
:10B0000050C651F62AEC3DF025D20A0EB35D05E19B
:10B0100003ECD8F0CEECD7F01DD20B0EB35D01E0FF
:10B0200019D2B45122E1DBEC11F0B3ECCEF001E126
:10B030000BD28A51400B09E0EDECC4F001E104D2DF
:10B04000040E0101765D01E0FFD149EC13F0070128
:10B05000BC0ED880AB55020EAC5501E3F5D1010111
:10B060008A51400B01E0F0D13AD0B40543E11FEC26
:10B07000CAF001E3E9D11FECCAF001E3E5D11B50AE
:10B08000080B01E0E1D1CCECCDF00DE2770E7CECC9
:10B09000C4F0CAECD7F09BECD2F0B10EE66EC00E55
:10B0A000E66E010EE6D0C80E01ECD3F02AEC13F0E8
:10B0B0000701A80E4DECD2F00DE2A00EE66EC00E18
:10B0C000E66E010EBDECC4F0980EE66EC00EE66EA4
:10B0D000010EA3D0760E4DECD2F001E3B5D1BD0E3A
:10B0E000E66EC00EE66E010EBDECC4F0770E7CEC91
:10B0F000C4F0E7D0020EB45D01E0E6D054EC10F0ED
:10B10000EDECC4F001E195D02050040B01E091D0AA
:10B110002050400B01E08DD05E0EDE6E010EDD6E24
:10B1200001012B51090804E2900EDE6E010EDD6E66
:10B13000E2A504D0F40EDE6E010EDD6E21B204D065
:10B14000640EDE26000EDD22AEECC4F001E37CD1FD
:10B150001B50080B01E078D154EC10F087ECD2F0D2
:10B16000AEECC4F001E370D154EC10F0050E9EEC8F
:10B17000C3F0AEECC4F001E367D12CA609D012EC09
:10B18000C4F003E08AECC4F00AE00DECD1F007D083
:10B190000101665183ECC9F0665FD1EC52F0460EB6
:10B1A00001ECD3F0AEECC4F001E34ED1170E0DEC80
:10B1B000C4F02CA609D012ECC4F003E08AECC4F071
:10B1C00011E00DECD1F00ED0800EE66EC00EE66EF2
:10B1D000010EBDECC4F0010166515CECD1F0665F7C
:10B1E000D1EC52F0960E01ECD3F08AECD0F0320E96
:10B1F000E4ECCDF00201CD51495CCE514A5801E357
:10B2000023D16D0EE66EC00EE66E010EBDECC4F0ED
:10B21000650EE66EC00EE66E010EFFECCBF0C4ECE0
:10B2200010F0010EE66ED9EC10F0E55209EC11F0C9
:10B230000BD103EC53F0000901E106D11B50080BC0
:10B2400001E002D154EC10F003EC53F0000901E1ED
:10B25000FBD0170E52ECD2F00101E2A510D04851FC
:10B2600029E0480594ECC6F0570EE66EC00EE66E77
:10B27000010EE66E85EC14F0E552E552E4D048513B
:10B28000320809E2360EE66EC00EE66E010EBDEC27
:10B29000C4F0320E0BD048511E080CE2280EE66EA8
:10B2A000C00EE66E010EBDECC4F01E0E94ECC6F0AE
:10B2B000640E86D0440EE66EC00EE66E010EBDEC46
:10B2C000C4F06DECC7F0C0D0030EB45D34E10601EC
:10B2D00050932450020B12E11F50020B04E0CBEC00
:10B2E00029F0000909E01250080B03E11250040B89
:10B2F00005E0E2ECCCF002E0060150832450020BA2
:10B3000001E0A2D0A4ECCBF001E09ED002013051CC
:10B3100001E09AD077ECC7F001E14A5001E194D006
:10B320002C50800B01E090D02C50400B01E08CD0D1
:10B330000601018189D0040EB45D4EE15651040B23
:10B3400049E01F50080B46E0EDECC4F043E0CCECC4
:10B35000CBF040E19AECC9F03DE1D70E99ECC6F094
:10B360002ABC24D07FECCFF004E68F0E495C000E9F
:10B370004A586AE2140E9EECC3F0D70E83ECD2F06A
:10B38000016E050E9EECC3F0D70E99ECC6F0040ECC
:10B3900097ECC7F00050E66E42ECC7F055E02A8CFF
:10B3A0002DEC0CF00201090E336F4ED059ECD1F0A8
:10B3B0000BE249508F08000E4A5406E22A9C140EF4
:10B3C000E66E8CEC21F03FD0020133513DE12DECD3
:10B3D0000CF03AD02A9C38D0050EB45D35E1A30EAE
:10B3E00099ECC6F00101E1A105D00050E66EBEEC7B
:10B3F00075F0E55204902150020B01E00480C00E6C
:10B40000005C02E2219204D00050F00801E22182A7
:10B410002150020B02E08F9001D08F800450010B6D
:10B42000496E2150020B01E0010E495C0DE08CECED
:10B4300004F0EEEC16F0D1EC52F0B5ECC5F0010ED4
:10B44000E66ECDEC1DF0E5520101B42BB4510508B8
:10B4500001E2B46B0101B32BB3510B0801E2B36BF2
:10B46000020EE15C02E2E16AE552E16E5BEFC3F0DD
:10B47000016A710E015C0DE2C70E496EDD0E4A6E67
:10B48000010E4B6E01501FECCEF097ECC9F0012A73
:10B49000F0D71200026A400E025C08E2B00E0224ED
:10B4A000016E320E97ECC9F0022AF5D71200BAEC01
:10B4B000D0F0060F016E040E97ECC7F08D0EE66E0D
:10B4C000020ED1ECC3F0096A5BEFC3F0BAECD0F026
:10B4D000060F016E040EE66E8D0EE66E020E4EEC49
:10B4E000D0F05BEFC3F0BAECD0F00A0F016E020EA1
:10B4F00097ECC7F0910EE66E020ED1ECC3F0096A2C
:10B500005BEFC3F0BAECD0F00A0F016E020EE66EEC
:10B51000910EE66E020E4EECD0F05BEFC3F014EC31
:10B52000CEF0340E62ECCCF0010E096EDF6A100E24
:10B53000DF5C42E2026A100E025C3CE246ECCFF0B5
:10B5400003E0050E025C06E1DF50E824820FBAEC4E
:10B55000C5F0006E020403E0060E025C07E1DF5056
:10B56000E824820F010FBAECC5F0006E020EDF5C1A
:10B5700003E3030EDF5C0AE10A0E025C02E1110E36
:10B58000006E0B0E025C02E1240E006E0C0E025CDB
:10B5900005E10A0EDF5C02E11B0E006E0D0E025C7F
:10B5A00005E10A0EDF5C02E1200E006EB1EC3AF01C
:10B5B000022AC1D7DF2ABBD7020E096EDF6A090E45
:10B5C000DF5C12E2026A100E025C0CE246ECCFF085
:10B5D00003E0050E025C02E11C0E006EB1EC3AF0D5
:10B5E000022AF1D7DF2AEBD7096A42DFDF6A200E91
:10B5F000DF5C09E2100E006E800EDF24016EB1ECFC
:10B600003AF0DF2AF4D7DF6A0B0EDF5C03E242DF99
:10B61000DF2AFAD7DF6A090EDF5C35E2DF28006E29
:10B620000038F00B006E090E0012DFCFE6FF1FECB2
:10B630000CF0E552D0ECD1F0EE52090EEF6E8AEC30
:10B64000C3F0020E38ECCFF02C0EEF6E8AECC3F094
:10B65000030E38ECCFF0010EEF6E8AECC3F0040E4F
:10B66000BAECCFF0050EBAECCFF0070EBAECCFF083
:10B67000080EBAECCFF0060EBAECCFF0090E39EC9A
:10B68000C8F0DF2AC8D71FD829D8DF6A060EDF5CCA
:10B690000DE2DF5002E1030E01D0010EE66EDF5035
:10B6A0009BECC4F0BFECC5F0DF2AF0D7D3ECD2F0AE
:10B6B000FD0E016EDB0E97ECC9F00101010EB16FBA
:10B6C000E5525BEFC3F0020E096E5A0EE66E000EF5
:10B6D000E66E030EE66EA20E82EFD3F0B3ECD3F06B
:10B6E000030E096EFE0EA2ECD3F0850E005C02E0A4
:10B6F000010EDF6E2D0E62ECCCF0140EE2ECC9F000
:10B70000000EE66E0A0E21ECC4F00A0EE2ECC9F05F
:10B71000CA0EE66E0A0E21ECC4F0040EE2ECC9F08B
:10B72000260EE66E0A0E21ECC4F0DF501DE00F0E6F
:10B73000E2ECC9F0140EE66E0A0E21ECC4F0030E22
:10B74000E2ECC9F0230EE66E0A0E21ECC4F00A0109
:10B750002D0E1B6F1BCA1AFA1BCA19FA410E206F55
:10B7600020CA1FFA20CA1EFA0A01D46BDA6BDA81EA
:10B77000D56B380ED66F040ED86F3C0ED96F190EEC
:10B78000D76F016A020E015C0CE20150050D86ECD8
:10B79000D3F0000EE9260A0EEA22360EEF6E012AD9
:10B7A000F1D70101D06B050ED05D18E20701010E43
:10B7B000B16FFF0EB15D0FE0F9EC13F012ECD3F0B6
:10B7C00063ECD0F00701B151F2ECD2F05FECC6F0BF
:10B7D0000701B107EED70101D02BE5D70701B16B07
:10B7E0000101D06BDFCFE6FF22EC48F0E5525AECC6
:10B7F00048F0030E096EFE0E016E850E97ECC9F03F
:10B80000096AE5525BEFC3F00490049201013EB176
:10B8100004803EB304820450010B02E08E8E01D0FE
:10B820008E9E0450020B02E08F8801D08F98405109
:10B83000E8240A0FE66EE66A43ECFCF0E552E552B6
:10B840000C0EBB6E006A01013E5104E1100E3F0375
:10B85000F350006E0050BC6E12005FECC3F051EC70
:10B86000CEF010ECFDF0E552000902E0C69EF7D7DD
:10B870005BEFC3F0C79EC698C78C1200C78EC68800
:10B88000C78C1200F29E080EDCECCBF0480E6EEC7A
:10B89000C3F0E66AE66A480E8BECD3F090ECD3F086
:10B8A0000701800E146FF90E156F23ECCEF028EC13
:10B8B000CEF0F28E1200D9CFE6FFE1CFD9FF030E12
:10B8C000E1260BEC10F0E668930EE66E9CECFCF0C3
:10B8D000E552E552AA9EC26A000000000000000086
:10B8E00000008A8A209A3386278A10EC14F0060119
:10B8F000B66BB76B37EC0DF0A3ECF6F037ECF7F066
:10B9000089888F0EE66EE668BDECFAF0E552E552E6
:10B91000CF0EE66EE6680EECFCF0E552E552050E41
:10B92000E66E2EECFDF0E5520101010E3E6F0101C5
:10B93000030E3F6F0101020E406F66DFE668870E5F
:10B94000E66E72ECFCF0E552E552B09E0201320E5A
:10B95000116F000EA56EA26E9F6EA282D08E010E98
:10B96000C26EC16A0A0EC06E0F01DF0E256F0F0195
:10B97000F70E246F0F01E00E236FDB0E006E9BECC1
:10B9800025F000C04AF5010EDB6A100EF36E010EC1
:10B99000DBCFF4FFF350F45C28E2A90E496EDF0E12
:10B9A0004A6E010E4B6E010EDBCF4CF04D6A4E6AB3
:10B9B00049504C24F36E4A504D20F46E4B504E20AB
:10B9C000F86EF4CFF7FFF3CFF6FF0800F550E66E00
:10B9D000010EDB50EA6AC50FE96E060EEA22E55257
:10B9E000E750EF6E010EDB2AD0D70101266B010173
:10B9F00026918850010B01E0268101012693885091
:10BA0000020B01E02683F28E060150692AEC3DF01C
:10BA100089ECD9F00101D60EAE6FD70EAF6F010ED3
:10BA2000B06F020184690601506B2AEC3DF0010100
:10BA3000010EB16FC8ECD3F0D8ECD3F091EC6FF0FD
:10BA4000060117810601416941C640F60601426BB5
:10BA5000138A128011881182138613880A01380E06
:10BA6000D66F0A01010ED76F76EC19F0CEECD7F045
:10BA700013EC20F0010EE66E90EC3DF0E552166EF0
:10BA8000200E165C0AE101013889010EE66E90EC89
:10BA90003DF0E552000901E0F8D7640EE66E62EC75
:10BAA000FDF0E5521C9E37ECF7F0096AFC0E016EC2
:10BAB000F4EC3AF0001CDF6EFC0E016EDF50006EFD
:10BAC000B1EC3AF0FC0E016EF4EC3AF0DF50005CA1
:10BAD00006E0210EE66E9AEC14F0E5524ED0830E8D
:10BAE000096EFC0E016EF4EC3AF0001CDF6EFC0EE9
:10BAF000016EDF50006EB1EC3AF0FC0E016EF4EC1A
:10BB00003AF0096ADF50005C06E0240EE66E9AEC1B
:10BB100014F0E55232D0FD0E016EF4EC3AF0DB0E7B
:10BB2000005C03E1210E165C02E1F9DC1ED0020E7E
:10BB3000016EF4EC3AF000C02AF1370E016EF4EC1D
:10BB40003AF000C05FF1110E016EF4EC3AF000C063
:10BB500039F1120E016EF4EC3AF000C03AF10F0E1A
:10BB6000016EF4EC3AF000C037F1E00E016EF4EC37
:10BB70003AF00050800801E28DDC31880701580E50
:10BB8000626F020E636F07018B69B6EC0CF05BEC21
:10BB90001EF037ECF7F055EC3DF01F860001116AFE
:10BBA000126A136A146A800E076E176A219A710E60
:10BBB000E66EE66A280EE66E010EE66E1FEC3BF0BE
:10BBC000E552E552E552E552020E096E5A0EE66E56
:10BBD000A20EE66E000EE66E030EE66E1FEC3BF064
:10BBE000E552E552E552E552030E096E2A0EE66E65
:10BBF000E66A000EE66E0A0EE66E1FEC3BF0E552BA
:10BC0000E552E552E552AA0EE66E300EE66E2A0EB9
:10BC1000E66E0A0EE66E1FEC3BF0E552E552E55289
:10BC2000E552FE0E016EF4EC3AF0096A850E005CF6
:10BC300001E054DD060EE66EF00EE66EB80EE66E1E
:10BC4000070EE66E1FEC3BF0E552E552E552E55279
:10BC5000040EE66EA00EE66EEA0EE66E060EE66EC8
:10BC60001FEC3BF0E552E552E552E5520601EA5180
:10BC70000A0802E20601EA6B0601EC51010802E241
:10BC80000601EC6B200EE66E800EE66E640EE66E2C
:10BC9000070EE66E1FEC3BF0E552E552E552E55229
:10BCA000830E096EF90E016EF4EC3AF000C071F2E9
:10BCB00002017151C80803E20201C80E716FF80E4B
:10BCC000016EF4EC3AF0339A6E0E005C01E1338AB7
:10BCD000DF0E016EF4EC3AF00101DF91720E005CB0
:10BCE00002E10101DF817E0E096E080EE66EE66A52
:10BCF000B60EE66E020EE66E1FEC3BF0E552E55224
:10BD0000E552E552096A1C0E165C10E10101368FFE
:10BD10000101368D0101369136833695010EE66EAE
:10BD200090EC3DF0E552000901E0F8D7090E165CF1
:10BD300009E11B86010EE66E90EC3DF0E55200092C
:10BD400001E0F8D701018051060802E20101806B91
:10BD5000CFEC04F0DBEC0CF001018DAB06D001015F
:10BD60003C9F01013C9D01013B9F0A0E0101985D32
:10BD700004E301019851640803E201011E0E986F6B
:10BD8000010101015751200B07E001010101575149
:10BD9000100B02E10101579BB6C201F0BDC202F0D7
:10BDA000FF0E015C07E0015005E0FF0E025C02E0BF
:10BDB000025008E102017C0EB66F0201FA0EB76F65
:10BDC00017EC4EF001018351050802E20101836B7B
:10BDD00001018451020802E20101846B0101425118
:10BDE00004E001014251020803E20101020E426F28
:10BDF00001016D51230803E201010A0E6D6F01017B
:10BE00005F8D0101505104E0010150510D0803E222
:10BE10000101010E506F0601EA510A0804E2060111
:10BE2000EA6B0601EB6B01018E9D01015783010155
:10BE30002E6B460E0101525D04E30101525173085D
:10BE400003E20101540E526F640E01014A5D0BE3DF
:10BE500001014A51496E4A6A4A3404E24950B40821
:10BE6000000E4A5403E201018C0E4A6F0101555144
:10BE7000150804E3030E0101555D03E20101150EEF
:10BE8000556F040E0101475D04E3010147510808A5
:10BE900003E20101050E476F01017D51496E4A6AB7
:10BEA000D8904A5004E6C80E495C000E4A5803E296
:10BEB0000101D70E7D6F01014D51496E4A6A4A3426
:10BEC00004E249509608000E4A5403E201018C0E28
:10BED0004D6F01014C51320803E20101280E4C6FF5
:10BEE00001014B51496E4A6A4A3404E24950C8087C
:10BEF000000E4A5402E201014B6B0A0E0101415D42
:10BF000004E3010141510F0803E201010F0E416FEB
:10BF100001013551500803E20101010E356F0101A5
:10BF20002851280803E20101280E286F550E01014F
:10BF30004E5D07E0680E01014E5D03E00101680EF1
:10BF40004E6FFF0E0101695D03E00101695109E1D6
:10BF50000101C80E696FD90E6A6FCF0E6B6F060EA6
:10BF60006C6F01017751010802E20101776B010159
:10BF700066513C0802E20101666B010167513C0811
:10BF800002E20101676B01016851280802E2010128
:10BF9000686B010101018D51020B05E101013A516C
:10BFA00002E001018D8301016151030802E20101F8
:10BFB000616BFF0E01015F5D02E101015F6B010139
:10BFC0007151496E4A6A4A3404E24950C808000E69
:10BFD0004A5403E20101C80E716F01017351496EA9
:10BFE0004A6A4A3404E24950C808000E4A5403E23F
:10BFF0000101280E736F01017251496E4A6A4A3479
:10C0000004E24950C808000E4A5403E201010C0E34
:10C01000726F01017551496E4A6A4A3404E249500F
:10C02000C808000E4A5403E201011E0E756F01019B
:10C030003151020803E20101010E316F3C0E010192
:10C04000E76E7C19E8AE02D07C3503D0E750D8808B
:10C050007C550BE3C40E0101E76E7C19E8AE02D0FB
:10C06000E73402D0E7507C5D02E201017C6B010104
:10C0700086510F0802E20101866B01017B510F0816
:10C0800002E201017B6B01016E513C0802E20101F9
:10C090006E6B01016F513C0802E201016F6B0601FA
:10C0A000EB511E0802E20601EB6B0601ED511E0882
:10C0B00002E20601ED6B01017F51640803E2010118
:10C0C0001E0E7F6F01012951496E4A6AD8904A506D
:10C0D00004E6280E495C000E4A580BE30101295181
:10C0E0004B6E4C6A4C3404E24B504608000E4C54E4
:10C0F00003E20101370E296F01018551C80802E2F0
:10C100000101856B01018551780803E20101780E78
:10C11000856F0201875104E002018751330803E271
:10C1200002010D0E876F01018751780803E20101BA
:10C13000640E876F010193510C0803E20101060EA2
:10C14000936F010195510C0803E20101060E956FF2
:10C15000010188511E0802E20101886B01018AAFCA
:10C1600002D001018A6B01018DAF02D001018D6BFC
:10C1700001018EAF03D001010A0E8E6F010196AF4F
:10C1800003D00101600E966F1E0E0101895D04E36C
:10C1900001018951280805E201011E0E896F010184
:10C1A0008A9101018B510A0802E201018B6B0101A6
:10C1B0007A51190804E201017A6B01018A930101A5
:10C1C000705104E0010170511E0803E201011E0ECE
:10C1D000706F01013E51010803E20101010E3E6F43
:10C1E000210EE66E1DEC14F0E552000909E0010194
:10C1F000010E3E6F0101030E3F6F0101020E406F01
:10C2000004EC5CF005014B69BCEC0AF00101DF8332
:10C2100001012951E8240301B86F54EC21F0300EDC
:10C22000010184250401F76F020E0101845D03E121
:10C230000401340EF76F6EECA7F004013B0EFE6FA5
:10C240000501106B10C512F510C511F50501800E22
:10C25000156F34ECF3F04EECF3F05AECF3F0000908
:10C2600005E12D0EE66E9AEC14F0E55207013C0E46
:10C27000846F0101D16BD1C1D0F10701B16B31ECF9
:10C2800075F00701BE81B6EC0CF05CEC1EF0D1EC51
:10C2900052F0EBEC52F00101010138510701099F06
:10C2A000040B01E0098F7FEC20F059ECF6F027DB5E
:10C2B00037ECF7F0DBEC11F0F3CF0EF0F4CF0FF02A
:10C2C000430E0E5C010E0F5806E3D30ED8800E54B9
:10C2D000020E0F5411E20EC049F00FC04AF0040ED6
:10C2E000D8904A324932E804FBE149C026F75A0E99
:10C2F000E66E9AEC14F0E5522AEC13F0F3CF0EF050
:10C30000F4CF0FF01F0E0E5C010E0F5806E3D30E94
:10C31000D8800E54020E0F5411E20EC049F00FC027
:10C320004AF0040ED8904A324932E804FBE149C091
:10C3300026F75D0EE66E9AEC14F0E552550EE66EA9
:10C34000020EE66E400EE66E79ECF6F0E552E5522E
:10C35000E552AA0EE66E020EE66E420EE66E79EC2D
:10C36000F6F0E552E552E552020EE66E400EE66E3C
:10C37000C6ECF6F0E552E552550802E1000E01D098
:10C38000010E006E005007E000C026F7600EE66E5A
:10C390009AEC14F0E552020EE66E420EE66EC6EC22
:10C3A000F6F0E552E552AA0802E1000E01D0010EB6
:10C3B000006E005007E000C026F7630EE66E9AECB0
:10C3C00014F0E552E66A020EE66E400EE66E79EC77
:10C3D000F6F0E552E552E552E66A020EE66E420ECE
:10C3E000E66E79ECF6F0E552E552E5520201440EB4
:10C3F000976F120EE66E420EE66EC6ECF6F0E55250
:10C40000E552046E026E0450800B01E0010E496E8D
:10C410000450400B01E0010E495C23E1047C045010
:10C42000E66E120EE66E420EE66E79ECF6F0E5521E
:10C43000E552E552120EE66E420EE66EC6ECF6F0DE
:10C44000E552E552046E0450800B01E0010E496E86
:10C450000450400B01E0010E495C03E10201450E6E
:10C46000976F0250E66E120EE66E420EE66E79ECA3
:10C47000F6F0E552E552E5520101835116E0B7ECC2
:10C48000DCF000090AE044ECDBF0A3ECDBF0010196
:10C490008351010801E2338C08D00701050E266F95
:10C4A0001E0EE66E9AEC14F0E552FFECBCF02B96F3
:10C4B000229601013A510101941101E17CD0150E3F
:10C4C000E66E020EE66E440EE66E79ECF6F0E5528C
:10C4D000E552E5522A0EE66E020EE66E460EE66E56
:10C4E00079ECF6F0E552E552E552020EE66E440EA6
:10C4F000E66EC6ECF6F0E552E552150802E1000ED4
:10C5000001D0010E006E005014E001013A5108E024
:10C5100000C026F7660EE66E9AEC14F0E55208D0DD
:10C520000701030E266F180EE66E9AEC14F0E55222
:10C5300042D001013A5118E0020EE66E460EE66E58
:10C54000C6ECF6F0E552E5522A0802E1000E01D0F1
:10C55000010E006E005008E000C026F7690EE66E7E
:10C560009AEC14F0E55227D0120EE66E440EE66EF9
:10C57000C6ECF6F0E552E552006EC00E0016010161
:10C580003A510CE0005008E000C026F7840EE66E39
:10C590009AEC14F0E55201D02B860DD0C00E005C51
:10C5A00009E00701040E266F180EE66E9AEC14F0EF
:10C5B000E55201D0228642EC5CF01B9201019451BD
:10C5C0001FE0370EE66E020EE66E480EE66E79EC60
:10C5D000F6F0E552E552E552020EE66E480EE66EC2
:10C5E000C6ECF6F0E552E552370809E00701010E06
:10C5F000266F180EE66E9AEC14F0E55201D01B82FD
:10C600002580E66818EC36F0E55239C1E6FF9BEC70
:10C61000C2F0E5520101B181219401013BBB06D07A
:10C6200006015095060150872AEC3DF00101D051DA
:10C6300004E0030E0101D05D04E10A01D46B149CF7
:10C6400004D00A01020ED46F148C93D901012ABDC3
:10C650000CD061ECF4F0C6C269F1C7C26AF1C8C27D
:10C660006BF1C9C26CF101012A8D64EC2EF002015C
:10C67000320E246F01010F0EB56F0501010E176F09
:10C680000901020EE56F0201582B0201320E226FE2
:10C6900052EC96F08CEC04F00201CF5108080AE24B
:10C6A00010EC14F0CFC226F72A0EE66E9AEC14F0C6
:10C6B000E5521B860D0EE66E15EC15F0E552870B64
:10C6C000006E005008E000C026F73C0EE66E9AECC3
:10C6D00014F0E55214D040EC20F03B0E0E5C000E3E
:10C6E0000F5806E3E60ED8800E54030E0F5407E2EF
:10C6F0000EC026F7570EE66E9AEC14F0E552030EC4
:10C70000E15C02E2E16AE552E16EE552E7CFD9FF72
:10C710001200430E0101B55D03E3B551480801E283
:10C72000000C010C01013B7B279D256B1DD8238A42
:10C73000258201013BBB13D009014F0EE66F460E67
:10C74000E76F060150A707D00901560EE66F420EAB
:10C75000E76F010136890601436B43C642F60101CA
:10C760003BBB0480C7EF09F00601509750950101CB
:10C770003BBB07D021B403D006015085120006014F
:10C78000508712000A01D651A6EFD3F0D0C100F0B5
:10C79000005003E0030E005C33E100500EE10101A4
:10C7A000CC7D0901430EE66F0101CCAD02D080ECD7
:10C7B000CAF00101CCAD20D010D0F2ECC6F00FE0F1
:10C7C0000101CC750901440EE66F0101CCA502D030
:10C7D00080ECCAF00101CCA50FD004800DD001017E
:10C7E000CB750901440EE66F0101CBA502D080ECA8
:10C7F000CAF00101CBB50480C7EC09F0DEEFCCF044
:10C80000000403E0020E005C16E1F9EC13F00004F2
:10C8100002E1020E01D0010E006E09014C0EE66F1E
:10C82000020E005C03E10480550EE66FC7EC09F0D0
:10C8300000C0D0F166D812000101325103E112ECC0
:10C84000C4F002E0000E01D0010E1492E8B0148290
:10C8500012ECC4F003E1E8ECCDF00CE112ECC4F012
:10C8600007E08AECC4F004E101013B51800B02E1D6
:10C87000000E01D0010E1490E8B01480120012ECEA
:10C88000C4F00AE0D4ECCBF007E1A8ECCBF004E074
:10C89000B3ECCEF001E1000C010CD0ECCBF003E0E6
:10C8A000010181511200010178511200D0ECCBF04E
:10C8B00003E00101825112000101795112005FEC85
:10C8C000C3F0D0ECCBF005E0FE0EDB500101816F30
:10C8D00004D0FE0EDB500101786F5BEFC3F05FEC1C
:10C8E000C3F0D0ECCBF005E0FE0EDB500101826F0F
:10C8F00004D0FE0EDB500101796F5BEFC3F025EF32
:10C90000D0F021902792D0C100F00050800802E2C0
:10C91000050E006E060E005C01E3006A000402E1F1
:10C920000101CB91020E005C02E10101CB8100C04C
:10C93000D0F1248A20BE03D065ECCDF002D08EEC7D
:10C9400039F041EF25F014ECCEF0030EDF6E01015B
:10C950004951496E4A6AB00E3D6E040E3E6ED7ECE8
:10C96000C3F03D50D880DF540201506FE5525BEFB9
:10C97000C3F014ECCEF026B00ED0320EDF6E080EEF
:10C980000101495D02E2080E496FDF50D880495528
:10C9900002E2DFCF49F1D7DFE5525BEFC3F050C2CF
:10C9A000ACF122AE33D0006A01013D510C0803E323
:10C9B000070E3D5D02E20C0E3D6F070E3D5D4D6EB4
:10C9C0004E6A02015051DBECC4F062ECCDF0010183
:10C9D000AC514B6E4C6AFF0ED8804B56000E4C5635
:10C9E0004A504C18E8AE02D04C3404D04B50495C4D
:10C9F0004C504A580BE20050D880AC5507E223A0B7
:10CA000003D00050AC2702D00050AC5F9AECC9F0C4
:10CA100008E102012D510601EA1106E02750400B02
:10CA200003E11D925BEC3CF01200050ED2ECC7F066
:10CA3000580E2BEFC8F0F9DF258E1200180E0DEC02
:10CA4000C4F0010136AD03D0580E2BEFC8F0258E8F
:10CA500012005FECC3F0050EE1261FA20FD0BBC190
:10CA6000DFFF010EBCC1DBFF020EBDC1DBFF030E09
:10CA7000BEC1DBFF040EBFC1DBFF0ED0B6C1DFFFBE
:10CA8000010EB7C1DBFF020EB8C1DBFF030EB9C157
:10CA9000DBFF040EBAC1DBFFB3ECCEF022E0E151C4
:10CAA000100B1FE13851010B03E19651040B06E016
:10CAB000320EDF5C62E3DF5033085FE32E50800B01
:10CAC00006E0320EDF5C59E3DF50350856E32E50A6
:10CAD000800B3BE12F0EDF5C50E3DF50380835E27E
:10CAE0004CD0DF504AE0DF0404E1460EA7ECC5F06D
:10CAF00044E3DF50180806E21C0EDF5C03E29651A7
:10CB0000010B23E1E1BD07D0DF50180815E21C0E30
:10CB1000DF5C12E232D0190EDF5C2FE01A0EDF5C10
:10CB200004E1010EDB505F0828E31B0EDF5C04E12B
:10CB3000290EA7ECC5F021E32B50100B06E12E5077
:10CB4000800B03E02B510A0802E2F36A1BD0630E4C
:10CB5000E66E020EE66ED9CFE6FFDACFE6FFBAEC5C
:10CB6000C6F00BE1D9CFE6FFDACFE6FF5E0EE66E48
:10CB7000020EE66EBAECC6F004E060DF010EF36E62
:10CB800001D0F36AF46A050EE15C02E2E16AE55263
:10CB9000E16E5BEFC3F065C301F022A802D078C359
:10CBA00001F00E0E015C01E2010C100E015C01E2CD
:10CBB000020C120E015C01E2030C140E015C01E296
:10CBC000040C160E015C01E2050C1B0E015C01E277
:10CBD000060C220E015C01E2070C080C35ECCEF0CD
:10CBE00083ECD2F0F00801E2006A00505BEFC3F082
:10CBF0005FECC3F051ECCEF0F1DFE552FE0EDB50FE
:10CC00009B0805E1030EAFECCEF04FECC7F07FECD4
:10CC1000CFF004E6BE0E495C000E4A580AE2560EFA
:10CC2000496ED90E4A6E010E4B6E00501FECCEF0CD
:10CC300001D0B00E0E6E0F6A7FECCFF004E6AA0EA4
:10CC4000495C000E4A580CE2AC0E496ED80E4A6E92
:10CC5000010E4B6E00501FECCEF00101D46F02D0DC
:10CC60000101D469D56B5BEFC3F014ECCEF00490F6
:10CC700034B80480B30E016E0101E2A539D01BB6B1
:10CC80002AD0B30EBEECCFF0D4C1D7F238EC20F0EE
:10CC9000026E300EDF6E020403E0020E025C02E15F
:10CCA000380EDF6EDF500201D880D75509E263EC01
:10CCB0000EF0210EE66EC00EE66E010E8FECC3F094
:10CCC000DF50496E4A6A0101D451495CD5514A5836
:10CCD00002E24851D6E1070114B108D0148123ECD7
:10CCE000CEF07D0E976E080EE9ECD0F09B0E016E33
:10CCF0000150BEECCFF0D2ECC4F012E00E500101B6
:10CD0000D26FD36BB30EBEECCFF00E50FFECCEF073
:10CD10000101D2274A50D323D2C10EF0D3C10FF064
:10CD20000101E2A502D0D46BD56BD4C161F3D5C1AA
:10CD300062F334B82CD113A64DD00B50016E2250A3
:10CD4000100B03E13450800B02E024D913D0D2EC55
:10CD5000C4F010E00701C1514D6E4E6A0B50DBEC80
:10CD6000C4F0016E2050800B05E00901EC5102E097
:10CD7000ECC901F0050E0124496E0A0E43ECC4F023
:10CD8000016E015005E12250400B02E0010E016EE0
:10CD900012ECC4F003E03450400B05E001C0A3F7EF
:10CDA00002010A0E08D00701A351015C05E301C08E
:10CDB000A3F702010C0E2A6FEEDE0701A46F2B50C1
:10CDC000100B03E1040E0B5C01E2A46B1DECC9F037
:10CDD00073ECC7F0F6ECC6F00480005009E0345064
:10CDE000400B06E1030E005C04E1020E0A5C01E167
:10CDF0000490070E016E04A004D0090EE3ECC4F009
:10CE0000016E0F0E01140201736F070E73170138C4
:10CE10000F0B016E04A0016A13A408D0020EE66E87
:10CE200073C2E6FF0150E66E73ECC7F052C100F02A
:10CE30000101E2A502D04AC100F00EECD3F025ECCE
:10CE4000C5F033ECCFF0A0ECCFF0640ED6ECD1F00F
:10CE50000E500B6EF6ECC6F0040E005C22E1100ED4
:10CE6000016E0150496E4A6AACC23DF0ADC23EF05F
:10CE7000D7ECC3F03DC0AEF20B50FFECCEF0020198
:10CE8000AC274A50AD23AE51496E4A6AAC51495C59
:10CE9000AD514A5806E2AE51FFECCEF0AC5F4A50BD
:10CEA000AD5B000409E0020E005C06E0030E005CCE
:10CEB0000AE1020E0A5C07E00201AF51D8800B5470
:10CEC00002E20BC0AFF20101E2A507D00301636BE0
:10CED000646B676B686B656B5AD0B70EBEECCFF0B6
:10CEE000D4C163F3D5C164F303016151635D625141
:10CEF000645906E3010E6325616F000E6421626FC1
:10CF000061516325676F62516421686F67516725BE
:10CF1000496E685168214A6E67C34BF068C34CF094
:10CF2000030ED8904B364C36E804FBE149504B24B5
:10CF30000301676F4A504C20686F6351615D496E11
:10CF4000625164554A6E33ECCFF067C33DF068C35D
:10CF50003EF0BDECFDF03DC067F33EC068F367C333
:10CF600065F367C349F068C34AF04B6A4C6A4C34B6
:10CF7000000E4C1809E6D880FF0E4954000E4A54A2
:10CF8000000E4B54000E4C5402E203016569E55259
:10CF90005BEFC3F048C101F02B50100B05E1D2EC60
:10CFA000C4F002E0D5C201F01200F6ECC6F0005069
:10CFB0000DE03450400B0AE1050E005C07E0030E63
:10CFC000005C03E1020E0A5C01E0000C010C04822B
:10CFD000ECDF000901E00492348604A23496349810
:10CFE00044DE34B81200F6ECC6F004980496030E42
:10CFF000005C01E10486000403E0020E005C01E134
:10D0000004882250400B01E10FD12250100B01E0A7
:10D010000BD13450800B01E007D13350080B01E1F4
:10D0200003D102011D5101E0FFD01950010B01E1B4
:10D03000FBD004820494B9DF000901E00492040EDD
:10D04000005C01E10484A6DF01505CECD1F0026ECB
:10D05000FAECC3F001C03EF017ECFEF03EC007F161
:10D06000020E0101075D02E2020E076F07510A0876
:10D0700002E20A0E076F04902050800B33E0090192
:10D08000ED5130E0D2ECC4F02DE00901EE51020880
:10D0900029E2030E006EEE51190802E2020E006E44
:10D0A000EE51280802E2010E006EEDA104D00050FE
:10D0B00072ECCBF00480020E0901ED150FE00EECCE
:10D0C000D3F002010051495C01514A5807E2005077
:10D0D000FFECCEF0005F4A50015B0480040E0901B2
:10D0E000ED1793D00450040B04E002500201AE5D32
:10D0F00006E30450040B4DE101500B5C4AE20201CF
:10D10000880E005D130E015901E37FD003016C0E00
:10D11000635D000E645901E378D004B209D00B506E
:10D12000015C0E6E0F6A0E50020100270F5005D0F1
:10D1300004A405D00201002B000E012365D00201DA
:10D140001E5163E10A0E1E6F0150AF5D20E2AF5128
:10D1500003E1735101081BE204A802D0020E1E6F06
:10D160000450080B0FE0030E0A5C03E07351010842
:10D1700009E20101075172ECCBF01F5107E01E914B
:10D180001E4304D0020E0027000E01230480AF6B63
:10D190003CD00450040B05E002500201D880AE558B
:10D1A00007E30450040B31E10150D8800B542DE209
:10D1B000010E036E04A402D0036E0AD004A208D0AC
:10D1C00007C103F004A804D0030E0302F3CF03F059
:10D1D00003500E6E0F6A0450020B06E00450080B59
:10D1E00009E002011F5106E001500B5C47ECD3F04F
:10D1F000A0ECCFF0020100510E5C01510F5805E286
:10D200000E50005F0F50015B048004A00DD002019E
:10D210000251001902E10351011906E0DFEC0BF0A5
:10D2200000C202F201C203F20201205102E00F0E1D
:10D23000206F1200B3ECD3F01750100B0CE0200E4F
:10D24000155C4CE0210E155C49E0150E155C03E100
:10D25000A8ECCBF043E01750010B09E0150E155C6C
:10D260003DE0220E155C3AE01D0E155C37E00A0E1B
:10D27000155C03E12EECC4F031E01950200B12E1F3
:10D28000020119510FE1230E155C28E00B0E155C0D
:10D2900025E0090E155C22E0090E155C1FE0220E48
:10D2A000155C1CE0ECECCDF004E05BEC96F00009C2
:10D2B00015E11D0E155C07E11750100B04E0FEECA4
:10D2C00018F000090BE12050800B06E102016851C3
:10D2D00003E03250200B02E0000E01D0010EDF6EA1
:10D2E000DF50E5525BEFC3F00101E2A509D0070171
:10D2F000158128ECCEF00701149F149323ECCEF097
:10D30000030E23ECCDF08A8607010B9107ECF7F0B2
:10D310001CEC19F012ECC4F003E03450400B11E0A7
:10D320005BEC0BF000090DE0D2EC08F0B3EC16F06A
:10D330006F0ECEECC3F0C80EEDECC6F0D5EC08F0E5
:10D3400002D0B3EC16F0060150912AEF3DF05BC21B
:10D3500048F15CC200F25DC201F2DFEC0BF090EC30
:10D3600023F0B7ECCAF0239612000101AC5103E19F
:10D370002B820850076E2050010B12E012ECC4F013
:10D380000FE11750800B03E013ECCBF006E02050C8
:10D39000040B06E19CECC6F003E06AD9A0EC71F046
:10D3A00012000101050EAB6F2050010B04E0195073
:10D3B000020B01E0AB6B120030ECD2F001013951ED
:10D3C0002BE105C2DFFFD5ECBDF0DF500201055DAA
:10D3D00023E0010E69C3DBFF020E6AC3DBFF030E0D
:10D3E0006BC3DBFF010EE66E78ECBEF0E552010E7A
:10D3F000DB500301695D08E1020EDB506A5D04E168
:10D40000030EDB506B5D08E023ECBDF037ECF7F06A
:10D410001C820101960EA86F040EE15C02E2E16A33
:10D42000E552E16E5BEFC3F00201185107E0186BA3
:10D4300030ECC8F00201D05101E1119412ECC4F0BB
:10D4400009E12050010B06E1E8ECCDF003E12050AA
:10D45000800B0FE09AECC9F00CE11E50400B09E183
:10D46000C3ECC5F004E1020E0101B55D02E0228CBF
:10D47000D18022BC06D0E66AE66A740E85ECC3F061
:10D4800017D0A8ECCBF012E13350080B0FE000C22C
:10D4900049F001C24AF0030E0F0B03E06BECC9F038
:10D4A000FDE149500201005F4A50015BDFEC0BF0E7
:10D4B00002010A0E1E6FAF6B20AE1C84C80E1F6FD8
:10D4C000ACEC16F0780E006E0050EDECC6F059ECA6
:10D4D00018F00201226B0101E2A509D00701148FA7
:10D4E00001012AA102D00701148323ECCEF08A9611
:10D4F000320EEDECC6F08EECC4F014E12B50080BAC
:10D5000011E02250100B0EE101013A050BE012EC84
:10D51000C4F007E12050800B04E102011E0E156FDC
:10D5200001D04ADF2050800B0EE12050010B0BE1AF
:10D5300012ECC4F008E03450400B05E102012D511B
:10D5400002E0050110511DAC02D016EC0CF0208C4D
:10D550003182D5CA85F2F6ECC6F0360E026E380E70
:10D56000036EB6C17DF2DCECD1F03EC07EF22EEC53
:10D570002FF0B6C17BF2DCECD1F03EC07CF21FA2F2
:10D580000AD0BBC17BF2FAECC3F0BCC13EF017EC91
:10D59000FEF03EC07CF222AC26D007010B8F0B813F
:10D5A00007ECF7F01AECCBF008E15751010B05E05E
:10D5B0000701088F089D84ECCEF0030E01012B5D5E
:10D5C00004E102017B51070808E3040E01012B5D11
:10D5D0000AE10A0E02017B5D06E20701088F089747
:10D5E000089584ECCEF02F8E02EC32F00201FA0E98
:10D5F000236F238A2582319222AC02D077ECCDF0C2
:10D600000DEC39F021AE12D0219E10EC0BF0FBECAA
:10D61000CFF03FECCEF00AE03FECCEF007E03FEC7D
:10D62000CEF004E003EC0BF038EF6BF00201145184
:10D6300009E00101E151080B05E1140E01ECC4F011
:10D640000101E187120014ECCEF0050123072451FB
:10D65000EA6A270FE96E050EEA22EFCFDFFF242BDF
:10D6600024511F0801E2246BDF50E5525BEFC3F049
:10D67000BEEC21F00201196B19C255F2C6ECCAF0DA
:10D6800007E0200E01011C5D03E0200E8FECC6F0C8
:10D690000101AC6B006A63EF75F04B0E026E140E65
:10D6A0000301655D07E31AECCBF01EE11E0E0301DA
:10D6B000655D1AE2100E01012B5D16E22B50100B76
:10D6C00003E0640E485D11E02B50100B0DE1280EB5
:10D6D000485D0BE03C0E485D08E0020E395D04E158
:10D6E0005A0E0224485D01E0000C010CB3ECD3F0AB
:10D6F0001B50080B0AE1C3ECC5F009E13B0E010128
:10D70000B55D03E0420EB55D02E1000E36D00101C9
:10D71000815102E0825104E1480E80ECC4F0DF2A1E
:10D720000101785102E0795104E14B0E80ECC4F024
:10D73000DF2AB3DF00091CE164EC35F0000906E0E4
:10D740003F0E80ECC4F0B1ECC9F0DF2A79EC35F083
:10D75000000907E0420E80ECC4F00201916B926B6D
:10D76000DF2A0701C05104E1450E80ECC4F0DF2A36
:10D77000DF5002E07DDF2094DF50E5525BEFC3F025
:10D78000D5ECC7F002E27B5112008651120014EC76
:10D79000CEF00750DF6E27AA03D002011E0E216FC4
:10D7A000050110510201191103E13751381109E047
:10D7B0001D50040B0FE01D50080B0CE01E50010B18
:10D7C00009E01750800B08E02750200B05E1050108
:10D7D000105102E04DDFB5D207504AE127BA05D01B
:10D7E000010EC7ECC6F0020E87D080DF000901E011
:10D7F000A8D20201245101E0A4D220B002D014DE4C
:10D800000AD02D5108E00501105105E1A4ECCBF040
:10D8100002E124ECD2F0A8ECCBF019E1020189A5D9
:10D8200014D0330E875D0EE10101E051800B03E15E
:10D830002D50080B0CE02D96A7EC04F00201330EDE
:10D840003A6F05D0A7EC04F002D0ABEC04F098DFFF
:10D85000050DF3CFABF10101E2A512D10A0EAB5DCC
:10D8600002E20A0EAB6F0701159128ECCEF008D149
:10D87000070420E10101AB5101E05FD21F9C8EEC57
:10D88000C4F002E01F8C05D0A4ECCBF002E134EC34
:10D890000BF00101280EAB6FE2A505D0070115853D
:10D8A000158328ECCEF020AE03D00101050EAC6F3D
:10D8B000072A17D0020E075C16E10201155102E09B
:10D8C0001E0E156F27BA06D00101AC5101E035D20A
:10D8D00008505DD10101AB5102E1E7EC67F03EEC8D
:10D8E0000BF043DD2AD2030E075C3CE127BA06D0D9
:10D8F000006A63EC75F0070E076E23D22BA218D0D6
:10D900005BC1ABF10101AC5105E03ADF050DF3500D
:10D910000101AB272B922050010B04E01950020BA0
:10D9200001E0AB6B02012D5103E0006A63EC75F07E
:10D930000101AB5106E012ECC4F00FE03450400B93
:10D940000CE11F50400B05E102012D5102E139ECC1
:10D950000BF00101280EAB6F19D126B8EED1E7EC20
:10D9600067F0EBD1050E075C62E10101AB5101E00C
:10D97000E4D1072A269820B0E0D11C0E016E00DF0A
:10D98000E8240124006E0201765107E00050765D24
:10D9900004E2090E076E2688D0D1318207010B9F61
:10D9A00007ECF7F01AECCBF008E15751010B05E05A
:10D9B0000701089F088D84ECCEF0030E01012B5D5A
:10D9C00004E102017B51070808E3040E01012B5D0D
:10D9D00011E10A0E02017B5D0DE20701089F030EB3
:10D9E00001012B5D03E10701088502D007010887CB
:10D9F00084ECCEF00101E2A508D00701159515933E
:10DA000028ECCEF001010A0EAB6F209C85C2D5FA3E
:10DA1000F2ECF6F041ECCDF012ECC4F003E034503F
:10DA2000400B03E00101050EAB6F319286D1060E6B
:10DA3000075C28E10101AB5101E07FD120B01ED08D
:10DA40002650100B0DE1325109E012ECC4F003E056
:10DA50003450400B03E0E8ECCDF002E145DC0ED0A1
:10DA600032C122F226A80AD08BDE99ECD0F0006EEB
:10DA700000500201225D02E200C022F20201566B58
:10DA8000072A5BD1070E075C24E10101AC510FE1CD
:10DA900017AE0BD013ECCBF003E018EC97F005D0E9
:10DAA0008BEC0BF0000901E0179E0850076E020195
:10DAB0002D5101E042D12A5106E03450400B03E1E0
:10DAC0001DECC9F003D0E66AE66AE66A91EC28F03C
:10DAD00047D0080E075C4BE10101AC5106E01D5038
:10DAE000040B03E01D50080B02E10850076E020111
:10DAF0002D5101E122D1E7EC67F03EEC0BF0020181
:10DB00002E5101E01AD17AEC0EF0000901E115D195
:10DB10000501020E266F235111E095DD006E020E05
:10DB20000A5C02E1005010D0016A0501235102E0B5
:10DB30008ADD016E005097ECC7F00ED0105114E151
:10DB4000020E0A5C07E1030EE66E150EE66E59EC56
:10DB500016F007D0E66AE66A160EE66E5FEC16F07F
:10DB6000E552E552E552E9D002012D6BE6D0090EEF
:10DB7000075C28E1020176417F0B76250101D88000
:10DB8000AD5507E20201766B76C2ADF1050E076E68
:10DB9000D4D01EB0D2D0010EAD6F320EAB6F010EDD
:10DBA000076E12ECC4F003E002012D5108E0A4EC72
:10DBB000CBF005E12750200B02E124ECD2F00B0E54
:10DBC000086EBBD00A0E075C06E121BAA9D0179EE9
:10DBD0000B0E076EA7D00B0E075C01E0A6D0175006
:10DBE000800B39E12050010B06E02050040B03E1CB
:10DBF0009CECC6F030E112ECC4F003E03450400B72
:10DC00000CE02050800B09E11E50010B06E01D5076
:10DC1000040B03E01D50080B1EE112ECC4F00CE0F5
:10DC20003450400B09E12050040B06E19CECC6F097
:10DC300003E0D2ECC9F00FE02050800B09E01D504A
:10DC4000040B09E01D50080B06E09CECC6F003E055
:10DC50008EECC4F05BE017AE18D01950800B07E0D3
:10DC60000A0E155C04E01DEC2DF000096AD013ECDF
:10DC7000CBF005E018EC97F0000907E162D08BECDF
:10DC80000BF0000902E0179E5CD012ECC4F023E018
:10DC90003450400B20E18AECC4F01DE119AA06D0F3
:10DCA00003EC0BF0AEEC08F0A0EC1DF09AECC9F020
:10DCB0000AE01950400B07E0249223BC248203ECB5
:10DCC0000BF0C5ECC9F00101885105E088C1E6FF01
:10DCD0008CEC21F0E552ADC176F20101AD5102E0CC
:10DCE000010EAD6F26A802D0E7EC67F00701A16B2B
:10DCF000030E076E800E086E2050800B03E1175054
:10DD0000800B08E020940C0E086E04D022A802D0EC
:10DD100035ECBFF00101AB5105E12650100B02E1DB
:10DD2000E7EC67F03EEC0BF008D00C0E075C05E169
:10DD300021BA03D0C5EC98F007D8DF50075C01E0AA
:10DD40001C8CE5525BEFC3F020AECCD01D50040B11
:10DD5000FDE01D50080BFAE02A840101B19B238AE3
:10DD6000B199258299510BE01FA203D099C1D1F13D
:10DD700002D099C1D0F12EEC2FF081EC64F022504A
:10DD8000100B03E13450800B04E0A7EC69F0349EE3
:10DD900084D083DC000971E0D2ECC4F06EE119ECB0
:10DDA000CDF000C20EF001C20FF00EC04DF00FC05A
:10DDB0004EF0F5ECC4F005ECCAF0FAECC3F00BC27F
:10DDC0003EF055ECD1F0006E0050516E526A536A2D
:10DDD000546A00504D6E4E6A4F6A506A4DC03BF017
:10DDE0004EC03CF04FC03DF050C03EF051C040F03E
:10DDF00052C041F053C042F054C043F091ECCFF018
:10DE0000C7ECC5F0D6ECFBF03AC0EDFF39C0EDFF32
:10DE100038C0EDFF37C0EFFFC40E406E160E416EE6
:10DE2000020E426E06ECD1F048C149F0D4ECCDF0C0
:10DE3000C7ECC5F0ECECFCF03EC0EDFF3DC0EDFFE3
:10DE40003CC0EDFF3BC0EFFF0701305131113211F3
:10DE500033110EE0C80E305D000E3159000E3259FC
:10DE6000000E335905E230C700F0B1EC3AF005D0AE
:10DE700030C726F74E0E80ECC4F018A804D0A7ECEB
:10DE800069F018980AD00901EC5107E0D2ECC4F00F
:10DE900004E00BC0D5F20901ED6B209E33A403D042
:10DEA0008EEC39F005D0010EE66E1DEC39F0E5522E
:10DEB000229805ECC6F041EC25F0010136BF04D0F4
:10DEC000050EC7ECC6F00ED036AD0CD0DF85E3836F
:10DED000E395E3970601FB29FC6F65C3E6FF3BEC86
:10DEE0000AF0E552800E076E12002F50100B04E06E
:10DEF0000101E451080B13E00701555110E1010144
:10DF0000B151200B0CE13B51200B0AE0C3ECC5F0F2
:10DF100007E0A95105E10101E451080B01E1000C02
:10DF2000010C070EE66EE66A200EE66E440EE66E03
:10DF3000060EE66EA3ECFAF0050EE15E120045C691
:10DF400044F646C645F647C646F648C647F649C6AD
:10DF500048F64AC649F6120049C64AF648C649F686
:10DF600047C648F646C647F645C646F644C645F691
:10DF70000601200E446F12005FECC3F031AA02D0FC
:10DF800003ECCCF00101E151020B0CE0280E090179
:10DF9000BB5D08E2BB51BB2BEA6A930FE96E090E29
:10DFA0008FECD0F00101E451200B0CE0280E0901A8
:10DFB000E45D08E2E451E42BEA6ABC0FE96E090E65
:10DFC0008FECD0F05BEFC3F05FECC3F00101E4B77E
:10DFD00004D051ECCEF003D8E5525BEFC3F018EC5F
:10DFE000CEF0010EDB6A1A50010B0AE0800EDBEC6A
:10DFF000C3F004E2FE0EDB50200802E11A905CD070
:10E000009EDFFE0EDBCF4AF6DB50800804E0850E73
:10E01000DBECC3F003E30601200E21D0FE0EDB5043
:10E02000300803E10601630E1AD02950200B1CE0D2
:10E030002850080B19E1DF6A150EDF5C15E2A9EC28
:10E04000D1F00FE1DE52010EDD6EDF2AC1ECC6F029
:10E0500006014A6F74DFDF2AC1ECC6F006014A6F81
:10E0600003D0030EDF26E8D7C3ECC5F012E0010EA3
:10E07000DB5004E049C6E6FF7FDFE5524AC600F008
:10E08000630E005C02E1300E006E0050E66E74DF3D
:10E09000E5522BDF000910E03DECC8F044C616F154
:10E0A00045C617F146C618F147C619F148C61AF118
:10E0B00049C61BF14AC61CF1020EE15C02E2E16AAC
:10E0C000E552E16E5BEFC3F014ECCEF00750DF6E6B
:10E0D0002392100E075C13E11C0E076E02015151D2
:10E0E000010B03E11D50040B02E1110E92D05151BE
:10E0F000040B27E11D50080B01E0B3D022D0110E14
:10E10000075C09E12380228E0201080E516F2382F1
:10E11000076A120EA5D0120E075C06E12390238237
:10E12000030E076E130E9CD0130E075C0CE11C0E41
:10E13000076E02015151040B04E11D50080B01E070
:10E1400090D0140E66D0140E075C10E12380228E4E
:10E15000180E076E1D50040B01E083D01D50080BF4
:10E1600001E07FD02382076A150E7AD0150E075C76
:10E170000CE101012AAF03D00201020E516F229E71
:10E180002382020E076E160E6BD0160E075C05E199
:10E190002382020E076E170E63D0180E075C07E18C
:10E1A0000201020E516F2382076A190E59D0190E0F
:10E1B000075C06E1229E2382020E076E1A0E50D0E3
:10E1C0001A0E075C05E12382020E076E1B0E48D073
:10E1D000170E075C08E101012ABF03D00201020EFD
:10E1E000516F1B0E16D01B0E075C05E12390228E8B
:10E1F0002382030E33D01C0E075C33E12390800E84
:10E20000076E02015151010B03E11D50040B03E1A4
:10E21000110E076E26D034AC0BD038EC20F001087C
:10E2200002E1520E01D0500ECEECC3F0349C19D056
:10E230001750800B16E19AECC9F004E0090E0201B8
:10E24000535D0AE30601EA5104E0080E0201535D42
:10E2500003E302012D5105E02382080E076E100E24
:10E26000086E23A202D0CFEC64F0DF50075C01E01F
:10E270001C8CE5525BEFC3F01C9612000201566B3A
:10E28000E66AE66AE66A73ECC7F002012A6B0701E8
:10E29000A36B0B6A20B003D0208014EC6AF012004C
:10E2A00014ECCEF00201050E2D6F280E2E6FE6DF66
:10E2B000020E0A5C05E14BECCAF0140E85ECC3F0CB
:10E2C0000501040E266FE5525BEFC3F0348C0101AB
:10E2D000CC51400B02E1530E01D0510ECEEFC3F0F2
:10E2E0000101DF51020B18E03C51800B15E1205079
:10E2F000010B12E12550040B0FE12450020B0CE13D
:10E30000DF932F88070EE66ED00EE66E010E8FECBF
:10E31000C3F00101AA0EA86F1200E8ECCDF004E1F1
:10E320002050010B01E1000C010C01015651800B42
:10E3300005E0020E005C03E0000401E0000C010CAB
:10E3400014ECCEF0D4ECCBF005E04BECCAF0140E9C
:10E3500085ECC3F0209020940701A16B1FECD2F054
:10E36000E5525BEFC3F0D7ECD0F0800E491843E1E3
:10E370004A5041E10101DF9B199ED190FF0E05013A
:10E380004B5D04E04BC507F04B6912000101E1A5AC
:10E3900003D0E19529EC19F00101E151080B08E0E7
:10E3A0002050400B05E1120E01ECC4F00101E19791
:10E3B00034AC0AD038EC20F0010802E1520E01D052
:10E3C000500ECEECC3F0349C20B013D0D4ECCBF084
:10E3D00002E0006A78DB2196020168510AE13250BE
:10E3E000010B07E12C50800B04E12C50400B01E1A4
:10E3F0001F86072A120046ECCAF001E00FD24A50ED
:10E4000001E00CD220A0229CD9EC14F0FF0801E01E
:10E4100005D12050200B01E101D11850800B01E003
:10E42000FDD00201766B76C2ADF11992F6ECC6F022
:10E43000349C1C901E50010B06E01D50040B03E0A1
:10E440001D50080B0DE100500BE01F50020B08E0BF
:10E450006CDF000905E0258E1F0E0DECC4F0DED048
:10E460001E50010B18E1005006E01F50020B13E193
:10E470005CDF000910E00101010EAD6F1982076A2F
:10E480000B0E086E005003E148DF000901E01C801C
:10E4900000502CE12DD01D50040B03E01D50080B43
:10E4A00029E100500CE0D4ECCBF009E11F50020B45
:10E4B00021E18AECC4F003E138DF00091BE01DB460
:10E4C00002D0110E05D01DB604D00201516B140EFE
:10E4D000076E005003E121DF000901E01C800050BD
:10E4E00007E07DECC5F002E1DBDE98D0EFDE96D0F0
:10E4F000F7DE94D0050110511EE027AA12D000507B
:10E5000003E08AECC4F010E0005003E106DF0009EC
:10E5100001E01C80005001E1E3DE8AECC4F001E080
:10E52000BFDE1E0E076E7AD0258E8A0ED2ECC7F0A3
:10E53000A1EC21F073D020AE05D0076A0A0E086E58
:10E540001C806CD0005051E09CECC6F006E02050DE
:10E55000040B03E11E50020B48E00201195114E0C4
:10E560001E50020B07E1D8EC08F000090DE19CEC0D
:10E57000C6F00AE10201376B386B196B19C255F20C
:10E5800003EC0BF015EC65F08EECC4F00AE09CECAB
:10E59000C6F0FDE0D2ECC9F0FAE120941E928CEFB7
:10E5A00004F01C809AECC9F013E01950400B10E005
:10E5B0001950040B0DE020A40AD01994050EE66E44
:10E5C000D00EE66EE80E0C2485ECC3F001D01C9052
:10E5D0001CA024D0000E02012A6F0701A36F0B6E4E
:10E5E0001E92076A0B0E086E19D0005017E12050DA
:10E5F000010B14E19CECC6F003E02050040B0EE08C
:10E600000101DF938CEC04F08EECC4F005E09CEC8F
:10E61000C6F0FDE0209412001C8030DE2050200B5C
:10E6200004E1A8EC0BF0000903E1020134514DE0D4
:10E63000C3ECC5F04AE00501106B20902094810ED8
:10E64000076EFBEC04F0000906E1190EE66EC00E41
:10E65000E66E010E0DD09CECC6F002E11B0E12D04E
:10E66000D2ECC9F00AE0110EE66EC00EE66E010EA5
:10E670009EECD2F0E552E55208D0A8EC0BF0000970
:10E6800005E01A0EE66EBBEC26F0E552A8EC0BF0A6
:10E69000000919E0A8C134F2FBEC04F0000905E11F
:10E6A0000101806BCFEC04F00ED0D2ECC9F00BE08E
:10E6B000CCECCBF003E001013C9D02D001013B9F7B
:10E6C0000AEC19F01490D0EC07F046ECCAF001E126
:10E6D0004A5042E08CEC04F00201D95102E0D5EC42
:10E6E00008F00201D85102E067EC48F027AA28D0D0
:10E6F000CEECDAF002012A6B2FAA02D0D4EC4EF055
:10E7000030A402D063EC51F030AC02D0E2EC4FF018
:10E7100024A002D02DEC4FF032A002D063EC4FF0D9
:10E7200023AE02D067EC4EF01FA802D02AEC10F006
:10E730002C50800B03E12C50400B02E085EC0EF0D6
:10E74000259A1AAC02D0BCEC09F028A203D028927A
:10E750008EEC39F01C8C12002050010B14E00201E9
:10E760002D5111E11750800B06E013ECCBF009E0BE
:10E770000B0E155C06E02050040B05E19CECC6F086
:10E7800002E0A0EF71F002012A5104E01DECC9F093
:10E7900073ECC7F017AE5BD018EC97F0EDECC4F05B
:10E7A00017E02F50200B14E13050040B11E12350DF
:10E7B000800B0EE13050400B0BE12450010B08E1BF
:10E7C0003250010B05E13250020B02E164EC2EF0F5
:10E7D00032921FAA3CD01F9A01013BAB38D03DECCE
:10E7E000C8F00201315110E193EC34F0190E155CC0
:10E7F00014E11750010B11E00101D051D15D0DE181
:10E800000201C80E316F1200316B1C0EE66E84ECF3
:10E81000DAF0E5520101960EA86F120077ECC7F00E
:10E8200016E14A5014E121BA12D0C1EC07F00009F8
:10E8300002E180ECCDF04AEC0DF0238A810E076EE8
:10E84000C1EC07F0000903E064EC2EF02582120011
:10E850000C04040F0701006F12000101B19B19ACF9
:10E8600027D003EC0BF0138225A41CD0D8ECD3F0F6
:10E87000090EE66EC00EE66E010E0AECD0F0CAEC90
:10E88000D7F0E30E0C24CEECC3F010EC0BF0D8EC78
:10E89000D3F0010EE66EC00EE66E010E0AECD0F06B
:10E8A000CAECD7F002010E0E376F060E386F120059
:10E8B000CFDF0701FA0E036F016B026B0201536B8E
:10E8C000546B1D90120000C709F00201555104E07D
:10E8D000800E47ECC4F01A800701035117E0035182
:10E8E00003072FECC5F0CC0E005C10E0FF0E005CBF
:10E8F0000DE0800E005C06E20050E66E3CEC04F099
:10E90000E552006E005047ECC4F0E6D7096A1200E9
:10E9100026ECD3F0DBCF55F22F88006A2388A5ECD4
:10E9200026F00101320EA86F17A802D00201558F00
:10E930000201195102E0010E196F179E5BEFC3F03F
:10E9400017A802D0F7EC47F019AC24D003EC0BF079
:10E950001392FBECCFF0D00ED8800E54050E0F545E
:10E9600005E21BEC65F00201196B12001382010134
:10E97000E283218EE5EC0AF0198AD8EC08F0000950
:10E980000FE120840101E0999CECC6F009E001014F
:10E99000E0891200278A02012D5102E0010E2D6F3D
:10E9A00012005FECC3F0198C12ECC4F003E08AECA7
:10E9B000C4F001E0199C25A410D0FE0EDB500C6EB3
:10E9C0004CDF25940101B187239C24B2238C24823F
:10E9D00019AC32D0198428802FD01950400B0EE08A
:10E9E000D8EC08F000090AE09CECC6F007E02050E3
:10E9F000040B04E11D0E0DECC4F01ED0FD0EDB5027
:10EA00000DE10201195103E12750400B07E051ECE1
:10EA1000CEF07EDFE5520201196B0ED0FE0EDB5008
:10EA20000C6E1BDF19BC07D04EDF0501105103E14E
:10EA30001BEC65F001D084DF5BEFC3F00601060E2E
:10EA4000406F0701BEA902D006014007D5ECC7F010
:10EA500004E2A45102E00601402B02011E0E276FC2
:10EA6000120001012951E8240301B86F0A01190EAF
:10EA7000D76F360ED66F0101D05103E0030ED05D83
:10EA800003E10A01080ED66F07ECCBF003E10A019F
:10EA90003C0ED66F0A01DA8FD46B3484B5EFC5F023
:10EAA0005FECC3F01CEC39F076EC19F0338851ECD4
:10EAB000CEF05AEC1BF0E5525BEFC3F0010EE66EB0
:10EAC000EFDFE5521200000403E15EECD0F01BD052
:10EAD000005045E0030E005C18E15EECD0F0DAEC8B
:10EAE000C9F004E0E80E0E6E030E0F6EF2ECC6F0F5
:10EAF00004E06AEC04F029ECC4F02EECC4F003E16D
:10EB0000640E0E6E0F6AE2EFD1F043EC15F0930E37
:10EB10000E6E020E0F6E0050030819E2700E0E6E9C
:10EB2000030E0F6E050E005C04E1930E0E6E020ED6
:10EB30000F6E060E005C04E1970E0E6E040E0F6E53
:10EB4000070E005C04E1200E0E6E060E0F6EE2EC66
:10EB5000D1F0020E005C05E1500E9EECC3F0BCEF5C
:10EB60000AF00050030803E20201040E356F070E9D
:10EB7000005C03E10201080E356F12005FECC3F088
:10EB8000280E8BECCEF0290E01ECC4F05BEFC3F045
:10EB9000D9CFE6FFE1CFD9FFE6528C9E00000000FE
:10EBA000000000008C9600000000060EE66E2DECC2
:10EBB0005CF0E5528C860000000000008C9600009E
:10EBC0000000D80EE66E2DEC5CF0E552A5C7E6FF1E
:10EBD0002DEC5CF0E552E66A2DEC5CF0E552E66A5D
:10EBE0002DEC5CF0E5528C868C8EDF6A1E0EDF5CAD
:10EBF00007E2640EE66E8CEC21F0E552DF2AF6D7D0
:10EC0000E552E552E7CFD9FF1200D9CFE6FFE1CFB9
:10EC1000D9FF8C9E00000000000000008C960000D0
:10EC20000000030EE66E2DEC5CF0E552A5C7E6FF92
:10EC30002DEC5CF0E552FC0EDBCFE6FF2DEC5CF03A
:10EC4000E552FB0EDBCFE6FF2DEC5CF0E552FA0E51
:10EC5000DBCFF3FFDB06F35000090FE090ECFDF093
:10EC6000006EFD0EDBCFE9FFDB2AFE0EDBCFEAFFF5
:10EC700001E3DB2A00C0EFFFEAD700008C86C69EC6
:10EC80008C8EE552E7CFD9FF120018ECCEF0DF6A88
:10EC9000DF2AFA0EDBCFE6FF24ECC9F056ECC7F012
:10ECA0002BECC9F0FA0EDBCFE6FF24ECC9F0A80E7E
:10ECB000E66E030EE66E2BECC9F0010EDB6AFA0E6F
:10ECC000DB50A7ECC5F017E2010EDB50E76E79ECE4
:10ECD000C6F0E75038ECCFF0EFCF49F0010EDB5033
:10ECE000EA6AA80FE96E030EEA22EF50495C03E1DD
:10ECF000010EDB2AE4D768ECCCF002E037EC0DF033
:10ED000068ECCCF003E00A0EDF5CC2E30A0EDF5CC5
:10ED100002E3000E01D0010EBCECCBF002E2E16A8E
:10ED2000E552E16E49505BEFC3F0D9CFE6FFE1CF8A
:10ED3000D9FF8C9E00000000000000008C960000AF
:10ED40000000060EE66E2DEC5CF0E5528C860000AD
:10ED5000000000008C9600000000020EE66E2DEC14
:10ED60005CF0E552A5C7E6FF2DEC5CF0E552FE0E27
:10ED7000DBCFE6FF2DEC5CF0E552FD0EDBCFE6FFCE
:10ED80002DEC5CF0E552FA0EDBCFF3FFDB06F3501F
:10ED9000000911E0FB0EDBCFE9FFDB2AFC0EDBCF25
:10EDA000EAFF01E3DB2AEF50006E0050E66E2DEC27
:10EDB0005CF0E552E8D700008C86C69E8C8E050E6E
:10EDC000E66E8CEC21F0E552E552E7CFD9FF120058
:10EDD000D9CFE6FFE1CFD9FFE6525BEC5CF0010151
:10EDE000640EA86F0400B7EC41F0020E07015A5DF3
:10EDF0000FE00701945109E0A1EC05F00401FD6F5B
:10EE0000FDC4E6FFC4EC05F0E5529DECA7F071D01F
:10EE1000070194516EE007019451496E4A6A4A34E1
:10EE200004E24950C008000E4A5408E20701040EEB
:10EE3000266F270EE66E9AEC14F0E552A1EC05F071
:10EE40000401FD6F3B0E0401FD5D0CE104013B0E6E
:10EE5000FE6F0601C46B309A0101379BB6EC0CF0D3
:10EE600007015A6B610E0401FD5D07E30401FD51CA
:10EE7000660803E3200E0401FD5F300E0401FD5D12
:10EE800022E30401FD5146081EE30601C42B410E96
:10EE90000401FD5D04E2300E0401FD5F06D0410E69
:10EEA0000401FD5D0A0F0401FD6F020E0601C45D41
:10EEB00008E10601C339F00B0401FD250401FD6FD3
:10EEC00002D0FDC4C3F6020E0601C45D11E1FDC40B
:10EED000E6FF11EC0DF0E552006E010EE66E8CECD3
:10EEE00021F0E5520601C46B0050E66E47DEE552A4
:10EEF0008FD70201685102E076EC8EF01C9C100E58
:10EF0000075C03E2C7EC6BF024D01E0E075C03E243
:10EF100064EC70F01ED00750496E4A6AD8904A508F
:10EF200004E6800E495C000E4A5803E2CCEC21F066
:10EF300010D00750496E4A6AD8904A5004E6920EA3
:10EF4000495C000E4A5803E2B3EC71F002D066EC63
:10EF50002DF01CBCD3D745EC53F0095008E0070155
:10EF6000070E266F270EE66E9AEC14F0E55222A2E9
:10EF700028D022922E98329AEDEC80F0DF682E5045
:10EF8000100B15E0010101012A51040B10E1295079
:10EF9000020B0DE1DF500BE00D5002E1010E0D6E92
:10EFA0002E9831EC8EF0EDEC80F0DF06E8D7DF50E4
:10EFB00008E10701050E266F270EE66E9AEC14F0A5
:10EFC000E55210D7E552E552E7CFD9FF1200010113
:10EFD000E2A507D0D00501E1020C020ED05D01E1EF
:10EFE000010CD0511200080E016E0101D05102E156
:10EFF000180E016E370EB55D09E1016A83EC0BF066
:10F00000000902E0100E016E1FEC19F01200200E34
:10F01000E66E640EE66E070EE66E800E03EFCFF02E
:10F0200026ECCFF082ECC8F0EFCFDFFFFF0EDF5C05
:10F0300002E1100EDF6EDF50E5525BEFC3F0D3DF6D
:10F0400003015E51012601501EECCDF0046E12004A
:10F050003DECC8F00101040E016F0450006E005039
:10F060000F0803E2100E005E04D0100ED88000548A
:10F07000006ED7ECD9F00101200E1A6F050E006E5C
:10F08000300E1B5D02E0040E006E04500F0805E216
:10F090000050D5ECC4F02B0E04D00050D5ECC4F0D9
:10F0A0002D0EEF6E010E016FE60E496EF30E4A6EE5
:10F0B000010E4B6E5EC34CF04D6A4E6A00ECCEF012
:10F0C000A3ECCEF00101188F12001C0E0101B55DFA
:10F0D00001E1010C000C14ECCEF00050EF085CE2F2
:10F0E000F00E005CDF6EDF50080862E32950010B70
:10F0F00005E10401F95102E1FA5108E00101E09152
:10F100000201246B3C6B9DECA7F0F0D73DECC8F0FE
:10F11000DEECC9F0DF50FE0BE842750F096E016AA4
:10F12000DFA002D0800E016E026A070E025C0CE2C4
:10F13000F4EC3AF0005008E0FF0E005C05E068ECEB
:10F14000DAF0012A022AF1D7CAECD7F00101E085F2
:10F15000080E016EDFA002D0800E0126026A780E32
:10F16000025C10E2F4EC3AF000500CE0FF0E005CA0
:10F1700009E00050036EE66EC4EC05F0E552012A8A
:10F18000022AEDD73B0E035C05E03B0EE66EC4ECB5
:10F1900005F0E552096A16D06FECCCF000501FEC78
:10F1A000CEF0056EFF0E055C05E16C0E7CECC4F044
:10F1B000258E08D0B5C157F205C0B5F129820201EC
:10F1C000010E686FE5525BEFC3F01C0E0101B55DE7
:10F1D00004E1F00E03015D2513D00068016A0150BF
:10F1E000F0ECC3F004E6960E495C000E4A580CE2BF
:10F1F0006FECCCF001501FECCEF0B55D03E1015097
:10F20000006E1200012AEBD71200020E016E2AC115
:10F2100000F0B1EC3AF02F0E016E57C100F0B1ECE6
:10F220003AF0370E016E5FC100F0B1EC3AF00F0E0C
:10F23000016E37C100F0B1EC3AF0100E016E38C12A
:10F2400000F0B1EC3AF02E0E016E56C100F0B1ECB8
:10F250003AF0620E016E8AC100F0B1EC3AF0650E30
:10F26000016E8DC100F0B1EC3AF0660E016E8EC1F8
:10F2700000F0B1EC3AF06E0E016E96C100F0B1EF05
:10F280003AF0130E016E3BC100F0B1EF3AF03E0EC2
:10F290000101B55D02E119A6CD7B160EB55D14E145
:10F2A00019A63B79C4EC1EF064EC2EF0C8ECCBF050
:10F2B00004E02150020B01E1E4893BB903D01E9A1E
:10F2C000B5ECC5F0050147873D0E0101B55D09E1CB
:10F2D00019B607D0020E425D02E1010E01D0020E06
:10F2E000426F050EB55D03E0060EB55D11E119B67E
:10F2F00008D0050EB55D03E10701BE7102D007011C
:10F30000BE73D9ECCAF074EC09F0020107812D84B8
:10F31000280E0101B55D04E119A677717FEC20F09C
:10F32000210E0101B55D02E119A68D790F0EB55DC3
:10F3300004E119A63E7104EC5CF0270E0101B55DF5
:10F340000AE119A638754FECCDF001E0098F08EC01
:10F35000F7F08EEC39F0100E0101B55D02E119A64F
:10F36000CE7B180EB55D02E119A6387F090EB55D9A
:10F3700002E119A6967DB55104E119A6337431EC6A
:10F380001FF0310E0101B55D02E119A62A752C0EA0
:10F39000B55D02E119A62A731A0EB55D01E12E745E
:10F3A0002F0EB55D01E12E723F0EB55D02E119A68B
:10F3B0003771120EB55D02E119A62A7F2E0EB55DDA
:10F3C0000CE119B608D05F9FFD0EE66EBF0EE66E2B
:10F3D000010E8FECC3F07FEC20F012004DECD3F067
:10F3E000FB0EDB50D880DF5403E2FB0EDB50DF6EF8
:10F3F000FC0EDB50DF5C03E2FC0EDB50DF6E0DAE7B
:10F400000CD0FC0EDB50D880DF5402E2DF0605D0C2
:10F4100032B603D0FB0EDB50DF6E0D040BE1FB0EAA
:10F42000DB50DF5C02E2DF2A05D032B603D0FC0EEF
:10F43000DB50DF6EE8EFD1F02DECD0F032ECC9F00C
:10F440005BEFC3F05FECC3F0328624ECC9F056ECFE
:10F45000C7F032ECC9F032965BEFC3F02DECD0F080
:10F46000C0ECD3F05BEFC3F04DECD3F076ECCCF016
:10F47000E8AE02D0493403D0E750D880495403E2C3
:10F48000FB0EDB50DF6E7DECCCF0E8AE02D0E73453
:10F4900002D0E750495C03E2FC0EDB50DF6E0DAE9C
:10F4A0000BD07DECCCF0E8AE02D0493403D0E7506D
:10F4B000D880495401E2DF060D040AE176ECCCF075
:10F4C000E8AE02D0E73402D0E750495C01E2DF2A1F
:10F4D000E8EFD1F0500E036EB3ECCEF005E01B5018
:10F4E000080B02E11E0E036E120014ECCEF0CFDE0C
:10F4F000300E0101B55D2AE13651070B006E0D0497
:10F500000EE136BF02D0368F1AD036BD03D0368D0D
:10F51000006A15D0070E005C12E2002A10D0FF0E20
:10F520000D5C0DE1005005E0000600AE08D0006A59
:10F5300002D036AD02D0369D02D036BF369F005085
:10F54000070BF36EF80E3615F310366F1E0EB55D11
:10F550001DE1D05103E0CCECCBF003E0D1EC0BF09B
:10F5600015D00D0409E1010156B102D056810ED02B
:10F5700056B50CD056850AD0FF0E0D5C07E101018F
:10F5800056A502D0569502D056B156910C0E0101E7
:10F59000B55D0BE1150EE66E030EE66E550EE66EDA
:10F5A000010E98ECC3F08CEC04F00D0E0101B55D7A
:10F5B00008E1050EE66E830EE66E010E93ECC3F0D5
:10F5C000339C0B0E0101B55D15E1020EE66E840E53
:10F5D000E66E010E93ECC3F0300E010184250401A8
:10F5E000F76F020E0101845D03E10401340EF76F31
:10F5F0006EECA7F0220E0101B55D11E1030ECC15F2
:10F60000066F065102E1010E066F030E54ECD3F0B3
:10F61000FC0E0101CC170651CC137FEC20F02B0E11
:10F620000101B55D07E119A6CE711E9AB5ECC5F0D2
:10F6300064EC2EF0110E0101B55D2EE10D0411E117
:10F64000080E505D02E10D0E26D0050E505D1EE045
:10F65000030E505D16E050050FE00D0E505D1CE0EE
:10F6600006D0FF0E0D5C18E1030E505D02E1010EA5
:10F6700012D0050E505D02E1030E0DD0080E505D54
:10F6800002E1050E08D00D0E505D02E1080E03D018
:10F69000500502E0010E506F230EB55D2DE1E3AB86
:10F6A00003D0D1EC0BF028D0640E006E0701BEAB86
:10F6B00002D00A0E006E0D0409E1000100500101A4
:10F6C0006927000E6A236B236C2310D0FF0E0D5C9C
:10F6D0000DE10050496ED4ECCDF049500101695F55
:10F6E0004A506A5B4B506B5B4C506C5B34ECF3F0F4
:10F6F000248433888EEC39F0130E0101B55D0BE1E3
:10F70000030E4F15066F020E05ECD3F0FC0E01013F
:10F710004F1706514F13140EB55D11E1300E4F1502
:10F72000066F06390F0B066F020E05ECD3F00101D0
:10F730000639F00B066FCF0E4F1706514F130E0E02
:10F74000B55D09E1820EE66E520EE66E510EE66E72
:10F75000010E98ECC3F03C0E0101B55D19E1070103
:10F76000BE51E840E8403F0B0101066F030E06174B
:10F7700005ECD3F00101040E0603F3CF06F1F30EFE
:10F780000701BE17010106510701BE1374EC09F011
:10F79000420E0101B55D13E1E2A508D0B40EE66E9C
:10F7A000640EE66E4A0EE66E010E07D0730EE66E2C
:10F7B000460EE66E520EE66E010E98ECC3F0E4ECD7
:10F7C000CBF033E12050040B30E00D0414E12B505A
:10F7D000040B02E0140E01D0010E496E4A6A49BEC4
:10F7E0004A682250040B01E0010EE3ECC6F04950D8
:10F7F000EE264A50ED22FF0E0D5C14E12B50040B57
:10F8000002E0140E01D0010E496E4A6A49BE4A68F0
:10F810002250040B01E0010EE3ECC6F04950EE5E0D
:10F820004A50ED5AE8EC15F01E88340E0101B55D22
:10F8300007E11B0EE66ED80EE66E010E5AECC6F01E
:10F84000390E0101B55D26E133A608D0F30EE66E50
:10F85000D70EE66E010E5AECC6F005D02B510A0801
:10F8600002E2D1EC0BF064ECC2F0E66E73EC13F044
:10F87000E552D2ECC4F00CE100C006F1C80E54EC25
:10F88000D3F006C100F0B1EC3AF049ECC5F002D07B
:10F89000D1EC0BF0170E0101B55D20E1DFAD12D008
:10F8A0000C0EE66E030EE66EB4ECCDF004E1950EA0
:10F8B000496E010E03D0930E496E010E4A6EA1EC03
:10F8C000C4F008D0780EE66E280EE66E870EE66E5F
:10F8D000010EE66EC0ECD3F00BEC09F0240E010132
:10F8E000B55D07E1FA0EE66E880EE66E020E93EC49
:10F8F000C3F0190E0101B55D07E1020EE66E700E50
:10F90000E66E020E93ECC3F0200E0101B55D1CE122
:10F91000020EE66E390EE66E010E93ECC3F00101A5
:10F92000395104E19BECD2F041EC25F088ECC8F0B1
:10F93000006A0101395102E0010E006E00C0D4F2EC
:10F9400000C0D3F200C0EBF9B50507E1050EE66E85
:10F95000940EE66E010E93ECC3F00A0E0101B55D44
:10F9600001E086D039512CE030A227D00901E851BE
:10F9700004E10D0401E07AD016D0E80511E10D0490
:10F9800008E1010EE86FF10EE66EBF0EE66E010EA5
:10F9900011D0E86BEB0EE66EBF0EE66E010E0AD0DC
:10F9A000FF0E0D5C63E1010EE86FF70EE66EBF0E11
:10F9B000E66E010EC4ECC3F059D0D1EC0BF058D078
:10F9C0001E862950020B0AE03A5108E03A5101081C
:10F9D00002E2010E01D0020E3A6F07D0130EE66E5E
:10F9E0003A0EE66E010E93ECC3F05AEC09F00101F9
:10F9F0003A5102E08D8303D03A5101E18D93030E19
:10FA00003A5D34E33A51130831E3000E036E026E9F
:10FA1000016E030E3A5D006E080E005C0BE2010EF3
:10FA200000C0E7FFE75204E0E846FE0BE706FCE112
:10FA3000016E12D0100E005C0CE2080E005C496EE4
:10FA4000010E495204E0E846FE0B4906FCE1026E55
:10FA500003D0100E005C036E010EE66E0350E66EDE
:10FA6000025097ECC7F03DECC7F002D023ECBDF09C
:10FA7000030E0101B55D0BE11E0EE66E010EE66E92
:10FA8000700EE66E010E98ECC3F02FEC1FF0070E1F
:10FA90000101B55D4FE1E55109E1080EE66E040E86
:10FAA000E66E470EE66E010E98ECC3F00101E50527
:10FAB00008E1E668C80EE66E7D0EE66E010E98EC73
:10FAC000C3F0020E0101E55D08E1C80EE66EE66ACC
:10FAD0004B0EE66E010E98ECC3F0030E0101E55DDE
:10FAE00013E10701BEA308D0960EE66E780EE66E0F
:10FAF0004D0EE66E010E06D0320EDCECCBF04C0E55
:10FB0000E66E010E98ECC3F0040E0101E55D08E11C
:10FB10000F0EDCECCBF0410EE66E010E98ECC3F05C
:10FB2000050E0101E55D04E119A662733DEC1EF0CE
:10FB30002FEC1FF0290E0101B55D3AE1016AD051A9
:10FB400002E0010E016E020E0901E55D1BE13CECD5
:10FB5000CFF00AE17FECCFF004E6E20E495C000E44
:10FB60004A5802E2190E0026FF0E0D5C05E1005016
:10FB7000180802E2190E005E0150F5ECC3F000C057
:10FB8000EFFF14D0020EE55D11E2FA0EE66E010EF3
:10FB9000E66E0150030D15ECC6F0B80E4B26020EB2
:10FBA0004C22E55135ECD0F0C0ECD3F025EC4EF012
:10FBB000330E0101B55D07E1640EE66E850EE66E5B
:10FBC000010E93ECC3F0040E0101B55D09E1020ED4
:10FBD000E66E310EE66E010E93ECC3F0C4EC1EF03F
:10FBE000360E0101B55D10E12B510A0806E20F0E39
:10FBF000E66E7B0EE66E010E05D00F0EE66E860EEB
:10FC0000E66E010E93ECC3F03A0E0101B55D0CE116
:10FC10001FEC19F0190EE66EE66A7A0EE66E010E1A
:10FC200098ECC3F0B3EC15F0380E0101B55D0BE1B3
:10FC3000280EE66E1E0EE66E890EE66E010E98EC3C
:10FC4000C3F0EBECCBF0400E0101B55D09E13C0ED9
:10FC5000E66E6E0EE66E010E93ECC3F00AEC19F040
:10FC6000410E0101B55D09E13C0EE66E6F0EE66ED8
:10FC7000010E93ECC3F00AEC19F0320E0101B55DF0
:10FC800028E181C306F13B0E016E03017F5104E1BF
:10FC900080C306F1170E016E020E7F5D02E182C382
:10FCA00006F101506EECCEF074ECC6F003017F510A
:10FCB00002E106C180F37F0502E106C181F3020E75
:10FCC0007F5D02E106C182F30101835102E0D9ECBC
:10FCD000DBF0080E0101B55D16E103017F5107E17C
:10FCE000170EE66E830EE66E030E74ECC6F003018B
:10FCF0007F0507E13B0EE66E840EE66E030E74ECA4
:10FD0000C6F0E2ECDBF0020E0101B55D0EE11B5026
:10FD1000080B02E0060E01D0050EE66E800EE66EC0
:10FD2000010E93ECC3F0CFEC04F0E0ECCDF02CE14D
:10FD3000016AD5CA03F0CE51010B12E03751080B0E
:10FD40000FE0040E036E1BA00BD0030E036E010E1A
:10FD5000016E0A011C5104E1280E216F21CA1CFA10
:10FD6000FE0E97ECC7F005011751050D15ECC6F016
:10FD7000140E4B260A0E4C22035035ECD0F032EC18
:10FD8000C9F02484B4EC0DF03B0E0101B55D0FE128
:10FD9000FA0EE66E2250040B01E0010E4A6A910F42
:10FDA000496E020E1EECD0F0E8EC15F01E88260E0F
:10FDB0000101B55D03E0370EB55D1BE1030ED05DBB
:10FDC00003E1D1EC0BF015D0D0ECCDF01FEC78F0C6
:10FDD00004C006F1200E05ECD3F0015082ECC8F00F
:10FDE00006C1EFFF308E06C104F028EC78F035EC48
:10FDF0001EF01D0E0101B55D0EE1D05103E0030EB2
:10FE0000D05D03E1D1EC0BF006D019B602D00201AF
:10FE10007879DDEC15F0250E0101B55D09E1030EE1
:10FE2000E66E430EE66E010E93ECC3F054EC21F047
:10FE30001B0E0101B55D0FE13EC1DFFF188C3E6B6B
:10FE4000070EE66E3F0EE66E010E93ECC3F084ECF7
:10FE5000CDF0DFCF3EF11F0E0101B55D02E10D5087
:10FE60003327150EB55D09E10C0EE66E070EE66E42
:10FE70003D0EE66E010E98ECC3F05CC3E6FF1FEC8E
:10FE80000CF0E552430E0101B55D14E119B611D035
:10FE900094ECD3F0040A01E0010E496E8AECC3F041
:10FEA0004950010BF36EF346F346FB0EEF14F310CB
:10FEB000EF6E2E86440EB55D32E1ABECD0F0016EF4
:10FEC000B5ECCFF0026E0D50022602AE0ED0630EDE
:10FED000026E01060150CEECC4F007E24950F90869
:10FEE000000E4A5402E2F90E016E0250630802E26B
:10FEF000026A012A0150CEECC4F006E24950F9082A
:10FF0000000E4A5401E2016A8AECC3F0030E01C0FC
:10FF1000EBFF8AECC3F0020E02C0EBFF2E86450E0B
:10FF2000B55D1BE1A6ECD0F0016E0D50E824012672
:10FF300001500A0802E20A0E016E080E015C02E19D
:10FF4000090E016E030E015C02E2030E016E8AECE3
:10FF5000C3F0010E01C0EBFF2E86470EB55D50E1E8
:10FF60003AECD2F0496E4A6A35ECD2F00A0DF35001
:10FF70004924D66FF4504A20D76F3FECD2F002E10B
:10FF8000DDECCAF00D040CE1D890D75104E6E70E81
:10FF9000D65D030ED75911E2D62B000ED7230DD014
:10FFA000FF0E0D5C0AE1D73504E3D6511908FC0EAB
:10FFB000D75503E2D607000ED75B2888800ED715E9
:10FFC00003E02898DDECCAF0D6C149F0D7C14AF069
:10FFD0000A0E79ECC3F08AECC3F0040E49C0EBFFC3
:10FFE0008AECC3F0050E39C0EBFF8AECC3F0285051
:10FFF000100B02E0EF8001D0EF902E8664EC2EF023
:020000040001F9
:10000000460E0101B55D3FE18AECC3F0060EEB50F0
:10001000006E8AECC3F00490EF50020B01E0048004
:100020000D500026005006E1047004806AEC7AF05E
:100030000350006E6AEC7AF00350D880005404E25A
:1000400004700480010E006E2FECCFF001E00490EC
:1000500004808AECC3F00450010B02E0EF8201D06F
:10006000EF928AECC3F0060E00C0EBFF100E010108
:100070002B5D03015C5D06E100C048F149ECC5F071
:100080005CC300F02E86480E0101B55D39E1049095
:100090002FECCFF001E004808AECC3F0EF50016E4A
:1000A0000F0E0114006E01380F0B016E0D5001266A
:1000B00004A00CD00150800803E2090E016E0490E8
:1000C000015009080CE2090E016E09D0015002E14D
:1000D000010E016E0150090802E2016A0480013834
:1000E000F00B016E01500012D0ECD1F0090E38EC8B
:1000F000CFF00450010B02E0EF8E01D0EF9E2E8670
:10010000E5525BEFC3F05C0E002456ECD2F0010127
:10011000100E136F145102E1100E146F1200B5ECA3
:10012000CFF0D9ECC7F0ABECD0F0006E0101030EBC
:10013000006FBAECD9F0060EE66E030E8EEFC8F033
:1001400035ECCEF00A0809E2FE0EDB50F00F006E2F
:10015000005034ECC8F0E3DF23D0FE0EDB50006E1D
:10016000D2DF020EDBECC3F00DE20101010E146FD1
:10017000080E156FFE0EDB040DE1030E146F050E65
:10018000156F08D013C112F114C113F115C114F188
:100190000101156BC8ECCDF002E1090E156F158F4A
:1001A0005BEFC3F0CCEC25F02E801200140E006E35
:1001B00004A002D0110E006ED2EF80F00E0E006E81
:1001C00004A002D0080E006ED2EF80F0DBEC11F03C
:1001D000D0C7F3FFD1C7F4FF120030ECD2F0010119
:1001E000B151800B04E02F50100B01E1DFD0D8ECAF
:1001F000D3F049EC8DF0010139510DE00A0EB55DE7
:100200000AE1016BE30EE66EBF0EE66E010E0AEC2C
:10021000D0F00101198F070EB55D49E1040E016FA1
:100220002A0E196FE55108E1DF0EE66EBF0EE66E8D
:10023000010EE66EECECC3F00101E50508E1DB0E12
:10024000E66EBF0EE66E010EE66EECECC3F0020E3B
:100250000101E55D08E1D70EE66EBF0EE66E010E08
:10026000E66EECECC3F0030E0101E55D08E1D30E90
:10027000E66EBF0EE66E010EE66EECECC3F0040E09
:100280000101E55D08E1CF0EE66EBF0EE66E010EE0
:10029000E66EECECC3F0050E0101E55D08E1CB0E66
:1002A000E66EBF0EE66E010EE66EECECC3F0290EB4
:1002B0000101B55D0FE1420E1C6F0901E50503E187
:1002C0000101440E1C6F020E0901E55D03E101010D
:1002D0004D0E1C6F340E0101B55D11E10201B051EC
:1002E0000EE0D8ECD3F0C40EE66EBF0EE66E010E43
:1002F0000AECD0F02CA203D00101370E1B6FE0EC0A
:10030000CDF007E13751080B04E04C0E1B6F2A0EAD
:100310001C6F230EB55D0CE196A302D0230E07D00F
:1003200057A906D02A0E196F57BB02D03F0E196F7E
:100330001FA805D0D8ECD3F0006AE1EC25F089ECD9
:1003400063F0000905E0310E03015C250101186F1F
:100350001C0E0101B55D05E1310E03015D250101B2
:100360001C6F260EB55D03E0370EB55D05E1310E5D
:1003700003015E2501011C6F420EB55D0CE1E251E7
:10038000040B09E0016BBC0EE66EBF0EE66E010EBB
:10039000E66EECECC3F0170E0101B55D07E1DF512D
:1003A000400B04E0500E166F4C0E176FC8ECD3F0E4
:1003B000DEECD0F00E0E136F146F65EC78F00009D0
:1003C00007E00101006B280EE66E5EECDAF0E55204
:1003D000016A400E0101B55D08E16EC100F00168DF
:1003E00002016E0EA46F010EA56F410E0101B55DF5
:1003F00008E16FC100F0016802016F0EA46F010EE9
:10040000A56F1F0E0101B55D08E10201330EA46F57
:10041000010EA56F33C100F00168150E0101B55D35
:100420000BE1050E3D03F350410F006E0168020120
:100430003D0EA46F010EA56F1B0E0101B55D08E115
:100440003F29006E016802013F0EA46F010EA56FE7
:10045000170E0101B55D26E18751FE0BE842006EE3
:100460000201870EA46F010EA56F0101DFAD18D048
:1004700093C100F00201930EA46F010EA56F330E1D
:10048000875D0AE101019551FE0BE842006E020111
:10049000950EA46F010EA56F050E0002F3CF00F0BC
:1004A00001682E88070E0101B55D65E1E55106E1A1
:1004B0000201470EA46F010E95ECC4F00101E505A1
:1004C00006E102017D0EA46F010E95ECC4F0020E50
:1004D0000101E55D06E102014B0EA46F010E95ECF2
:1004E000C4F0030E0101E55D1DE1006B0701BEA331
:1004F0000CD0B80EE66EBF0EE66E010E80ECC3F0B7
:1005000002014D0EA46F010E0BD0B40EE66EBF0EAD
:10051000E66E010E80ECC3F002014C0EA46F010EDA
:1005200095ECC4F0040E0101E55D06E10201410E07
:10053000A46F010E95ECC4F00168050E0101E55DA4
:1005400017E1016A62A306D0B00EE66EBF0EE66E3A
:10055000010E05D0AC0EE66EBF0EE66E010E80EC0D
:10056000C3F00201620EA46F010EA56F020EA66F0A
:100570000101050E006F290EB55D1CE1026AD05124
:1005800002E0010E026E0250030DAAECCEF0B80E8E
:100590004926020E4A220901E55114ECD1F0020E5F
:1005A0000901E55D05E1190EAFECCEF04FECC7F0A7
:1005B00001682E883C0E0101B55D0AE1D0C1E6FF5D
:1005C00051EC0DF0E552016886ECCAF00C0EA66FF6
:1005D000015002E0BAECD9F0150E0101B55D09E059
:1005E000170EB55D08E1DF51400B05E0B4ECCDF02E
:1005F00002E00101148F3C0E0101B55D09E0170E08
:10060000B55D0CE1DF51400B03E0B4ECCDF006E149
:100610000101135102E1100E136F158F0C0E010131
:10062000B55D1FE1150E555D0BE1006BA30EE66E87
:10063000BF0EE66E010EE66E58ECDAF0E5520AD017
:1006400055C100F0BAECD9F0060EE66E050EE66E66
:1006500021EC09F0E552E5520201550EA46F010E9E
:10066000A56F3E0E0101B55D10E1CDAB02D0080EC5
:1006700001D00E0ECEECC6F02E800201CD0EA46F7E
:10068000010EA56F200EA66F2E88050E0101B55D27
:100690000DE10701BEB102D00E0E01D0080ECEEC66
:1006A000C6F086ECCAF0010EA66F2E80060E010180
:1006B000B55D17E10701BEB306D0B40EE66EBF0EFE
:1006C000E66E010E07D0010100079E0EE66EBF0E1A
:1006D000E66E010E80ECC3F086ECCAF0020EA66F47
:1006E0002E800101B5052EE10B0ECEECC6F0010106
:1006F000945106E1010E006F440E006ECCEC25F023
:1007000001019451010819E2006B950EE66EBF0ECF
:10071000E66E010E80ECC3F0050E0101945D02E16E
:10072000158F0BD0050E006F9405190DF350D9EC01
:10073000C7F00101100E136F148F0201940EA46F05
:10074000010EA56F100E0101B55D1EE12BC1E6FF84
:10075000F7DCE55212C10EF113C10FF114C110F113
:1007600015C111F10101100E126F050E006FCEAB15
:1007700002D0290E01D02A0EE66E5EECDAF0E552C8
:100780008CECCAF0200EA66F2B0E0101B55D1AE1AC
:10079000E4ECC5F0DEECD0F00B0ECEECC6F00101BF
:1007A000CEA10BD0050E006F910EE66EBF0EE66E69
:1007B000010E80ECC3F00101158F8CECCAF0010E24
:1007C000A66F2E88220E0101B55D20E1E4ECC5F094
:1007D0000101030E006F8B0EE66EBF0EE66E010E7A
:1007E00080ECC3F00101CC51010B05E0CC51020BB0
:1007F00002E0030E03D0CCA302D0020E126F02015E
:10080000CC0EA46F010EA56F030EA66FE4ECCBF027
:1008100029E12250040B01E0010E010F0E6F030EBF
:10082000006F04902250040B01E0010EE3ECC6F0CF
:10083000EECF0EF0EDCF0FF058EC26F00101100EC8
:10084000116F2BB4156F2250040B01E0010E020D45
:10085000F3CFF3F6F4CFF4F68D0E0601F327020E74
:10086000F4232E88340E0101B55D01E019D124B8BE
:100870000CD0006B4DEC64F0D9ECC7F0DEECD0F09E
:1008800056EC64F0D9ECC7F00AD154EC10F021EC2E
:10089000C8F054EC10F00E500101D4270F50D523AE
:1008A000D4C10EF0D5C10FF0010E0F0B04E00BEC1C
:1008B000CBF0E806FCE107010E500C5D0F500D591E
:1008C00005E20C510E5E0D510F5A02D00E6A0F6AEE
:1008D0000EC00EF70FC00FF70201B0511CE0190E49
:1008E000AFECCEF0B0C23EF0A0ECCBF004E17EEC79
:1008F00004F00201B16FB1C200F00101126BBEEC55
:10090000D0F017ECFEF03EC013F13AC014F1010133
:10091000110E156F138F4DEC64F0026E006E2CA259
:1009200004D056EC64F0026E006E0201B05157E044
:10093000960E0101D46FD56B1FA003D0F00ED46FBB
:10094000D56BD0ECCBF004E0320E0101D46FD56B47
:100950000101D4510E5CD5510F5810E27FECCFF05D
:1009600004E6F00E495C000E4A5808E2002A640EC4
:100970000201B05D1DE2190EB0271AD00C0E4A6AB2
:10098000D425496ED5514A2294ECD0F005E20050AE
:10099000640802E200060CD00201B051CEECC4F0B3
:1009A00007E24950C808000E4A5402E2C80EB06F70
:1009B0000250005C73E02CB208D0E66A0050E66E8C
:1009C0005FEC64F0E552E66E07D00050E66E6FEC27
:1009D00064F0E552E66EE66A8DECC7F05FD02CB2AB
:1009E00044D04DEC64F0496E640E495C09E34DEC73
:1009F00064F04A6E4B6A4B340DE2ECECCAF00AE24A
:100A00004DEC64F00701266F510E80ECC4F054ECFD
:100A10008EF044D0E66AE66A8DECC7F00201FA0E69
:100A2000B06F0EECCFF005E0D8900D330C33E80634
:100A3000FBE156EC64F0496E640E495C09E356EC48
:100A400064F04A6E4B6A4B3408E2ECECCAF005E203
:100A5000A00EE66E6FEC64F0E55256EC64F0E66EC4
:100A6000E66A8DECC7F02C8219D054EC8EF056EC6F
:100A700064F0496E640E495C09E356EC64F04A6E1A
:100A80004B6A4B340AE2ECECCAF007E256EC64F035
:100A90000701266F540E80ECC4F02C9225822E881C
:100AA000380E0101B55D18E1020E006F080E006EF0
:100AB0008AB102D00E0E006ECCEC25F089C100F098
:100AC0005BECC7F0100E136F158F02018A0EA46F36
:100AD000010EA56F010EA66F110E0101B55D27E194
:100AE000156B15C114F1100E136F0D0E505D03E15F
:100AF000010E146F19D0080E505D02E1050E09D0E9
:100B0000050E505D02E1030E04D0030E505D03E1BB
:100B1000020E156F09D0500507E1010E156F006F29
:100B20000B0E006ECCEC25F00101158F2E883A0ECD
:100B3000B55D17E1020E006F080E006E8AB302D099
:100B40000E0E006ECCEC25F07AC100F05BECC7F025
:100B5000100E136F02018A0EA46F010EA56F020E14
:100B6000A66F360E0101B55D19E1C0EC6BF0050F03
:100B7000D9ECC7F0C0EC6BF0000903E1010184EC93
:100B8000CCF00201860EA46F010EA56FD5ECC7F064
:100B900005E202017B0EA46F010EA56F030E010199
:100BA000B55D0FE170C100F0BAECD9F01E0E010185
:100BB000705D02E184ECCCF00201700EA46F010EB6
:100BC000A56F330E0101B55D11E1855104E10B0EF6
:100BD000CEECC6F006D085C100F0BAECD9F0010128
:100BE000158F0201850EA46F010EA56F040E010181
:100BF000B55D1FE10201310EA46F010EA56F010169
:100C0000040E5AECD2F00101310506E1020E006F2C
:100C10009E0E006ECCEC25F0020E0101315D09E163
:100C2000020E006F850EE66EBF0EE66E010E80ECC2
:100C3000C3F0240E0101B55D11E102018851140DCC
:100C400029ECC4F094ECC8F00101100E116F006B98
:100C5000328A0201880EA46F020EA56F260E0101D2
:100C6000B55D03E0370EB55D34E1F3EC77F0026A71
:100C7000080E025C2EE2015002241EECCDF0006E44
:100C8000100E005C03E07DECC5F002E1020E13D013
:100C90000050120802E2040E0ED00050100802E2CA
:100CA000030E09D00E0E005C02E2006A05D0100EA1
:100CB000005C02E2010E006E410E0024E8ECC4F07C
:100CC000D00FE66E02505DECC4F0BFECC5F0022A16
:100CD000CFD7120E0101B55D0EE1100E146F14C1D5
:100CE00013F1110E156F2ABF152B020188ECCDF000
:100CF000800EA66F2E80420E0101B55D18E1050E33
:100D0000006F52C100F00201520EA46F010EA56FD8
:100D10000101E2A507D04AC100F002014A0EA46F0A
:100D2000010EA56FBAECD9F00101148F2E88390E8F
:100D3000B55D4AE1006B800EE66EBF0EE66E010EF9
:100D400080ECC3F033B603D001010E0E0E6FD5EC6C
:100D5000C7F039E3050E006FD2ECC4F003E119ECE3
:100D6000CDF01FD00101E09DB00E0D252FECC5F098
:100D70000F0E005C03E3005030080DE2230E006EFE
:100D80000901EB510E0807E2310EEB5D04E2EBC9FD
:100D900000F00101E08D0101E0BD03D0005059ECED
:100DA000CEF0BAECD9F00101135102E1100E136F2D
:100DB000D2ECC4F008E00101158F240E136FE0ADF2
:100DC00002D0110E136F2E882D0E0101B55D09E1C1
:100DD0004AEC09F09C0E0E5C630E0F5802E294EC94
:100DE000C8F0B8ECCBF001E028D1006BE3ABF8D051
:100DF000C9ECD1F0D7ECC3F03D50D9ECC7F00101FC
:100E0000240E0E6F9D0E86ECD0F00EC0DEFF0FC0DC
:100E1000DDFFC80E93ECC9F004E3840E57ECC9F073
:100E200004E20701080EA7ECCFF094ECC8F0010132
:100E3000100E116F160E126FE6EC80F0F3CF57F024
:100E4000F4CF58F057C0E6FF58C0E6FF1EECCBF0D9
:100E5000E7CF58F0E552E7CF57F05750F324556EDF
:100E60005850F420566E55C0E6FF56C0E6FF1EEC03
:100E7000CBF0E7CF56F0E552E7CF55F05550F324CD
:100E8000536E5650F420546E53C0E6FF54C0E6FF34
:100E90001EECCBF0E7CF54F0E552E7CF53F05350C0
:100EA000F324516E5450F420526E51C0E6FF52C0EC
:100EB000E6FF1EECCBF0E7CF52F0E552E7CF51F062
:100EC0005150F3244F6E5250F420506E4FC0E6FF45
:100ED00050C0E6FF1EECCBF0E7CF50F0E552E7CF75
:100EE0004FF0BAECC8F01EECCBF0E7CF4EF0E55275
:100EF000E7CF4DF08AECCCF032ECCDF01EECCBF02D
:100F0000E7CF4CF0E552E7CF4BF01EECC5F0030EF7
:100F10000F0B03E06BECC9F0FDE1020E49C0DBFFF3
:100F2000030E4AC0DBFF0101E3AD58D0780EE66E38
:100F3000BF0EE66E010E8FECC3F0020EDBCFD4F1D4
:100F4000030EDBCFD5F101017F0ED880D455050EFD
:100F5000D55505E20701090EA7ECCFF03FD005EC0F
:100F6000CDF0070E53ECC9F0FDE16A0E4924096E7D
:100F7000D4C149F0E2ECD0F0FF0E005C2EE1010E8E
:100F8000DB5097ECC9F0012ADF5097ECC9F0010162
:100F90002A0E1C6F730EE66EBF0EE66E010EC4ECD9
:100FA000C3F0020EDBCFE6FF030EDBCFE6FF8DECD6
:100FB000CDF06F0EE66EBF0EE66E010EC4ECC3F010
:100FC000DECFE6FFDDCFE6FF8DECCDF0680EE66EFE
:100FD000BF0EE66E010EC4ECC3F0096A25822CD068
:100FE00069C11DF16AC11EF16BC11FF16CC120F115
:100FF0000A0E406E416A426A436A1DC13BF01EC13F
:101000003CF01FC13DF020C13EF0ECECFCF03BC0D9
:101010001DF13CC01EF13DC01FF13EC020F1F7ECB8
:10102000D9F021ECDAF00101118F148F0701BEBB5A
:1010300003D00101100E156F2E880490180E0101C7
:10104000B55D06E138BF0480EFECD1F0800EA66FED
:101050000F0E0101B55D09E13E5101E00480E6ECAF
:10106000C9F03E0EA46F010EA56F090E0101B55D1A
:101070000AE196BD0480E6ECC9F0960EA46F010E5D
:10108000A56F400EA66F300E0101B55D22E136ADB1
:1010900015D0C8ECD3F0610EE66EBF0EE66E010E01
:1010A00080ECC3F001013651070B050DF3500A0F18
:1010B000006EBEECD0F091ECCCF004D036BF0480D2
:1010C000DEEC80F00201360EA46F010EA56FC70E94
:1010D000A66F270E0101B55D06E138B50480EFEC7F
:1010E000D1F0040EA66F3F0E0101B55D0AE137B1E4
:1010F0000480E6ECC9F0370EA46F010EA56F010E57
:10110000A66F0B0E0101B55D23E1845106E1050ECA
:10111000006F0B0ECEECC6F015D0C8ECD3F0010179
:10112000840506E1580EE66EBF0EE66E010E08D08D
:10113000020E845D07E14F0EE66EBF0EE66E010EF5
:1011400080ECC3F00201840EA46F010EA56F2E88FF
:10115000160E0101B55D13E1050E006F0E0E006E57
:101160003BA904D04B0E006E040E006F02013B0E33
:10117000A46F010EA56F100EA66FD2EC80F01E0EAC
:101180000101B55D23E156A50BD0006B460EE66E5E
:10119000BF0EE66E010E80ECC3F00101148F0ED07D
:1011A00056A108D0420EE66EBF0EE66E010E80EC30
:1011B000C3F004D00E0E006ECCEC25F00201560EEA
:1011C000A46F010EA56F050EA66F2E800101B5510B
:1011D00006E133B40480DEEC80F02E88328A020E01
:1011E0000101B55D4FE1006B390EE66EBF0EE66E94
:1011F000010E80ECC3F00101006B800507E1300EA9
:10120000E66EBF0EE66E010E80ECC3F0020E010129
:10121000805D07E1270EE66EBF0EE66E010E80ECE4
:10122000C3F0030E0101805D07E11E0EE66EBF0EE6
:10123000E66E010E80ECC3F0040E0101805D07E153
:10124000150EE66EBF0EE66E010E80ECC3F0050EC5
:101250000101805D07E10C0EE66EBF0EE66E010E29
:1012600080ECC3F0060E0101805D07E1030EE66E1F
:10127000BF0EE66E010E80ECC3F00201800EA46F7B
:10128000010EA56F0D0E0101B55D3FE1835106E131
:10129000010E006F440ECEECC6F032D083050DE196
:1012A000010E006FFB0EE66EBE0EE66E010EE66EE0
:1012B00058ECDAF0E552E55206D033AC06D0010E18
:1012C000E66E0CECDDF0E5521BD0030E006FF50E60
:1012D000E66EBE0EE66E010E80ECC3F001018305E2
:1012E000040DF350006EBEECD0F017ECFEF03EC0E3
:1012F00011F13AC012F10101115102E1100E116F0A
:101300000201830EA46F010EA56F2C0E0101B55DC5
:1013100012E10B0E006E04902AB3048004B004D0D6
:10132000010E006F440E006ED2EC80F0020188ECDA
:10133000CDF0020EA66F2E0E0101B55D10E10B0E71
:10134000006E5FAF02D0CF0E006ED2EC80F00201D3
:101350005F0EA46F010EA56F800EA66F2E88310E52
:101360000101B55D08E12AB50480E6ECC9F088EC1E
:10137000CDF0040EA66F0101040E006F1D0EB55DC9
:101380000DE1050E006F020178B90480E6ECC9F0AA
:10139000780EA46F020EA56F100EA66F210E01012C
:1013A000B55D17E18DA908D0050E006FAC0EE66E95
:1013B000BF0EE66E010E06D0006BEC0EE66EBE0EA2
:1013C000E66E010E80ECC3F08CECCAF0800EA66FC6
:1013D0002E80190E0101B55D3CE1C8ECD3F0110E71
:1013E00002017025BAECC5F001010E6F140E020166
:1013F0007025BAECC5F001010F6F0E6A0F6A020189
:10140000705103E1E9ECC7F014D0700506E140EC3F
:1014100020F00101200E106F0CD0020E705D09E16A
:1014200092ECCDF00101395104E0EFC90EF0F0C9A2
:101430000FF00E0ED8800E54270E0F5402E20E6AE3
:101440000F6A94ECC8F00101115102E1100E116F06
:10145000148F0A0EB55D61E1395120E030A213D03E
:10146000040E006F0901E85102E12A0E0FD0E805D1
:1014700008E1E70EE66EBE0EE66E010E80ECC3F0EC
:1014800008D04B0E03D0010E006F440E006ECCEC62
:1014900025F00201E80EA46F090E3ED0DAECBBF095
:1014A0000101010E006F3A5102E1440E0CD03A05E1
:1014B00004E1040E006F2A0E06D0020E3A5D06E12A
:1014C000040E006F4B0ECEECC6F020D0030E3A5D3A
:1014D0001DE33A5113081AE3550ECEECC6F0030E85
:1014E00001013A5D006E080E005C04E21C0E146FF0
:1014F00000280BD0100E005C05E2130E146F070ECF
:10150000005C03D0130E146F240E156F328A2E80E8
:1015100002013A0EA46F010EA56F200E0101B55D08
:1015200017E1395102E10E0E03D0390504E1080E2E
:10153000CEECC6F008D0006BDE0EE66EBE0EE66E98
:10154000010E80ECC3F00201390EA46F010EA56FED
:101550001A0E0101B55D3BE12EA435D0016A1E0EC5
:10156000015C0AE298ECCCF0EF50E66E9FECCCF018
:10157000BFECC5F0012AF3D7D5ECDAF029ECD9F0AD
:101580000101279D269D1750800B0CE1010126517A
:10159000400B08E12751400B05E145EC53F0B7EC57
:1015A00041F0F1D7016A1E0E015C0AE29FECCCF01B
:1015B000EF50E66E98ECCCF0BFECC5F0012AF3D703
:1015C00029ECD9F00101050E5AECD2F0328A2F0E27
:1015D0000101B55D43E1050E5AECD2F02EA23CD0DC
:1015E0000101010E006F2F0ECEECC6F08250010BF0
:1015F00003E08250020B0DE1C8ECD3F00101010EB3
:10160000106F82B202D0040E106F050E006F006AD8
:101610001DD0066A060E065C1EE20650040DF3504D
:101620008309006E050E065C02E1BB0E006E0050E1
:1016300083ECD2F01A080DE2F00E005C0AE2C8EC6E
:10164000D3F006C010F10101050E006FBAECD9F01D
:1016500002D0062ADFD725822E88328AE0ECCDF030
:1016600062E1D5CA03F0CE51010B10E03751080BEF
:101670000DE0040E036E1BA009D0030E036E0A01D9
:101680001C5104E1280E216F21CA1CFA0201D65117
:1016900019E00101170E0E6F010E006F03506AEC86
:1016A000C8F0EF50D9ECC7F00101200E126F050E03
:1016B000006F035070ECC8F0EF50D9ECC7F0010197
:1016C000128F30D0C8ECD3F00501170506E1D90E12
:1016D000E66EBE0EE66E010E05D0D30EE66EBE0EB1
:1016E000E66E010E80ECC3F01BA00AD00101010ED2
:1016F000006FCE0EE66EBE0EE66E010E80ECC3F0FD
:1017000005011751050DAAECCEF0140E49260A0E5C
:101710004A22035014ECD1F05BECC7F0135102E104
:10172000100E136F2E883B0EB55D27E1C8ECD3F089
:1017300022B406D0D90EE66EBE0EE66E010E05D0BE
:10174000D30EE66EBE0EE66E010E80ECC3F02250A4
:10175000040B01E0010E0201A46FA56B910EA427FA
:10176000020EA523C3ECCFF0EF50006E5BECC7F088
:10177000135102E1100E136F2E880E0EB55D1DE1A0
:10178000050E006F51C100F0BAECD9F00101158FC0
:10179000135102E1100E136F0601426B010151510A
:1017A00002010B5D05E20601700E426F5A0E436F97
:1017B0000201510EA46F010EA56F280E0101B55D47
:1017C0000AE1775101E00480E6ECC9F0770EA46FDE
:1017D000010EA56F2E88250E0101B55D1AE1020EDE
:1017E000006F1E0E432556ECD2F00101006B1A0E5D
:1017F000432556ECD2F00101136B100E146F120E3C
:10180000156F0E5102E1100E0E6F0F5102E1100E16
:101810000F6F3D0EB55D17E1050E006F420506E145
:10182000CA0EE66EBE0EE66E010E05D0C60EE66E60
:10183000BE0EE66E010E80ECC3F00201420EA46FF4
:10184000010EA56F2E80130E0101B55D1BE14FA3A4
:1018500005D0040E006F1BECD1F00DD0006B640EB0
:10186000CEECC6F05D0E006E01014FA102D0600EFD
:10187000006ECCEC25F002014F0EA46F010EA56F97
:10188000030EA66F140E0101B55D1EE1040E006F7C
:101890004FBB11D01C0E0E6F160E0F6F240E106F63
:1018A0000D0E116F5D0E006E4FA902D0600E006E1E
:1018B000CCEC25F002D01BECD1F002014F0EA46F4E
:1018C000010EA56F300EA66F320E0101B55D02E16B
:1018D0005DECDCF0080E0101B55D20E1C8ECD3F051
:1018E00001015FB90480DEEC80F0FAECC3F083C341
:1018F0003EF017ECFEF03EC012F13AC013F1FAECE4
:10190000C3F084C33EF091ECCCF00101148F0201CE
:101910005F0EA46F010EA56F100EA66F5CC305F0DD
:10192000055034ECC8F0DEECD0F0430EB55D0BE1B1
:10193000140E006E94ECD3F002E0110E006ED2ECA7
:1019400080F0328A2E88440E0101B55D14E1B5ECB9
:10195000CFF0496E4A6AABECD0F0640D6DECC6F086
:10196000030E006F58EC26F0060EE66E030E8EECAA
:10197000C8F0328A2E88450E0101B55D07E1A6EC5C
:10198000D0F0006E83EC80F0328A2E88470E010181
:10199000B55D12E135ECD2F0006E040EE7ECCCF050
:1019A000100E126F3FECD2F002E10E0E126F3AEC05
:1019B000D2F0156F148F2E88460EB55D1FE12FEC07
:1019C000CFF006E18AECC3F0A6ECCCF00A0803E104
:1019D0008AECC3F0EF928AECC3F0060EEB50006E77
:1019E000005001E1002ABAECD9F00101135102E1E3
:1019F000100E136F180E126F158F2E88480EB55DDE
:101A00001DE18AECC3F0A6ECCCF0006E240E126F40
:101A1000220E136F1E0E146F2FECCFF008E0010E94
:101A20000E6F1E0E0F6F240E106F118F04D000501A
:101A300002E10528006E00C015F12E88129E129C4E
:101A40002E50100B07E01E50040B04E11B50080B36
:101A500001E1128C1F0EB55D03E01B0EB55D05E1C3
:101A6000060EE66E050E8EECC8F0290E0101B55D7E
:101A700008E1135106E1100E136F145102E1100E2C
:101A8000146F040EE15C02E2E16AE552E16E5BEF85
:101A9000C3F018ECCEF00101B551DE6EDD6AD9CF8E
:101AA000E9FFDACFEAFF070EEC02F3CFEDFFEF021A
:101AB000F3CFEEFFF450ED26026AE30E496EDA0E24
:101AC0004A6E010E4B6E0250E76E000EDFCF4CF0F7
:101AD000010EDBCF4DF0E7504C26000E4D2266EC98
:101AE000CFF0006E68ECDAF0022A070E025CE5E344
:101AF000020EE15C02E2E16AE552E16E5BEFC3F0E7
:101B000012000201030E686FA46BA56BA6691996FB
:101B1000B8ECCBF004E1E39DE39BBCEC0AF00601DA
:101B2000426BDFECD7F024B8BFD8E4ECCBF003E095
:101B30003B0EB55D05E12050040B02E06DECC7F0F3
:101B400078EC09F02DA452D02D940D0E0101B55D55
:101B50001DE1339C83C100F00050010813E2000432
:101B6000E66E83ECDCF0E552338CC80E9EECC3F0DD
:101B7000E66A0CECDDF0E552000908E00201020E15
:101B8000686F04D0E66A83ECDCF0E5521EA602D052
:101B900097EC35F01E9634EC0EF047EC0EF024A4D2
:101BA00005D07CECC8F02494DEECCCF01EA80BD061
:101BB0001E980DC1E6FF66EC5AF0E5520DC1E6FF36
:101BC00082EC5AF0E5522EA60CD02E9663EC5BF018
:101BD000D5ECC7F006E28AECC6F00EECD2F064EC6D
:101BE0002EF030AE03D0309E07EC78F018AC03D066
:101BF000189C84ECCDF01E941200B6EC0CF02992E7
:101C00000201355101E1258AA5EC16F02E942E92A1
:101C100009EC0DF00601426B0101B193DFECD7F046
:101C200091EC6FF02D9C0201686B0C0E076EB4EC0A
:101C300063F00101129C3B51010B01E0128C129EDA
:101C40003B51020B01E0128E17A004D0E66A4D0E44
:101C5000E6ECC3F09C0ECEECC3F00101E39DE39BE8
:101C600012000D500101B527B5AF02D0480EB56F77
:101C7000B551480801E2B56B1200230E7CECC4F0AC
:101C8000020E006E1A0E155C05E10050D5ECC4F092
:101C9000320EEF6E12000101AA6BD890A833D890D3
:101CA000A83328962AEFC7F007010B9F07ECF7F03F
:101CB00025ECD0F0209C338677ECCDF0249830ECE6
:101CC000C8F074EF69F0E66AE66A8DECC7F00701C8
:101CD000086B37ECF7F0ACEC16F08A96208C339654
:101CE00077ECCDF007010B8F07EFF7F05FECC3F057
:101CF000100EE1263250200B14E01D50040B02E1BF
:101D00004AEF96F01D50080B02E14AEF96F09CEC6A
:101D1000C6F002E14AEF96F0D2ECC9F002E04AEFD9
:101D200096F002016851030A02E148EF96F0010AB9
:101D30001DE0030A02E04AEF96F02D942E902498BD
:101D40002E98329A189C0101B1830201A46BA56BF5
:101D5000A6691996A3ECDBF01F960101269D279D2D
:101D60000201020E686F25822AEC3DF02950020B19
:101D700016E02E50010B13E02E50100B10E175EC05
:101D80007AF029922F88EDEC80F00101B18DB18FAE
:101D9000640EA86F05EC79F0B4DE57C2B5F117AE4A
:101DA000E5EF95F099ECC8F0D9EC14F0FF0813E0DA
:101DB000F4EC14F0006E0101395105E01B0E005CDB
:101DC00002E122ECD1F00101B19BB199179E25826D
:101DD000238A4AEF96F02E50100B12E01E50040B8F
:101DE0000FE11B50080B0CE1090E155C09E00C0E0D
:101DF000155C03E11750100B03E1EDEC08F004D083
:101E00000B0E155C04E17DDE179E4AEF96F017A0DD
:101E100093EF94F028B697EF94F0090E155C02E169
:101E20009DEF94F0EDECC4F075E01750010B72E0FB
:101E3000100E155C09E0110E155C06E0080E155C2D
:101E400003E0290E155C66E11550DF6E91C2F9F6CC
:101E500092C2FAF68DC2F5F68EC2F6F68FC2F7F68A
